:04000000ADEF00F070
:100008005682D9CF08F0DACF09F00F0112A91BD018
:100018008EBC02D0839483928EA802D083A20ED085
:10002800899425EE04F0010EDBBE07D0000EDE5CDD
:10003800020EDE5802E3899201D089828EB883B21B
:1000480001D08984129912A17CD08EB883B289928A
:10005800901C0A6E8E1C0B6E04C50CF005C50DF0C5
:100068000DBE03D0020E0D5C2FE28EA802D083A233
:100078002BD00C4A0D2A0CC004F50DC005F502C59D
:100088000CF003C50DF0060E0C24D96E050E0D20DC
:10009800DA6E0AC0DFFF060E0C24D96E070E0D209B
:1000A800DA6E0BC0DFFF0C4A0D2A0468010E056EDC
:1000B8000CC006F00DC007F00450061605500716D0
:1000C80006C002F507C003F58EB883B28984898417
:1000D8008EA0FED78EA802D083A202D0899401D028
:1000E800898425EE04F0010EDBBE07D0FE0EDE5C2F
:1000F800010EDE5802E3899201D089820BA81FD035
:100108000BD0838202D0838405D0839418D083A235
:1001180016D08394839213D00A507F0B046E056A1D
:1001280005500DE10450040AF2E0100AF0E0340A28
:10013800E8E01F0AEFE07F0AE6E01F0AE6E00F01A9
:1001480012910E01CA9909C0DAFF08C0D9FF569268
:10015800110036EF4EF07DC0D9FF7EC0DAFFDE6AAF
:10016800DD6A7CC00EF008EC47F00EC098F00FC0B6
:1001780099F0000199BF0B0CD8909835D96E993534
:10018800DA6E820ED926010EDA22DECFAFF0DDCF8D
:10019800B0F0AF51B01101E10C0C7DC0D9FF7EC0A9
:1001A800DAFFAFC0DEFFB0C0DDFF7F91AFC0D9FF7F
:1001B800B0C0DAFFDF5012E020EE01F0AF51D926CF
:1001C800B051DA22DF50D4EC61F00001A46FA4B181
:1001D80005D07F51D8A4A4A5000C0A0CAFC0D9FF44
:1001E800B0C0DAFFDF6A20EE01F0AF51D926B05176
:1001F800DA2298C0DFFF20EE01F0AF51D926B051C6
:10020800DA22DF50AAEC43F00001A46FA4B1030C7A
:100218007F5102E0A4B50A0CAFC060F0B0C061F035
:10022800636B626BA3EC47F060C0ADF061C0AEF0E9
:10023800040EAD19AE1101E1010CAE5103E1020E3D
:10024800AD5D01E30D0C20EE2BF0AF51D926B05176
:10025800DA22DECFA0F0DECFA1F0DECFA2F0DECF33
:10026800A3F03A0EAF250E6E000EB0210F6EC9EC4A
:100278005FF0020E0F180E1001E00D0C450E000184
:10028800AF250E6E000EB0210F6EC9EC5FF00EC0E8
:10029800A9F00FC0AAF00001AB6BAC6BA951AA1171
:1002A800AB11AC1110E1530EAF250E6E000EB0214C
:1002B8000F6E7CEC54F00EC0A9F00FC0AAF010C06D
:1002C800ABF011C0ACF0000120EE17F0AF51D92609
:1002D800B051DA22A9C0DEFFAAC0DEFFABC0DEFF44
:1002E800ACC0DEFF20EE3FF0AF51D926B051DA2284
:1002F80010EE02F0AF51E126B051E222DFCFE7FF66
:1003080020EE02F0AF51D926B051DA22DE040AE01D
:1003180020EE02F0AF51D926B051DA22020EDE18D3
:1003280001E00D0CA9C00EF0AAC00FF0ABC010F090
:10033800ACC011F020EE02F0AF51D926B051DA224C
:10034800DF50126E136A146A156A89EC58F00EC0F1
:10035800A9F00FC0AAF010C0ABF011C0ACF020EEAD
:100368003CF0AF51D926B051DA22DF50806F816B53
:1003780020EE09F0AF51D926B051DA2280C0DEFF55
:1003880081C0DDFF20EE09F0AF51D926B051DA2245
:10039800DE50DE10D8B40D0C20EE09F0AF51D9268E
:1003A800B051DA22DECF80F0DDCF81F08269836937
:1003B80020EE09F0AF51D926B051DA22DECF84F011
:1003C800DDCF85F08251842783518523805184179E
:1003D800815185178451851101E00D0C400EAF2520
:1003E8000E6E000EB0210F6EC9EC5FF0000120EE1A
:1003F80007F0AF51D926B051DA220EC0DEFF0FC088
:10040800DDFF20EE07F0AF51D926B051DA22DF50D8
:10041800806F0F0E801701E00D0C420EAF250E6E97
:10042800000EB0210F6EC9EC5FF00EC09CF00FC03B
:100438009DF000019E6B9F6B9C519D119E119F1119
:1004480010E14F0EAF250E6E000EB0210F6E7CEC42
:1004580054F00EC09CF00FC09DF010C09EF011C06B
:100468009FF03D0E0001AF250E6E000EB0210F6EFD
:10047800C9EC5FF00EC09AF00FC09BF000019A51D2
:100488009B1101E10D0C20EE07F0AF51D926B051B8
:10049800DA22DECF80F0DDCF81F0040E826FD890B3
:1004A80081338033822FFBD79A518025836F9B51EC
:1004B8008121846F856BD8B0852B866BA9518325E4
:1004C800946FAA518421956FAB518521966FAC51D9
:1004D8008621976F94519C5D95519D5996519E59CF
:1004E80097519F5901E20D0C94519C5D0E6E9551E8
:1004F8009D590F6E96519E59106E97519F59116EC6
:1005080020EE09F0AF51D926B051DA22DECF80F0C3
:10051800DDCF81F080C012F081C013F0146A156A33
:1005280045EC59F00EC0A5F00FC0A6F010C0A7F01A
:1005380011C0A8F00001A551A611A711A81101E149
:100548000D0CAD6BAE6BF60EA55DFF0EA659FF0E3A
:10055800A7590F0EA85903E2AE6B030EAD6FA85151
:10056800A71108E1F60EA55DFF0EA65903E2AE6BD2
:10057800020EAD6FA851A71108E1F60EA55D0F0E8A
:10058800A65903E2AE6B010EAD6FAD51AE1101E19C
:100598000D0C020EA525806F000EA621816F000E9E
:1005A800A721826F000EA821836F20EE13F0AF51B0
:1005B800D926B051DA2280C0DEFF81C0DEFF82C0BA
:1005C800DEFF83C0DEFF20EE1BF0AF51D926B0510D
:1005D800DA22A0C0DEFFA1C0DEFFA2C0DEFFA3C0FA
:1005E800DEFF9A51A025806F9B51A121816F000EDB
:1005F800A221826F000EA321836F20EE1FF0AF515E
:10060800D926B051DA2280C0DEFF81C0DEFF82C069
:10061800DEFF83C0DEFF9451A025806F9551A12194
:10062800816F9651A221826F9751A321836F20EE8B
:1006380027F0AF51D926B051DA2280C0DEFF81C041
:10064800DEFF82C0DEFF83C0DEFF030EAD19AE11F0
:100658004DE1590EAF250E6E000EB0210F6EC9EC9C
:100668005FF00E500F1001E00D0C000120EE07F0B6
:10067800AF51D926B051DA22DE50DE1001E00D0C60
:100688005B0EAF250E6E000EB0210F6E7CEC54F0A1
:10069800000120EE23F0AF51D926B051DA220EC066
:1006A800DEFF0FC0DEFF10C0DEFF11C0DEFF20EE50
:1006B80013F0AF51D926B051DA22DECF80F0DECF69
:1006C80081F0DECF82F0DECF83F0020ED890803743
:1006D800813782378337E82EF9D780C090F081C000
:1006E80091F082C092F083C093F0B8D020EE07F06A
:1006F800AF51D926B051DA22DE50DE1001E10D0CDF
:1007080020EE1FF0AF51D926B051DA22DECF80F0AB
:10071800DECF81F0DECF82F0DECF83F0A9518025D5
:10072800846FAA518121856FAB518221866FAC51AC
:100738008321876F20EE23F0AF51D926B051DA22FA
:1007480084C0DEFF85C0DEFF86C0DEFF87C0DEFF17
:10075800020EAD19AE116BE020EE13F0AF51D926A1
:10076800B051DA22DECF80F0DECF81F0DECF82F02A
:10077800DECF83F0010E8015846F856B866B876BE7
:1007880020EE13F0AF51D926B051DA22DECF88F02F
:10079800DECF89F0DECF8AF0DECF8BF0030E880340
:1007A800F3CF8CF0F4CF8DF08E6B8F6B8903F35001
:1007B8008D27F4508E23000E8F238803F3508D2746
:1007C800F4508E23000E8F23030E8A03F3508E27D6
:1007D800F4508F23000E8903F3508E27F4508F2393
:1007E800000E8803F3508E27F4508F23030E8B03DB
:1007F800F3508F27000E8A03F3508F27000E8903CA
:10080800F3508F27000E8803F3508F27D8908F332B
:100818008E338D338C3384518C25906F85518D2187
:10082800916F86518E21926F87518F2116D020EEBD
:1008380013F0AF51D926B051DA22DECF80F0DECFE7
:1008480081F0DECF82F0DECF83F0D8908035906FD4
:100858008135916F8235926F8335936FFF0E9025A6
:10086800806F010E9121816F000E9221826F000E20
:100878009321836F0A0E05D0D89083338233813356
:100888008033E82EF9D720EE17F0AF51D926B051B2
:10089800DA228051DE5C8151DE588251DE58835164
:1008A800DE5801E20D0C20EE0FF0AF51D926B05101
:1008B800DA22DE68DE68DE68DD68DD52DD5210EEC1
:1008C8000BF0AF51E126B051E222DECFE6FFDECFDA
:1008D800E6FFDECFE6FFDECFE6FF20EE04F0AF5105
:1008E800D926B051DA22800EDF6E030EAD19AE1193
:1008F80001E090D05F0EAF250E6E000EB0210F6E96
:10090800C9EC5FF00E040F1001E084D0AFC03AF0DC
:10091800B0C03BF0010E0001A0253C6E000EA121E5
:100928003D6E000EA2213E6E000EA3213F6E71ECBB
:1009380055F000096FE1000120EE04F0AF51D9260F
:10094800B051DA22DF6A2D0EAF250E6E020EB021ED
:100958000F6EC9EC5FF0550E0E185CE1AA0E0F1869
:1009680059E12F0E0001AF250E6E000EB0210F6E5B
:100978007CEC54F0520E0E184DE1520E0F184AE15D
:10098800610E101847E1410E111844E1130E0001E1
:10099800AF250E6E020EB0210F6E7CEC54F0720E75
:1009A8000E1838E1720E0F1835E1410E101832E1B9
:1009B800610E11182FE1170E0001AF250E6E020E01
:1009C800B0210F6E7CEC54F0000120EE0FF0AF5117
:1009D800D926B051DA220EC0DEFF0FC0DEFF10C0EC
:1009E800DEFF11C0DEFF1B0EAF250E6E020EB0211A
:1009F8000F6E7CEC54F0000120EE0BF0AF51D926BD
:100A0800B051DA220EC0DEFF0FC0DEFF10C0DEFFDD
:100A180011C0DEFFAFC0D9FFB0C0DAFFADC0DFFF45
:100A28000101804B812B000120EE05F0AF51D92642
:100A3800B051DA2280C1DEFF81C1DDFF000C77C032
:100A48007AF078C07BF00101766B776B96D376C02D
:100A580060F07A0E0001616F79C062F06151D96E61
:100A6800DA6ADECFF6FFDDCFF7FFF86A000EF86E20
:100A78000800F550250AD8A45ED36151D96EDA6A08
:100A8800DE2A000EDD220101786B796B4C6A4D6A13
:100A98007A697B6900016151D96EDA6ADECFF6FFA7
:100AA800DDCFF7FFF86A000EF86E0800F550640A0B
:100AB800D8B40FD06151D96EDA6ADECFF6FFDDCF38
:100AC800F7FFF86A000EF86E0800F550690AD8A416
:100AD8007DD16151D96EDA6ADE2A000EDD226251BB
:100AE800D96EDA6ADF50DF2ADF2AD96EDA6ADECFFA
:100AF80065F0DDCF66F0000E66BFFF0E676F686FAA
:100B0800696F6A6F6B6F6C6F60C028F065C029F001
:100B180066C02AF067C02BF068C02CF069C02DF0C1
:100B28006AC02EF06BC02FF06CC030F029C041F0C5
:100B38002AC042F02BC043F02CC044F02DC045F031
:100B48002EC046F02FC047F030C048F048AE02D063
:100B5800010E01D0000E3F6E406A3F504010D8B4DD
:100B680010D0481E471E461E451E441E431E421EE8
:100B7800416C000E4222432244224522462247224B
:100B8800482201017BBF01D04C927BBF05D07B512D
:100B980007E17A05D8B004D03C6A010E3B6E04D058
:100BA8007AC13BF07BC13CF078C13DF079C13EF0A1
:100BB8003F504010D8A402D04CA403D03D06D8A082
:100BC8003E064A6A1F0E496E0301B36B6ED0490692
:100BD800D8A04A06940E4924D96E030E4A20DA6E2C
:100BE80041C00EF042C00FF043C010F044C011F0F5
:100BF80045C012F046C013F047C014F048C015F0C5
:100C08000A0E166E176A186A196A1A6A1B6A1C6A2B
:100C18001D6A13EC4BF00EC031F00FC032F010C05B
:100C280033F011C034F012C035F013C036F014C0E0
:100C380037F015C038F031C020F033C021F014EC83
:100C480060F02050300FDF6E3B06D8A03C063D0612
:100C5800D8A03E0641C00EF042C00FF043C010F0CD
:100C680044C011F045C012F046C013F047C014F05C
:100C780048C015F00A0E166E176A186A196A1A6AB9
:100C88001B6A1C6A1D6A66EC46F00EC041F00FC074
:100C980042F010C043F011C044F012C045F013C038
:100CA80046F014C047F015C048F04ABE1FD04A505D
:100CB80003E14904D8A01AD041504210431044100F
:100CC8004510461047104810D8A481D73CBE05D01F
:100CD8003C5002E13B04D8B07AD73EBE07D03E5024
:100CE80003E13D04D8A002D04CB271D73F50401068
:100CF800D8A402D04CA415D04906D8A04A063F5023
:100D08004010D8A403D03A6A2B0E02D03A6A2D0EAE
:100D1800396E940E4924D96E030E4A20DA6E39C012
:100D2800DFFF28C01DF0940E49241E6E030E4A20D2
:100D38001F6E3DC020F03EC021F04CA008D01EC060
:100D480017F01FC018F01DC019F02CEC60F021BE80
:100D580005D020C025F021C026F002D0256A266AD9
:100D6800236A246A0AD0000E106E200E0F6E1DC072
:100D780011F002EC58F0234A242A2550235C245011
:100D8800800A226E2650800A2258D8A0ECD74CB090
:100D980008D01EC017F01FC018F01DC019F02CECA9
:100DA80060F01EC00EF01FC00FF00AEC5EF0255078
:100DB8000E241D6E26500F201E6E1DC028F01EC06A
:100DC80029F028C060F029C061F0CFD16151D96EF7
:100DD800DA6ADECFF6FFDDCFF7FFF86A000EF86EAD
:100DE8000800F550780AD8B40FD06151D96EDA6A84
:100DF800DECFF6FFDDCFF7FFF86A000EF86E0800C9
:100E0800F550580AD8A46CD16151D96EDA6ADECF90
:100E1800F6FFDDCFF7FFF86A000EF86E0800F5CF91
:100E280075F06151D96EDA6ADE2A000EDD22625150
:100E3800D96EDA6ADF50DF2ADF2AD96EDA6ADECFA6
:100E480063F0DDCF64F063C06DF064C06EF06F6B6B
:100E5800706B716B726B736B746B60C027F06DC0D5
:100E680028F06EC029F06FC02AF070C02BF071C056
:100E78002CF072C02DF073C02EF074C02FF075C026
:100E880030F001017BBF01D04C927BBF05D07B5174
:100E980007E17A05D8B004D03A6A010E396E04D059
:100EA8007AC139F07BC13AF078C143F079C144F096
:100EB8004CA804D0FE0E4326FF0E442228C03BF067
:100EC80029C03CF02AC03DF02BC03EF02CC03FF0BA
:100ED8002DC040F02EC041F02FC042F0486A1F0ECE
:100EE800476E0301B36B6DD04706D8A048060F0EB6
:100EF8003B14456E466A46BE08D0465004E10A0EC9
:100F0800455CD8A002D0570E01D0300E4526000E01
:100F18004622BF0E316E32683050336E346A31501B
:100F2800332632503422345005E11A0E335C02E283
:100F3800010E01D0000E356E366A35503610D8B421
:100F480025D09F0E316E3268200E4510336E000E8C
:100F58004610346E3150332632503422345005E175
:100F68001A0E335C02E2010E01D0000E376E386AA9
:100F780037503810D8B40AD045C014F046C015F020
:100F8800C7EC5DF014C045F015C046F0940E472438
:100F9800D96E030E4820DA6E45C0DFFF3906D8A0A7
:100FA8003A064306D8A04406040E316ED890423261
:100FB800413240323F323E323D323C323B32312EBA
:100FC800F5D748BE20D0485004E1020E475CD8A0AF
:100FD8001AD03B503C103D103E103F1040104110BD
:100FE8004210D8A481D73ABE05D03A5002E139045C
:100FF800D8B07AD744BE07D0445003E14304D8A000
:1010080002D04CB271D74CA816D04706D8A04806D3
:10101800940E4724D96E030E4820DA6E30C0DFFFE5
:101028004706D8A04806940E4724D96E030E4820D8
:10103800DA6E300EDF6E27C01DF0940E47241E6E48
:10104800030E48201F6E43C020F044C021F04CA07E
:1010580008D01EC017F01FC018F01DC019F02CECE6
:1010680060F021BE05D020C025F021C026F002D0B6
:10107800256A266A236A246A0AD0000E106E200E9A
:101088000F6E1DC011F002EC58F0234A242A255097
:10109800235C2450800A226E2650800A2258D8A049
:1010A800ECD74CB008D01EC017F01FC018F01DC0F8
:1010B80019F02CEC60F01EC00EF01FC00FF00AEC07
:1010C8005EF025500E241D6E26500F201E6E1DC08A
:1010D80027F01EC028F027C060F028C061F045D076
:1010E8006151D96EDA6ADECFF6FFDDCFF7FFF86A15
:1010F800000EF86E0800F550250AD8A413D06151E7
:10110800D96EDA6ADE2A000EDD22000E106E250E78
:101118000F6E60C011F002EC58F00001616B010E17
:10112800606F23D06151D96EDA6ADE2A000EDD22A3
:10113800606B616B1AD06151D96EDA6ADECFF6FF47
:10114800DDCFF7FFF86A000EF86E0800F5500F6E55
:10115800106A60C011F002EC58F000016151D96EBC
:10116800DA6ADE2A000EDD22D8D7000160510101BB
:10117800762700016151010177237AC0F6FF7BC011
:10118800F7FF0800F55001E062D476C176F077C128
:1011980077F01200A0C0B6F0A1C0B7F0A451D96E84
:1011A800DA6ADE6ADD6A9EC00FF09FC010F0C60ED4
:1011B800116E26EC54F00001B56FB5510AE120EE2E
:1011C8000FF09E51D9269F51DA22DF50B56FB551E5
:1011D80002E0B551120020EE0EF09E51D9269F5123
:1011E800DA22DFA2070C20EE10F09E51D9269F517B
:1011F800DA2210EE10F09E51E1269F51E222E6CF4E
:10120800A9F0E6CFAAF0E6CFABF0E6CFACF0A2515A
:10121800A925AD6FA351AA21AE6F000EAB21AF6F08
:10122800000EAC21B06FDE50AD5DDE50AE59DE5021
:10123800AF59DE50B05901E3DFD220EE10F09E51D5
:10124800D9269F51DA22DECFA5F0DDCFA6F0A51D65
:10125800A26FA61DA36FD0D220EE10F09E51D92602
:101268009F51DA22FF0EDE14A56F010EDE14A66F61
:10127800000EDE14A76F000EDE14A86FA551A6118C
:10128800A711A81101E0FDD120EE10F09E51D9263A
:101298009F51DA22DECFA5F0DECFA6F0DECFA7F091
:1012A800DECFA8F00A0E05D0D890A833A733A6330E
:1012B800A533E82EF9D7A969AA6920EE09F0C65125
:1012C800D926C751DA22DECFABF0DDCFACF0A95179
:1012D800AB27AA51AC23A551AB15B86FA651AC15D5
:1012E800B96FB81101E091D020EE10F09E51D926C7
:1012F8009F51DA22DE50DE10DE10DE101EE120EEF5
:1013080006F09E51D9269F51DA22DECFC0F0DECFFB
:10131800C1F0DECFC2F0DECFC3F0C051C111C2119F
:10132800C31127E19EC081F09FC082F0836B846B5C
:10133800856B866B30EC25F014D09EC081F09FC081
:1013480082F020EE14F09E51D9269F51DA22DECF8A
:1013580083F0DECF84F0DECF85F0DECF86F030EC90
:1013680025F081C0C0F082C0C1F083C0C2F084C043
:10137800C3F0C051C111C211C31101E141D2C0056E
:10138800C111C211C31109E120EE0FF09E51D926F7
:101398009F51DA22020EDF6E020CC0290FE1C1292B
:1013A8000DE1C2290BE1C32909E120EE0FF09E519E
:1013B800D9269F51DA22010EDF6E010C20EE14F0BF
:1013C8009E51D9269F51DA22C0C0DEFFC1C0DEFF80
:1013D800C2C0DEFFC3C0DEFF20EE06F09E51D92654
:1013E8009F51DA22DE50DE10DE10DE100EE120EE14
:1013F80006F09E51D9269F51DA22C0C0DEFFC1C037
:10140800DEFFC2C0DEFFC3C0DEFF20EE18F09E5133
:10141800D9269F51DA2210EE2BF0C651E126C7518A
:10142800E222DE50E61812E1DE50E6180FE1DE5047
:10143800E6180CE1DE50E61809E1C6C027F0C7C07F
:1014480028F068EC44F0000901E053D1C6C00EF062
:10145800C7C00FF0000120EE14F09E51D9269F510D
:10146800DA22DECF10F0DECF11F0DECF12F0DECFC1
:1014780013F0A1EC4BF00EC0BCF00FC0BDF010C0D3
:10148800BEF011C0BFF00001BC51BD11BE11BF11AB
:1014980001E17AD7B851BC27B951BD23000EBE234C
:1014A800BF23A2C0A5F0A3C0A6F0090EA76FD890CD
:1014B800A633A533A72FFBD7A5C0BAF0A6C0BBF0AB
:1014C800BA51BB1101E1A2D0BA51B825A56FBB51E1
:1014D800B921A66F20EE09F0C651D926C751DA22E4
:1014E800A551DE5CA651DE5810E220EE09F0C65187
:1014F800D926C751DA22DECFA5F0DDCFA6F0B85144
:10150800A55DBA6FB951A659BB6FB6C01DF0B7C07B
:101518001EF0BCC01FF0BDC020F0BEC021F0BFC08F
:1015280022F0BAC023F0BBC024F020EE01F0C6516F
:10153800D926C751DA22DF5094EC50F0000901E0B7
:10154800D8D00001BA51A56FBB51A66FA76BA86B85
:1015580020EE2BF0C651D926C751DA22DECFA9F0EA
:10156800DECFAAF0DECFABF0DECFACF0BC51A95D88
:10157800AD6FBD51AA59AE6FBE51AB59AF6FBF51D8
:10158800AC59B06FA551AD5DA651AE59A751AF5931
:10159800A851B0592CE22F0EC6250E6E000EC72199
:1015A8000F6E20EE2BF0C651D926C751DA22DECFB6
:1015B800A5F0DDCFA6F0BC51A55FBD51A65B090E15
:1015C800D890A537A637E82EFBD7A551B625106EBB
:1015D800A651B721116E020E136E126A2BEC5EF043
:1015E80020EE03F0C651D926C751DA22DF6ABAC005
:1015F800A5F0BBC0A6F0090ED890A537A637E82EEF
:10160800FBD7A5C0C4F0A6C0C5F0A7D020EE0AF04D
:101618009E51D9269F51DA2210EE10F09E51E126F4
:101628009F51E222DE50E65CDE50E658DE50E65876
:10163800DE50E65818E3C6C027F0C7C028F068ECAB
:1016480044F0000901E055D0000120EE2BF0C6510E
:10165800D926C751DA22BCC0DEFFBDC0DEFFBEC03E
:10166800DEFFBFC0DEFF20EE18F09E51D9269F5145
:10167800DA22BCC0DEFFBDC0DEFFBEC0DEFFBFC0D9
:10168800DEFFA569010EA66F20EE10F09E51D92647
:101698009F51DA22DECFA7F0DDCFA8F0A551A7171A
:1016A800A651A817A7510008C46FA851D8A0E82AC6
:1016B8000208C56FC451A25DC551A35904E2A2C076
:1016C800C4F0A3C0C5F0C6C03AF0C7C03BF020EED6
:1016D80018F09E51D9269F51DA22DECF3CF0DECF9A
:1016E8003DF0DECF3EF0DECF3FF071EC55F0000963
:1016F80002E000015AD60001A569010EA66F20EE8E
:1017080010F09E51D9269F51DA22DECFA7F0DDCF07
:10171800A8F0A551A717A651A817C6C0A9F0C7C019
:10172800AAF0A751A927A851AA232F0EA9250E6E02
:10173800000EAA210F6EB6C010F0B7C011F0C4C0D9
:1017480012F0C5C013F02BEC5EF020EE03F0C6518A
:10175800D926C751DA22010EDF6EC451A25FC551E6
:10176800A35BA451D96EDA6AC451DE26C551DD22C5
:10177800C451B627C551B72320EE10F09E51D92683
:101788009F51DA22C451DE26C551DE22000EDE2228
:10179800DE2220EE10F09E51D9269F51DA2210EE5B
:1017A8000AF09E51E1269F51E222DE50E65CDE50AF
:1017B800E658DE50E658DE50E65820EE0AF0D8A08B
:1017C80020EE10F09E51D9269F51DA22DECFB1F0DB
:1017D800DECFB2F0DECFB3F0DECFB4F020EE0AF009
:1017E8009E51D9269F51DA22B1C0DEFFB2C0DEFF7A
:1017F800B3C0DEFFB4C0DEFFA251A31101E02CD5B7
:1018080020EE0EF09E51D9269F51DA22000EDB8C75
:10181800000C0F6E0E6AB4D20F5009E1515007E068
:101828000E6A01017F6B0A0EA6D083901BD3020EAD
:101838000F1807E1515005E00E6A01017F6B140E85
:101848009AD01F0E0F6438D0300E0F6035D051502B
:1018580033E00F50E00F526E0E6A0F0E521805E17A
:101868008DC150F001018D6B6DD25250220D420E88
:10187800F324D96E020EF420DA6EDE50DE10DE108C
:10188800DE1003E0030E52645DD2526A010E506E00
:1018980052501C0D1B0EF324D96E010EF420DA6E83
:1018A80052501C0D1B0EF324E16E010EF420E26E63
:1018B800E7501009DF6E46D23F0E0F6428D0500E55
:1018C8000F6025D0515023E052501C0D000EF32418
:1018D800D96E010EF420DA6E0F50C00FDF6E525031
:1018E8001C0D000EF324D96E010EF420DA6EDF50C1
:1018F8000CE052501C0D1B0EF324D96E010EF4207F
:10190800DA6E100EDF6E010E506E0E6A1BD2310EAB
:101918000F1807E1515005E00C0E01017F6F1D0EF5
:1019280026D2340E0F1807E1515005E001017E6BF5
:101938007F6B0E6A7AD7350E0F1808E1515006E012
:101948000E6A0D0E01017F6FAC0E15D0370E0F1801
:1019580008E1515006E083800E0E01017F6F750E7D
:1019680006D20D0E0F1809E1515007E00E6A020E5B
:1019780001017F6FBC0E7E6F58D7100E0F1807E15C
:10198800515005E0030E01017F6FE90EF0D1180EEA
:101998000F1807E1515005E0070E01017F6F090E8E
:1019A800E6D13B0E0F1807E1515005E00E0E01017C
:1019B8007F6F7E0EDCD13E0E0F1801E053D25150DE
:1019C80001E150D20F0E01017F6F3D0ED0D1525070
:1019D8001C0D010EF324D96E010EF420DA6E0FC02F
:1019E800DFFF030E01017F6FEA0EC1D152501C0DBB
:1019F800020EF324D96E010EF420DA6E0FC0DFFF59
:101A0800030E01017F6FEB0EB2D152501C0D030E75
:101A1800F324D96E010EF420DA6E0FC0DFFF030E37
:101A280001017F6FEC0EA3D152501C0D040EF3245C
:101A3800D96E010EF420DA6E0FC0DFFF030E01012C
:101A48007F6FED0E94D152501C0D050EF324D96E04
:101A5800010EF420DA6E0FC0DFFF030E01017F6F65
:101A6800EE0E85D152501C0D060EF324D96E010ED0
:101A7800F420DA6E0FC0DFFF52501C0D060EF3245F
:101A8800D96E010EF420DA6EDF50606F60C061F02D
:101A9800626B636B646B63C064F062C063F061C0C7
:101AA80062F0616B61C065F062C066F063C067F0A8
:101AB80064C068F0696B68BF696969C06AF069C029
:101AC8006BF069C06CF052501C0D050EF324D96EF2
:101AD800010EF420DA6EDF506D6F6DC06EF06F6B23
:101AE800706B716B6FC071F06EC070F06F6B6E6B66
:101AF8006EC072F06FC073F070C074F071C075F092
:101B0800766B75BF766976C077F076C078F076C068
:101B180079F052501C0D040EF324D96E010EF420F6
:101B2800DA6EDF507A6F7AC07BF07C6B7D6B7E6BF0
:101B38007BC07EF07D6B7C6B7B6B7BC07FF07CC059
:101B480080F07DC081F07EC082F0836B82BF8369A4
:101B580083C084F083C085F083C086F052501C0D8A
:101B6800030EF324D96E010EF420DA6EDF50876F6E
:101B780087C088F0896B8A6B8B6B8C6B8D6B8E6BD7
:101B88008F6B200ED890883789378A378B378C37F8
:101B98008D378E378F37E82EF5D77F518825906F90
:101BA80080518921916F81518A21926F82518B21B5
:101BB800936F83518C21946F84518D21956F85513A
:101BC8008E21966F86518F21976F72519025986F4D
:101BD80073519121996F745192219A6F7551932184
:101BE8009B6F765194219C6F775195219D6F785109
:101BF80096219E6F795197219F6F65519825A06F07
:101C080066519921A16F67519A21A26F68519B2152
:101C1800A36F69519C21A46F6A519D21A56F6B51D7
:101C28009E21A66F6C519F21A76F52501C0D070E65
:101C3800F324D96E010EF420DA6EA0C0DEFFA1C035
:101C4800DEFFA2C0DEFFA3C0DEFFA4C0DEFFA5C08A
:101C5800DEFFA6C0DEFFA7C0DEFF839001017E6B1A
:101C68007F6B00D152501C0D1A0EF324D96E010E51
:101C7800F420DA6E0FC0DFFF070E01017F6F0A0E36
:101C880076D052501C0D190EF324D96E010EF42093
:101C9800DA6E0FC0DFFF070E01017F6F0B0E67D0F2
:101CA80052501C0D180EF324D96E010EF420DA6E72
:101CB8000FC0DFFF070E01017F6F0C0E58D0525086
:101CC8001C0D170EF324D96E010EF420DA6E0FC026
:101CD800DFFF38D001017E6B7F6B506AA6D50FC03D
:101CE80030F20F0E01017F6F3E0E41D00FC031F26E
:101CF8000F0E01017F6F3F0E3AD00FC032F20F0E68
:101D080001017F6F400E33D00FC033F20F0E010177
:101D18007F6F410E2CD00FC034F20F0E01017F6F80
:101D2800420E25D00FC035F20F0E01017F6F430E12
:101D38001ED00FC036F20F0E01017F6F440E17D070
:101D48000FC037F201017E6B7F6B6FD50C0E01015E
:101D58007F6F1E0E0CD00C0E01017F6F1C0E7E6F64
:101D68000A0E0E6E62D50E0E01017F6F760E7E6F23
:101D780079D001017E6B7F6B090E0E6E838072D065
:101D88007EC160F07FC161F00001615111E0030A7A
:101D980013E0040A25E00B0A31E0010A35E0030AE2
:101DA80039E0010A40E0130A58E03B0A59E05AD0EA
:101DB800605101E131D556D06051E90A01E107D6F9
:101DC800030A01E113D6010A01E11FD6070A01E15E
:101DD8002BD6010A01E137D6030A01E143D642D0E6
:101DE8006051090A01E13ED7030A01E14AD7010A15
:101DF80001E156D7070A01E162D734D060511D0AC4
:101E0800A5E0030AA8E02ED06051480A01E126D7D0
:101E1800E40A28D06051750AA6E0030AAAE0080A75
:101E280001E158D71FD060513D0A01E158D7030A94
:101E380001E15CD7010A01E160D77F0A01E164D7BB
:101E4800010A01E168D7030A01E16CD7010A01E13F
:101E580070D7070A01E174D705D060512A0A02D069
:101E680060510F0A0E5012000F6A0E6A84EC61F07E
:101E78000101FC6F916B070E8C6E010EFB6F976B67
:101E88000F0E0F01596F116B196B216B266B2E6B9F
:101E98000E6B166B1E6B236B2B6B886889688A68C0
:101EA8008A8E889088928382020E026E9BEC60F084
:101EB80088948384889C839C889E838E8B68896899
:101EC8006A0E00019C6FF90E9D6FA70E9E6FFF0EA4
:101ED8009F6FBA0EA06FFE0EA16F0E0EA26FFF0EBF
:101EE800A36FB1EC61F08A988588E3EC5FF0820E0D
:101EF80000019C6FFB0E9D6FFCC19EF09F6BB1ECC7
:101F080061F00101FC2901E1FC6B0F0EFC17B0EC3C
:101F18004CF00101FC6F9A0E00019C6FFB0E9D6F47
:101F2800FCC19EF09F6BB1EC61F00400520E010100
:101F3800EB6F2B0EEA6F000EE82EFED7EA2FFCD7C8
:101F4800EB2FFAD700F0D250F00B0109D26ED09ED9
:101F58000E01C691CF0ECF16CF82CF80C2890F0156
:101F6800138113891489F28E0E01BA8963EC5AF031
:101F78008392839421EC50F021EC50F0000E0E6E09
:101F8800340E56EC5DF03B0E126EFF0E136ECCEC69
:101F980058F0A70E126EFF0E136ECCEC58F0000E20
:101FA8000E6E390E56EC5DF08FA22FD0290E01016E
:101FB800EB6F960EEA6F7F0EE82EFED7EA2FFCD75E
:101FC800EB2FFAD7000E0E6E800E56EC5DF02C0E3D
:101FD800126EFE0E136ECCEC58F017D06E0E000188
:101FE8009C6FFE0E9D6F8FCF9EF09F6BB1EC61F0E2
:101FF800290E0101EB6F960EEA6F7F0EE82EFED7D1
:10200800EA2FFCD7EB2FFAD704008FB2E7D78380EB
:10201800040085EC4AF00101EF6F93EC33F0010105
:10202800EF6FFB050EE195510CE1590E00019C6F15
:10203800FD0E9D6FB1EC61F0020E0101956F220E4D
:10204800946FFB510EE195510CE1490E00019C6F14
:10205800FD0E9D6FB1EC61F0010E0101956F040E4C
:10206800946F905102E03AEC41F0F9C193FF4FECC4
:1020780030F049EC52F0000E0E6E800E56EC5DF01A
:10208800C5EC60F0000E0E6E800E56EC5DF001019E
:10209800FC510F0D350EF324126E0D0EF420136E45
:1020A800CCEC58F0010197BFC3EC45F00101EE6B91
:1020B800F46B000EF26F010EF16FF2BF05D0F25112
:1020C80066E1040EF15D63E20F0EF103F3CFEAF16E
:1020D800F4CFEBF1F203F350EB27250EEA250E6E51
:1020E8000E0EEB210F6E0AEC5EF00F5003E1030EAB
:1020F8000E5C49E3B60E00019C6FFD0E9D6F0F0E3E
:102108000101F103F3CFEAF1F4CFEBF1F203F3505D
:10211800EB27250EEA2500019E6F0E0E0101EB212B
:1021280000019F6FB1EC61F0220E0101F103F3CFC2
:10213800EAF1F4CFEBF1F203F350EB27380EEA257E
:102148000001CE6F020E0101EB210001CF6F0F0ECF
:102158000101F103F3CFECF1F4CFEDF1F203F35009
:10216800ED27250EEC250001D06F0E0E0101ED21A3
:102178000001D16F030ED26F2CEC15F00101EF6F47
:10218800EF5105EC5DF00101F14BF22B96D792056A
:1021980002E1070E8C6E020E921901E03FD10F0189
:1021A800108B070E2D6F3AD18EA88994A3EC5DF0A1
:1021B8002150221001E106D1F4C1F0F1F30E0E6EA8
:1021C800010E0F6EBEEC57F00101F46FF3B9F49FE6
:1021D80097511BE0350EF41907E1980E00019C6F2A
:1021E800F90E9D6FB1EC61F0290E00019C6FFF0E96
:1021F8009D6FF4C19EF09F6B0101010EF3A9000EC3
:102208000001A06FA16BB1EC61F00101F3A947D007
:10221800600EF41944E15F0EF01941E1790E0001F6
:102228009C6FFC0E9D6FF4C19EF09F6BF0C1A0F0F7
:10223800A16B010E8EA2000EA26FA36B010E8EA4DD
:10224800000EA46FA56BB1EC61F002500209026E9A
:10225800170E9C6FFF0E9D6F95C19EF09F6BB1ECA2
:1022680061F0200E9C6FFF0E9D6F94C19EF09F6BD6
:10227800B1EC61F02BEE35F095C1DFFF2BEE36F0B7
:1022880094C1DFFF8384020E9AEC5AF08394029281
:102298000101996B5DEC61F00101F46BBFD0FB515A
:1022A80046E0F351100B0001C26F000EC36F01012D
:1022B800F451D2EC39F0C2C0F5F1C3C0F6F1080E02
:1022C8000101F519F61101E100F0070E0101F519F8
:1022D800F61102E1D5EC5BF0F505F61102E1E0EC50
:1022E80051F0020E0101F519F61102E1D9EC38F0AE
:1022F800030E0101F519F61104E11DEC2BF00101A3
:10230800EE6F050EF519F61104E1C1EC3BF0010181
:10231800EE6F090EF519F61102E1CAEC53F00A0E38
:102328000101F519F6117AE1DAEC61F077D0F35191
:10233800100B216E000E226EF451BDEC1CF021C072
:10234800F5F122C0F6F1070E0101F519F61102E1C7
:1023580071EC5BF0020EF519F61102E13CEC5BF052
:10236800F505F61102E17CEC1AF0030EF519F611E9
:1023780002E176EC51F0040EF519F61102E1B0EC29
:1023880060F0050EF519F61102E12BEC4CF0060E83
:102398000101F519F61102E1E2EC61F0080EF519F8
:1023A800F61102E177EC3FF0090EF519F61102E19A
:1023B800ACEC4FF00A0E0101F519F6112FE1ACEC67
:1023C8005EF02CD0B0EC4CF00101916F925126E0F8
:1023D800FC51911923E0838E000E0E6EC00E56EC50
:1023E8005DF0C5EC60F0000E0E6EC00E56EC5DF0B0
:1023F800DD0E126EFE0E136ECCEC58F091C1FCF19E
:10240800380E00016D6F020E6E6FE9EC5EF093EC12
:1024180033F00101905102E03AEC41F08FB22ED036
:10242800050E0101EE192AE0BFD66E0E00019C6F61
:10243800FE0E9D6F8FCF9EF09F6BB1EC61F0290E61
:102448000101EB6F960EEA6F7F0EE82EFED7EA2F9A
:10245800FCD7EB2FFAD70400000E0E6EC00E56EC18
:102468005DF0C5EC60F0000E0E6EC00E56EC5DF02F
:10247800430E126EFF0E136ECCEC58F08FB2D5D708
:10248800090E0101EB6F1E0EEA6FE40EE82EFED76F
:10249800EA2FFCD7EB2FFAD700F083948392000140
:1024A800B16BB26B9A0EB36FF90EB46FB56BE8EC03
:1024B80056F0AED59EC00FF09FC010F0BC0E116E46
:1024C80026EC54F00001BE6FBE5108E120EE0FF07B
:1024D8009E51D9269F51DA22DF50BE6FBE5102E0CD
:1024E800BE51120020EE0AF09E51D9269F51DA22E1
:1024F800A051DE5CA151DE58A251DE58A351DE582E
:1025080016E220EE0EF09E51D9269F51DA22DFB254
:102518000ED020EE0AF09E51D9269F51DA22DECF46
:10252800A0F0DECFA1F0DECFA2F0DECFA3F020EE48
:1025380010F09E51D9269F51DA22DECFB4F0DECFBB
:10254800B5F0DECFB6F0DECFB7F0B86BB96BBA6BCB
:10255800BB6B20EE10F09E51D9269F51DA22B8C0ED
:10256800DEFFB9C0DEFFBAC0DEFFBBC0DEFFA05190
:10257800A111A211A31101E100D220EE09F0BC5172
:10258800D926BD51DA22DECFA4F0DDCFA5F0A451C3
:10259800A66FA551A76FA86BA96B090ED890A6378F
:1025A800A737A837A937E82EF9D7A6C0BFF0A7C024
:1025B800C0F0A8C0C1F0A9C0C2F0B451B511B6119D
:1025C800B71101E196D0FF0EA0250E6EFF0EA121D6
:1025D8000F6EFF0EA221106EFF0EA321116EBFC059
:1025E80012F0C0C013F0C1C014F0C2C015F045EC21
:1025F80059F00EC0A4F00FC0A5F010C0A6F011C08D
:10260800A7F0FF0E0001B4250E6EFF0EB5210F6E68
:10261800FF0EB621106EFF0EB721116EBFC012F06B
:10262800C0C013F0C1C014F0C2C015F045EC59F099
:102638000E500001A45D0F50A5591050A659115015
:10264800A75957E3FF0EBF25A46FFF0EC021A56F42
:10265800FF0EC121A66FFF0EC221A76FA41DA86F90
:10266800A51DA96FA61DAA6FA71DAB6FFF0EB425E8
:10267800AC6FFF0EB521AD6FFF0EB621AE6FFF0E2A
:10268800B721AF6FA851AC15B06FA951AD15B16F97
:10269800AA51AE15B26FAB51AF15B36F20EE10F063
:1026A8009E51D9269F51DA22B0C0DEFFB1C0DEFFAD
:1026B800B2C0DEFFB3C0DEFF20EE10F09E51D92677
:1026C8009F51DA22DE50A05FDE50A15BDE50A25B94
:1026D800DD50A35B20EE14F09E51D9269F51DA22DB
:1026E800DECFC3F0DECFC4F0DECFC5F0DECFC6F05C
:1026F80060D020EE06F09E51D9269F51DA22DECF17
:10270800C3F0DECFC4F0DECFC5F0DECFC6F0C351D4
:10271800C411C511C6113FE19EC081F09FC082F06F
:10272800836B846B856B866B30EC25F081C0C3F0BE
:1027380082C0C4F083C0C5F084C0C6F0C305C4110C
:10274800C511C61109E120EE0FF09E51D9269F51FF
:10275800DA22020EDF6E020CC3290FE1C4290DE153
:10276800C5290BE1C62909E120EE0FF09E51D926B3
:102778009F51DA22010EDF6E010C20EE06F09E5109
:10278800D9269F51DA22C3C0DEFFC4C0DEFFC5C010
:10279800DEFFC6C0DEFF20EE14F09E51D9269F5101
:1027A800DA22C3C0DEFFC4C0DEFFC5C0DEFFC6C07C
:1027B800DEFFC351C411C511C61101E085D0DDD0BB
:1027C800BF51A05FC051A15BC151A25BC251A35BC5
:1027D80020EE10F09E51D9269F51DA22BF51DE26F5
:1027E800C051DE22C151DE22C251DE2220EE0EF09F
:1027F8009E51D9269F51DA22DFA220D09EC081F0B7
:102808009FC082F0C3C083F0C4C084F0C5C085F007
:10281800C6C086F030EC25F081C0C3F082C0C4F099
:1028280083C0C5F084C0C6F0C351C411C511C61118
:102838001BE1A06BA16BA26BA36B50D09EC045F0AF
:102848009FC046F0C3C047F0C4C048F0C5C049F0B7
:10285800C6C04AF0DDEC2CF045C0C3F046C0C4F059
:1028680047C0C5F048C0C6F00001C32907E1C42924
:1028780005E1C52903E1C62901E176D7C651C5118D
:10288800C41104E1020EC35D01E25DD720EE13F02E
:10289800BC51D926BD51DA22DE50C35DDE50C45981
:1028A800DE50C559DE50C65901E34DD720EE14F06D
:1028B8009E51D9269F51DA22C3C0DEFFC4C0DEFF75
:1028C800C5C0DEFFC6C0DEFFA051BF5DA151C05923
:1028D800A251C159A351C25901E272D720EE10F09A
:1028E8009E51D9269F51DA22A051DE26A151DE221F
:1028F800A251DE22A351DE22A051A46F010EA11520
:10290800A56FA66BA76BA411A611A71136E0BCC0D2
:102918000EF0BDC00FF0C3C010F0C4C011F0C5C0A8
:1029280012F0C6C013F0A1EC4BF00EC0B8F00FC007
:10293800B9F010C0BAF011C0BBF00001B851B9111C
:10294800BA11BB1101E1FFD6A0C0A4F0A1C0A5F047
:10295800A2C0A6F0A3C0A7F00A0E05D0D890A7334E
:10296800A633A533A433E82EF9D7A451B827A55127
:10297800B923A651BA23A751BB2320EE10F09E51CC
:10298800D9269F51DA2210EE0AF09E51E1269F5176
:10299800E222DE50E65CDE50E658DE50E658DE50B5
:1029A800E6581CE220EE10F09E51D9269F51DA22FB
:1029B80010EE0AF09E51E1269F51E222DECFE6FF9B
:1029C800DECFE6FFDECFE6FFDECFE6FF20EE0EF03D
:1029D8009E51D9269F51DA22000EDB8C20EE10F092
:1029E8009E51D9269F51DA22FF0EDE14A46F010EE4
:1029F800DE14A56F000EDE14A66F000EDE14A76F9E
:102A0800A451A511A611A71101E16AD520EE18F06D
:102A18009E51D9269F51DA22B851DE180AE1B951E0
:102A2800DE1807E1BA51DE1804E1BB51DE1801E1F6
:102A380057D520EE18F09E51D9269F51DA22B8C0FA
:102A4800DEFFB9C0DEFFBAC0DEFFBBC0DEFF48D57F
:102A5800CE51CF1101E1090C3F0ED217D00E7C6F79
:102A6800AE0E7D6F010E7E6FD2C07FF0AFEC00F02E
:102A78000101B06FB05101E0A8D2AEC1B1F1AFC150
:102A8800B2F1B10E0001C06F010EC16FD0C0C2F02B
:102A9800D1C0C3F014EC42F00101B06FB05104E1B1
:102AA800D8AF02D0060EB06FD2C0D3F01C0E000112
:102AB800D31701E1D1D00101B0510FE0040EB019D4
:102AC80009E1B10E0001C46F010EC56F0FEC53F0A0
:102AD8000101B06F0001D2870DD0B5C1D3F0110E3E
:102AE8000001D31702E0070E03D0D2A503D0080EC9
:102AF8000101B06F0101B05101E0BDD00001D2A7C2
:102B0800BAD0AEC115F0AFC116F0CBC117F0CCC129
:102B180018F080EC59F015C09EF116C09FF117C04F
:102B2800A0F118C0A1F10E0E0101CB250E6E000E0A
:102B3800CC210F6E106A116A210E126E500E136EA0
:102B480006EC5BF0010120EE0BF0CB51D926CC51FD
:102B5800DA22200EDF6EAEC112F0AFC113F0CBC186
:102B680014F0CCC115F0166A176A186A196A8CEC49
:102B78005EF01C0E0101CB250E6E000ECC210F6EEF
:102B8800106A116A126A136A06EC5BF0010120EE02
:102B980003F0AE51D926AF51DA22010EDF6E9E51F5
:102BA8009F11A011A11167E020EE2BF0AE51D9269C
:102BB800AF51DA22DECFA2F1DECFA3F1DECFA4F14E
:102BC800DECFA5F1B10E0001816F010E826F9EC1AB
:102BD80083F09FC184F0A0C185F0A1C186F0876B06
:102BE800886B896B8A6BE1EC42F00101B06FB051E0
:102BF80042E1AEC13AF0AFC13BF0A2C13CF0A3C183
:102C08003DF0A4C13EF0A5C13FF071EC55F00101C3
:102C1800B06FFF0E9E250001D36FFF0E01019F21AB
:102C28000001D46FFF0E0101A0210001D56FFF0E36
:102C38000101A1210001D66F010120EE0BF0AE5178
:102C4800D926AF51DA22D3C0DEFFD4C0DEFFD5C00B
:102C5800DEFFD6C0DEFF0FD00101B0510CE1B5A9EF
:102C680002D0040E07D00001D2A305D00101B5A1FE
:102C780002D0070EB06F0101B05123E10001D2B7B5
:102C8800D28D010120EE2BF0AE51D926AF51DA22B8
:102C9800000110EE1CF0CE51E126CF51E222DECF2A
:102CA800E6FFDECFE6FFDECFE6FFDECFE6FF20EE73
:102CB80020F0CE51D926CF51DA22CBC1DEFFCCC1CC
:102CC800DDFF0101B05101E080D1AEC115F0AFC107
:102CD80016F0CBC117F0CCC118F080EC59F0000108
:102CE80020EE06F0CE51D926CF51DA2215C0DEFFEC
:102CF80016C0DEFF17C0DEFF18C0DEFF1C0E010184
:102D0800CB250E6E000ECC210F6E7CEC54F000012A
:102D180020EE0AF0CE51D926CF51DA220EC0DEFFBE
:102D28000FC0DEFF10C0DEFF11C0DEFFCEC0D9FF2E
:102D3800CFC0DAFFAEC1DEFFAFC1DDFF010120EE7B
:102D480005F0AE51D926AF51DA22000110EE02F09B
:102D5800CE51E126CF51E222DECFE6FFDDCFE5FFFF
:102D680020EE0EF0CE51D926CF51DA22D2C0DFFFA5
:102D780020EE0FF0CE51D926CF51DA22DF6A20EEAD
:102D880018F0CE51D926CF51DA22DE6ADE6ADE6A21
:102D9800DD6A20EE10F0CE51D926CF51DA22DE6A54
:102DA800DE6ADE6ADD6AD2AB10D120EE0AF0CE51BF
:102DB800D926CF51DA22DE50DE10DE10DE1001E116
:102DC80004D120EE0AF0CE51D926CF51DA2210EEE6
:102DD80010F0CE51E126CF51E222DECFE6FFDECF62
:102DE800E6FFDECFE6FFDECFE6FF010120EE09F0C9
:102DF800AE51D926AF51DA22DECFD3F0DDCFD4F0F1
:102E08000001D351D56FD451D66FD76BD86B090E4B
:102E1800D890D537D637D737D837E82EF9D7D5C091
:102E28009AF1D6C09BF1D7C09CF1D8C09DF120EE95
:102E380006F0CE51D926CF51DA22DECFAAF1DECF65
:102E4800ABF1DECFACF1DECFADF120EE0AF0CE5122
:102E5800D926CF51DA22DECFA6F1DECFA7F1DECF19
:102E6800A8F1DECFA9F132D0CEC045F0CFC046F0F0
:102E7800AAC147F0ABC148F0ACC149F0ADC14AF0B6
:102E8800DDEC2CF045C0AAF146C0ABF147C0ACF16F
:102E980048C0ADF10101AD51AC11AB1105E1020E15
:102EA800AA5D02E2020EB06FAA2908E1AB2906E189
:102EB800AC2904E1AD2902E1010EB06F9A51A65F79
:102EC8009B51A75B9C51A85B9D51A95B0101B05127
:102ED80009E1A6519A5DA7519B59A8519C59A9513E
:102EE8009D59C2E3000120EE14F0CE51D926CF51EE
:102EF800DA22AAC1DEFFABC1DEFFACC1DEFFADC185
:102F0800DEFF0101B05161E1A6510001D36F010E4E
:102F18000101A7150001D46FD56BD66BD311D5115C
:102F2800D61153E0AEC10EF0AFC10FF0AAC110F038
:102F3800ABC111F0ACC112F0ADC113F0A1EC4BF074
:102F48000EC0A2F10FC0A3F110C0A4F111C0A5F1E9
:102F58000101A251A311A411A51103E1020EB06F42
:102F680034D0A6C1D3F0A7C1D4F0A8C1D5F0A9C167
:102F7800D6F00A0E06D00001D890D633D533D43314
:102F8800D333E82EF8D70101A2510001D325D76F1A
:102F98000101A3510001D421D86F0101A4510001FE
:102FA800D521D96F0101A5510001D621DA6F20EE94
:102FB80018F0CE51D926CF51DA22D7C0DEFFD8C0BB
:102FC800DEFFD9C0DEFFDAC0DEFF0101B05106E046
:102FD800CEC0D9FFCFC0DAFFDE6ADD6AB051120079
:102FE80076C091F077C092F07AC0D9FF7BC0DAFF43
:102FF800DE6ADD6A74C00FF075C010F09D0E116EA8
:1030080026EC54F000018C6F8C510AE120EE0FF091
:103018007451D9267551DA22DF508C6F8C5102E039
:103028008C51120020EE0EF07451D9267551DA2217
:10303800DFA0070C20EE10F07451D9267551DA2262
:10304800DECF7CF0DECF7DF0DECF7EF0DECF7FF00E
:1030580020EE0AF07451D9267551DA22DECF80F0BD
:10306800DECF81F0DECF82F0DECF83F07C51805D51
:10307800886F7D518159896F7E5182598A6F7F513E
:1030880083598B6F78517C6F79517D6F7E6B7F6B25
:103098007C51885D7D5189597E518A597F518B5960
:1030A80001E321D288C078F089C079F01CD220EEE3
:1030B80010F07451D9267551DA22FF0EDE147C6F98
:1030C800010EDE147D6F000EDE147E6F000EDE141E
:1030D8007F6F7C517D117E117F1101E083D120EE3D
:1030E80010F07451D9267551DA22DECF7CF0DECF8C
:1030F8007DF0DECF7EF0DECF7FF00A0E05D0D890CF
:103108007F337E337D337C33E82EF9D7806981693C
:1031180020EE09F09D51D9269E51DA22DECF82F0A9
:10312800DDCF83F080518227815183237C51821522
:10313800936F7D518315946F931166E120EE10F023
:103148007451D9267551DA22DE50DE10DE10DE10F9
:103158000FE120EE06F07451D9267551DA22DECF40
:103168008DF0DECF8EF0DECF8FF0DECF90F01CD06A
:1031780074C045F075C046F020EE14F07451D9269D
:103188007551DA22DECF47F0DECF48F0DECF49F0C6
:10319800DECF4AF0DDEC2CF045C08DF046C08EF055
:1031A80047C08FF048C090F0000190518F118E11E8
:1031B8000CE1020E8D5D09E220EE0FF07451D92664
:1031C8007551DA22020EDF6E020C8D290FE18E296D
:1031D8000DE18F290BE1902909E120EE0FF07451E0
:1031E800D9267551DA22010EDF6E010C20EE14F09B
:1031F8007451D9267551DA228DC0DEFF8EC0DEFFEC
:103208008FC0DEFF90C0DEFF9DC00EF09EC00FF0A5
:1032180020EE14F07451D9267551DA22DECF10F061
:10322800DECF11F0DECF12F0DECF13F0A1EC4BF0C1
:103238000EC095F00FC096F010C097F011C098F02E
:103248000001955196119711981101E1B5D7935145
:10325800952794519623000E9723982378C07CF0E5
:1032680079C07DF0090E7E6FD8907D337C337E2F38
:10327800FBD77CC099F07DC09AF099519A1101E171
:10328800A3D0995193257C6F9A5194217D6F20EE9C
:1032980009F09D51D9269E51DA227C51DE5C7D5180
:1032A800DE5810E220EE09F09D51D9269E51DA220F
:1032B800DECF7CF0DDCF7DF093517C5D996F94512A
:1032C8007D599A6F91C01DF092C01EF095C01FF0F5
:1032D80096C020F097C021F098C022F099C023F042
:1032E8009AC024F020EE01F09D51D9269E51DA2291
:1032F800DF50D0EC54F0000901E0ACD0000120EE22
:1033080003F09D51D9269E51DA22DF504EE09951A3
:103318007C6F9A517D6F7E6B7F6B20EE2BF09D51F9
:10332800D9269E51DA22DECF80F0DECF81F0DECFC3
:1033380082F0DECF83F09551805D846F965181597C
:10334800856F97518259866F98518359876F7C5141
:10335800845D7D5185597E5186597F51875925E273
:1033680020EE2BF09D51D9269E51DA22DECF7CF03B
:10337800DDCF7DF095517C5F96517D5B090ED8902D
:103388007C377D37E82EFBD77C5191250E6E7D5119
:1033980092210F6E2F0E9D25106E000E9E21116E2C
:1033A800020E136E126A2BEC5EF099C07CF09AC084
:1033B8007DF0090ED8907C377D37E82EFBD77CC08E
:1033C8009BF07DC09CF072D020EE18F07451D92685
:1033D8007551DA2295C0DEFF96C0DEFF97C0DEFF8A
:1033E80098C0DEFF7C69010E7D6F20EE10F07451ED
:1033F800D9267551DA22DECF7EF0DDCF7FF07C5101
:103408007E177D517F177E5100089B6F7F51D8A092
:10341800E82A02089C6F9B51785D9C51795904E217
:1034280078C09BF079C09CF09DC03AF09EC03BF0FC
:1034380020EE18F07451D9267551DA22DECF3CF00F
:10344800DECF3DF0DECF3EF0DECF3FF071EC55F041
:10345800000902E00001C1D691C00EF092C00FF041
:1034680000017C69010E7D6F20EE10F07451D926A1
:103478007551DA22DECF7EF0DDCF7FF07C517E17EA
:103488007D517F179DC080F09EC081F07E518027BE
:103498007F5181232F0E8025106E000E8121116E21
:1034A8009BC012F09CC013F02BEC5EF09B51785F30
:1034B8009C51795B7AC0D9FF7BC0DAFF9B51DE262D
:1034C8009C51DD229B5191279C51922320EE10F0B4
:1034D8007451D9267551DA229B51DE269C51DE2281
:1034E800000EDE22DE227851791101E0E0D5000CD1
:1034F80052500C0D000EF324D96E020EF420DA6E31
:103508000001C969CA6952500C0D080EF324E16E16
:10351800020EF420E26EE6CFCBF0E5CFCCF0C95135
:10352800CB27CA51CC23DE50CB5DCC51800ACD6F5E
:10353800DE50800ACD594AE352500C0D020EF32496
:10354800D96E020EF420DA6EDF50C76FC86BC969F6
:10355800CA6952500C0D0A0EF324D96E020EF420DB
:10356800DA6EDF50CB6FCC6BC951CB27CA51CC2355
:10357800C751CB5DCC51800ACD6FC851800ACD5957
:1035880025E352500C0D030EF324D96E020EF420DD
:10359800DA6EDF50C76FC86BC969CA6952500C0D23
:1035A8000B0EF324D96E020EF420DA6EDF50CB6FC7
:1035B800CC6BC951CB27CA51CC23C751CB5DCC5159
:1035C800800ACD6FC851800ACD5961E21F0E0101F2
:1035D800896F010E8B6F8390E80E00019C6FF90EC6
:1035E8009D6F52500C0D000EF324D96E020EF4207C
:1035F800DA6EDECF9EF0DDCF9FF052500C0D080E34
:10360800F324D96E020EF420DA6EDECFC7F0DDCFD8
:10361800C8F0FF0EC725A06FFF0EC821A16F52503A
:103628000C0D020EF324D96E020EF420DA6EDF5070
:10363800A26FA36B52500C0D0A0EF324D96E020E22
:10364800F420DA6EDF50C96FFF0EC925A46FA56B91
:10365800FF0EA52352500C0D030EF324D96E020E53
:10366800F420DA6EDF50A66FA76B52500C0D0B0ECC
:10367800F324D96E020EF420DA6EDF50CA6FFF0E03
:10368800CA25A86FA96BFF0EA923B1EC61F05250AF
:103698000C0D030EF324D96E020EF420DA6EDF50FF
:1036A800C76FC7C0C8F0C96BCA6BCB6BCAC0CBF0B9
:1036B800C9C0CAF0C8C0C9F0C86B52500C0D0B0E77
:1036C800F324D96E020EF420DA6EDF50CC6FCCC032
:1036D800CDF0CE6BCF6BD06B52500C0D020EF32495
:1036E800D96E020EF420DA6EDF50D16FD1C0D2F05D
:1036F800D36BD46BD56BD4C0D5F0D3C0D4F0D2C0C3
:10370800D3F0D26BD251CD03F3CFD6F0F4CFD7F0AC
:10371800D86BD96BCE03F350D727F450D823000EBB
:10372800D923D351CD03F350D727F450D823000E13
:10373800D923D251CF03F350D827F450D923D351EA
:10374800CE03F350D827F450D923D451CD03F350E6
:10375800D827F450D923D051D203F350D927D351C5
:10376800CF03F350D927D451CE03F350D927D551DD
:10377800CD03F350D92752500C0D0A0EF324D96EFD
:10378800020EF420DA6EDF50DA6FDAC0DBF0DC6BA1
:10379800DD6BDE6B52500C0D0B0EF324D96E020E4E
:1037A800F420DA6EDF50DF6FDFC0E0F0E16BE26B30
:1037B800E36B52500C0D000EF324D96E020EF42068
:1037C800DA6EDECFE4F0DDCFE5F0E4C0E6F0E5C088
:1037D800E7F0000EE7BFFF0EE86FE96FE651E00380
:1037E800F3CFEAF0F4CFEBF0EC6BED6BE103F350C1
:1037F800EB27F450EC23000EED23E751E003F350E0
:10380800EB27F450EC23000EED23E651E203F350CE
:10381800EC27F450ED23E751E103F350EC27F45083
:10382800ED23E851E003F350EC27F450ED23E35186
:10383800E603F350ED27E751E203F350ED27E85193
:10384800E103F350ED27E951E003F350ED27ECC015
:10385800EDF0EBC0ECF0EAC0EBF0EA6BEA51DB0309
:10386800F3CFEEF0F4CFEFF0F06BF16BDC03F35035
:10387800EF27F450F023000EF123EB51DB03F35054
:10388800EF27F450F023000EF123EA51DD03F35043
:10389800F027F450F123EB51DC03F350F027F450F8
:1038A800F123EC51DB03F350F027F450F123DE5100
:1038B800EA03F350F127EB51DD03F350F127EC5104
:1038C800DC03F350F127ED51DB03F350F127D65118
:1038D800EE25F26FD751EF21F36FD851F021F46F35
:1038E800D951F121F56FC851F225F76FC951F3216C
:1038F800F86FCA51F421F96FCB51F521FA6F525084
:10390800220D380EF3249E6F020EF4209F6FF7C02D
:10391800A0F0F8C0A1F0F9C0A2F0FAC0A3F05EECE4
:1039280012F0F66FF65111E0520E9C6FFB0E9D6F70
:10393800F7C09EF0F8C09FF0F9C0A0F0FAC0A1F05F
:10394800F6C0A2F0A36BB1EC61F052500C0D040E5E
:10395800F324D96E020EF420DA6EF7C0DEFFF8C049
:10396800DEFFF9C0DEFFFAC0DEFF01018B6B83903A
:103978001200266E225002E049EC52F0256A2150CE
:1039880001E1C9D1269E040E261802E14E5003E13A
:10399800140E261807E101017C6B7D6B226A070E65
:1039A800216E070C3F0E261807E14E6A01017C6B59
:1039B8007D6B216A226A12005F0E261807E1010159
:1039C8008C6B7C6B7D6B216A226A12003F0E266429
:1039D8000BD05F0E266008D0400E261805E00101C6
:1039E8008C6B216A226A1200400E26180AE1010E29
:1039F80001018C6F4E6A01017C6B7D6B216A226A22
:103A08001200200E261801E086D1010E4E6EF3D763
:103A1800600E261809E101018C5106E08A51080E52
:103A2800D8B4030E256E7CD0600E261809E14E50DE
:103A380007E001018A5102E0090E15D0050E13D0E6
:103A4800680E261809E14E5007E01A0E01017D6F35
:103A5800900E54D18380BCD1680E261806E101016E
:103A68008C5103E0020E256E5BD06A0E261807E122
:103A78004E5005E01A0E01017D6FF40E3FD16C0E19
:103A8800261807E14E5005E01A0E01017D6F2C0E35
:103A980035D1700E261810E101018C510DE0830E0E
:103AA80000019C6FFF0E9D6FB1EC61F0040E256E56
:103AB80001017C6B7D6BCED7700E261801E088D192
:103AC8004E5001E185D11B0E01017D6F620E16D1AA
:103AD8008380020E261805E11A0E01017D6F920EF1
:103AE8007C6F050E261805E11A0E01017D6FAE0EDA
:103AF8007C6F070E261805E11A0E01017D6FB80EBE
:103B08007C6F080E261805E11A0E01017D6FCC0E98
:103B18007C6F030E261802E0262806E1256A8390AA
:103B280001017C6B7D6B54D1140E261805E11A0E29
:103B380001017D6F9E0E7C6F160E261801E048D19C
:103B48001A0E01017D6FA40ECAD0050E261805E1D4
:103B58001A0E01017D6FF50E7C6F080E261801E024
:103B680037D11A0E01017D6FCC0E7C6F010E8A6F62
:103B78002FD126C052F01A0E01017D6F950EAFD0DD
:103B88002650246E236A52500C0D000EF324D96E71
:103B9800020EF420DA6E23C0DEFF24C0DDFF1A0E09
:103BA80001017D6F960E9BD02650236E246A5250D9
:103BB8000C0D000EF324D96E020EF420DA6E23C029
:103BC800DEFF24C0DDFF1A0E01017D6F970E87D03E
:103BD80052500C0D020EF324D96E020EF420DA6E48
:103BE80026C0DFFF1A0E01017D6F980E78D0525063
:103BF8000C0D030EF324D96E020EF420DA6E26C0E3
:103C0800DFFF01017C6B7D6B010E37D01A0E0101BD
:103C18007D6FB90E73D01A0E01017D6FBA0E5FD099
:103C28001A0E01017D6FBB0E7C6F3A0E00019C6F6E
:103C3800FE0E9D6FB1EC61F001018B6B7C6B7D6BAF
:103C480055D001017C6B7D6B3A0E00019C6FFE0E16
:103C58009D6FB1EC61F04AD0E80E00019C6FFE0E3A
:103C68009D6FB1EC61F001017C6B7D6B010E886F7B
:103C78003DD001017C6B7D6B060E256EA9D026C058
:103C880052F001017C6B7D6B256A30D001018A6B93
:103C98001A0E7D6FF70E7C6F29D01A0E01017D6F09
:103CA800F70E1DD08390270E01017D6F0F0E17D0E0
:103CB800180E261801E08CD01A0E01017D6F2D0E0A
:103CC8000ED01A0E01017D6F2E0E09D01A0E0101B9
:103CD8007D6F2F0E04D01A0E01017D6F300E7C6FA0
:103CE80077D001017C6B7D6B0A0E256E839070D0B6
:103CF800040E256E270E01017D6F0F0E7C6FAAD66C
:103D08008380010104D08390010E01018A6F7C6BCE
:103D18007D6B256A5DD07CC123F07DC124F02450E1
:103D280007E01A0A09E0010A4BE03C0A4FE050D0CC
:103D3800235001E16DD64CD023502C0AB9E0010A7A
:103D4800C0E0030AC3E0010AC6E01F0ACAE0A00AED
:103D580001E1BED6020A01E10CD7070A01E110D73A
:103D6800030A01E121D7010A01E132D70F0A01E173
:103D78003ED7060A01E170D73A0A01E17AD70A0A62
:103D8800C2E0160A01E142D7010A01E144D7030A59
:103D980001E146D7010A01E154D7790A01E162D667
:103DA8000E0A01E16CD7380A01E1CFD6010A01E118
:103DB8006DD7030A01E171D7010A01E173D708D071
:103DC8002350580A95E03A0A9BE002D023500F0A84
:103DD80025C021F0226A1200020E806F655164111D
:103DE800631104E1020E625D01E211D220EE13F0CC
:103DF8006051D9266151DA22DE50625DDE50635986
:103E0800DE506459DE50655901E2EED100D262C03D
:103E18007EF063C07FF0D8907F316B6F7E316A6F20
:103E28006A517E276B517F2360C03AF061C03BF036
:103E380020EE1FF06051D9266151DA22DECF6AF0F8
:103E4800DECF6BF0DECF6CF0DECF6DF07EC06EF0B3
:103E58007FC06FF0090E706FD8906F336E33702F7C
:103E6800FBD76E516A253C6E6F516B213D6E000E7B
:103E78006C213E6E000E6D213F6E71EC55F0000115
:103E8800806F805101E0C3D16A69010E6B6F7EC0FB
:103E98006CF07FC06DF06A516C176B516D1760C084
:103EA8006EF061C06FF06C516E276D516F232F0E4D
:103EB8006E257C6F000E6F217D6F7E4B7F2B62B16C
:103EC80004D066C078F0796B1AD066516A6F6B6B54
:103ED8006A3B6B3BF00E6B176A510F0B6B13F00EBE
:103EE8006A177CC0D9FF7DC0DAFFDF500F0B6C6FFB
:103EF8006D6B6A516C11786F6B516D11796F7CC065
:103F0800D9FF7DC0DAFF78C0DFFF20EE03F06051F3
:103F1800D9266151DA22010EDF6E60C03AF061C025
:103F28003BF020EE1FF06051D9266151DA22DECF36
:103F38006AF0DECF6BF0DECF6CF0DECF6DF07EC0C6
:103F48006EF07FC06FF0090E706FD8906F336E33CC
:103F5800702FFBD76E516A253C6E6F516B213D6EF9
:103F6800000E6C213E6E000E6D213F6E71EC55F017
:103F78000001806F805101E04AD16A69010E6B6FC0
:103F88007EC06CF07FC06DF06A516C176B516D1775
:103F980060C06EF061C06FF06C516E276D516F2379
:103FA8002F0E6E257C6F000E6F217D6F62B10CD0D5
:103FB80067C06AF00F0E6A177CC0D9FF7DC0DAFFB0
:103FC800DF50F00B6A1112D066C06AF067C06BF060
:103FD80068C06CF069C06DF0050E05D0D8906D33DF
:103FE8006C336B336A33E82EF9D76A517A6F7B6B7F
:103FF8007CC0D9FF7DC0DAFF7AC0DFFF4FD060C038
:104008003AF061C03BF020EE1FF06051D9266151B3
:10401800DA22DECF6AF0DECF6BF0DECF6CF0DECFD7
:104028006DF063516E6F64516F6F6551706F716B96
:104038006A516E253C6E6B516F213D6E6C5170213B
:104048003E6E6D5171213F6E71EC55F00001806F2D
:10405800805101E0DCD06A69010E6B6F62C06CF0C0
:1040680063C06DF0D8906C376D376A516C176B511F
:104078006D1760C06EF061C06FF06C516E276D51A6
:104088006F232F0E6E250E6E000E6F210F6E66C009
:1040980010F067C011F0EEEC60F0A4D020EE03F051
:1040A8006051D9266151DA22010EDF6EB0D060C0AE
:1040B8003AF061C03BF020EE1FF06051D926615103
:1040C800DA22DECF6AF0DECF6BF0DECF6CF0DECF27
:1040D8006DF062C06EF063C06FF064C070F065C0D0
:1040E80071F0080E05D0D890713370336F336E338A
:1040F800E82EF9D76A516E253C6E6B516F213D6EE3
:104108006C5170213E6E6D5171213F6E71EC55F00E
:104118000001806F80517BE16A69010E6B6F62C09C
:104128006CF063C06DF0D8906C376D37D8906C37F1
:104138006D376A516C176B516D1760C06EF061C0B6
:104148006FF06C516E276D516F232F0E6E250E6E1A
:10415800000E6F210F6E7CEC54F00001706B716BD8
:10416800726BF00E1114736F6651746F6751756F2F
:104178006851766F0F0E6915776F70517411666FFD
:1041880071517511676F72517611686F735177119C
:10419800696F6A69010E6B6F62C06CF063C06DF085
:1041A800D8906C376D37D8906C376D376A516C176B
:1041B8006B516D1760C06EF061C06FF06C516E2767
:1041C8006D516F232F0E6E250E6E000E6F210F6E30
:1041D80066C010F067C011F068C012F069C013F033
:1041E80006EC5BF000015AD760C0D9FF61C0DAFF66
:1041F800DF506A6F6B6B6B510AE16A51010A01E18A
:1042080006D6030A01E1FBD6010A01E150D7805125
:1042180012002D6E1EC044F01FC045F02D5001E065
:10422800040C010E426E55B0030CE9D178EC61F034
:10423800000901E1FDD1426AFBD1176A186A196ABF
:104248001A6A090E5CEC5FF0000901E0F1D12E0E4C
:104258000E6E0F6A116A100E106E05EC5CF0000904
:1042680001E1E6D12E44E846030BE8064DE135C0EE
:1042780020F03F0E201620C021F0226A236A246A0B
:1042880022C024F021C023F0226A216A3650266E0B
:10429800256A3750276E286A255027262650282257
:1042A80027502124296E285022202A6E000E232010
:1042B8002B6E000E24202C6E29283E6E000E2A201C
:1042C8003F6E000E2B20406E000E2C20416E3EC02B
:1042D80020F03FC021F040C022F041C023F00A0E78
:1042E800D8902036213622362336E82EF9D71EC03C
:1042F800D9FF1FC0DAFF20C0DEFF21C0DEFF22C0C9
:10430800DEFF23C0DEFF97D7206A38AE01D0202A0F
:10431800010E201633C021F00F0E21163750030B63
:10432800020DF35021242024020F436E3450030B56
:10433800206E216A0A0ED89020362136E82EFBD747
:104348003550226E236AD89022362336D8902236EA
:1043580023363644E846030B246E256A2250242669
:10436800235025222050242621502522242A000EBD
:10437800252224C03EF025C03FF0406A416A43C070
:1043880020F0F70E20263EC021F03FC022F040C0AA
:1043980023F041C024F0202A05D0D89021362236B7
:1043A80023362436202EF9D734D053A43FD0176AA9
:1043B800186A196A1A6A8D0E5CEC5FF0000901E050
:1043C80037D1CDEC61F02E0E0E6E0F6A116A100E09
:1043D800106E05EC5CF0000901E12AD1300E436E45
:1043E80003D0CDEC61F043064350FBE138C020F028
:1043F800203A0F0E2016100E216E226A236A246AB4
:10440800202A05D0D8902136223623362436202E6D
:10441800F9D71EC0D9FF1FC0DAFF21C0DEFF22C0B6
:10442800DEFF23C0DEFF24C0DEFF05D7176A186A47
:10443800196A1A6A090E5CEC5FF0000901E0F8D00D
:104448002E0E0E6E0F6A116A100E106E05EC5CF0DF
:10445800000901E1EDD053A232D03BC020F0060E96
:10446800216ED8902032212EFCD7FF0E20263850FE
:104478003F0B226E236AD890223623363944010B2B
:104488002226000E2322222A2322202A03D0D89073
:1044980022362336202EFBD72250246E2350256E39
:1044A800266A276A1EC0D9FF1FC0DAFF24C0DEFFB4
:1044B80025C0DEFF26C0DEFF27C0DEFFBCD6395090
:1044C800030B206E216AD89020362136D8902036EA
:1044D8002136D890203621363938E842070B202675
:1044E800000E2122202A21223840E8423F0B1F0BD0
:1044F800226E236A222A000E232220502202F3CFA2
:1045080024F0F4CF25F02302F3502526215022026F
:10451800F35025262450266E2550276E286A296ACE
:104528001EC0D9FF1FC0DAFF26C0DEFF27C0DEFF8E
:1045380028C0DEFF29C0DEFF7ED644C0D9FF45C0B3
:10454800DAFF53C0DFFF77D6176A186A196A1A6A42
:10455800090E5CEC5FF000096BE144C00EF045C049
:104568000FF0116A100E106E05EC5CF0000901E006
:1045780062D65ED0176A186A196A1A6A0A0E5CEC63
:104588005FF0000955E144C00EF045C00FF0116A14
:10459800100E106E05EC5CF0E9D7176A186A196AF4
:1045A8001A6A3A0E5CEC5FF0000942E1040E436EB1
:1045B8000AD0CDEC61F044C0D9FF45C0DAFFDF6E08
:1045C800444A452A4306435001E135D6F2D7176AD3
:1045D800186A196A1A6A8D0E5CEC5FF0000928E106
:1045E800CDEC61F044C00EF045C00FF0116A400EEA
:1045F800106E05EC5CF0BAD7040E426E19D01D504F
:10460800206E216A2150F8E1205001E10FD6010AFD
:1046180001E113D6020A01E1C8D6090A8EE0010AAF
:1046280093E0070AA7E0010AB8E0030AD0E0E4D75C
:10463800DEEC61F0425012001BC0F6FF1CC0F7FF11
:104648000800F5CF9BF01B4A1C2A00019B5101E191
:104658001200250E9B1904E09B519BEC61F0ECD7EE
:10466800946B956B966B976B1BC0F6FF1CC0F7FF9E
:104678000800F5CF9BF01B4A1C2A300E9B190DE150
:10468800976B010E966F1BC0F6FF1CC0F7FF080062
:10469800F5CF9BF01B4A1C2A06D02D0E9B1903E16F
:1046A800976B020EEFD72A0E9B1943E11D50D96E66
:1046B800DA6A020EDF26DF5CD96EDA6ADECF8CF0AA
:1046C800DECF8DF08DAF0BD08C5100088C6F8D51E3
:1046D800D8A0E82A00088D6F976B020E966F8CC0E1
:1046E80094F08DC095F01BC0F6FF1CC0F7FF0800C2
:1046F800F5CF9BF01B4A1C2A22D00A0E9403F3CF55
:104708001EF0F4CF1FF09503F3501F269B511E2671
:10471800000E1F22D00E1E24946FFF0E1F20956FCF
:104728001BC0F6FF1CC0F7FF0800F5CF9BF01B4A23
:104738001C2A2F0E9B6503D0390E9B65DED76C0EA5
:104748009B1903E04C0E9B190AE196851BC0F6FFE6
:104758001CC0F7FF0800F5CF9BF01B4A1C2A9B5191
:1047680001E112009BC09AF0600E9A6575D0200E88
:104778009A5F72D01D50D96EDA6A020EDF26DF5CAE
:10478800D96EDA6ADECF84F0DECF85F0926B936B58
:1047980003D00001924B932B925184251E6E9351A6
:1047A80085211F6E1EC0F6FF1FC0F7FF000EF86EB2
:1047B8000E0EF76403D00800F55005D0F6CFE9FFD8
:1047C800F7CFEAFFEF50000904E0E3D7200E9BEC97
:1047D80061F0000196B30BD092511E6E93511F6E7B
:1047E800924B932B94511E5C95511F58EFE384C054
:1047F8000FF085C010F089EC5CF003D0200E9BEC24
:1048080061F0000192511E6E93511F6E924B932BD3
:1048180094511E5C95511F5801E30ED7EFD71D50D8
:10482800D96EDA6ADF50DF2ADF2AD96EDA6ADF50FA
:104838009BEC61F001D7876B020E08D0876B080EDE
:1048480005D0876B0A0E02D0876B100E866F1AD0C0
:104858009B519BEC61F0F0D69A511E6E1F6A1F5057
:10486800F7E11E50420AE7E0010AD9E0070AE9E049
:104878000B0AE4E01C0A01E17DD7060AE2E00D0A12
:10488800E3E0E6D796A511D01D50D96EDA6A040E7A
:10489800DF26DF5CD96EDA6ADECF8EF0DECF8FF0EE
:1048A800DECF90F0DECF91F027D0440E9A1913E0B6
:1048B8001D50D96EDA6ADF50DF2ADF2AD96EDA6A2C
:1048C800DECF1EF0DDCF1FF01EC08EF01FC08FF0B0
:1048D800906B916B11D01D50D96EDA6ADF50DF2AC8
:1048E800DF2AD96EDA6ADECF8EF0DDCF8FF0000EC8
:1048F8008FBFFF0E906F916F440E9A190CE191AF24
:104908000AD08E6D8F1FD8B08F2B901FD8B0902BE8
:10491800000E91579689986B996B8EC088F08FC05E
:1049280089F090C08AF091C08BF088C00EF089C0E1
:104938000FF08AC010F08BC011F086C012F087C04B
:1049480013F0146A156AA4EC5BF00E5000019A6F1C
:1049580088C00EF089C00FF08AC010F08BC011F02B
:1049680086C012F087C013F0146A156A45EC59F036
:104978000EC088F00FC089F010C08AF011C08BF00B
:10498800090E00019A650BD0780E9B1903E0816B24
:10499800070E02D0816B270E806F80519A2798519D
:1049A800600FD96EDA6A9A51300FDF6E984B992BE7
:1049B800885189118A118B1105E0995103E1200E64
:1049C800985DB3E396A908D09851600FD96EDA6A5A
:1049D8002D0EDF6E984B992B98C092F099C093F0EA
:1049E80096B103D0836B200E02D0836B300E826F9A
:1049F80082C09AF003D09A519BEC61F0000196B303
:104A08000BD092511E6E93511F6E924B932B945163
:104A18001E5C95511F58EFE39807D8A09907985145
:104A2800600FD96EDA6ADF509BEC61F00001985193
:104A3800991104E0F1D7200E9BEC61F0000192512E
:104A48001E6E93511F6E924B932B94511E5C955181
:104A58001F5801E3F1D5EFD781C0D9FF82C0DAFF33
:104A6800DECF98F0DDCF99F083518411851186113E
:104A780028E120EE0BF09851D9269951DA22DECFA1
:104A880090F0DECF91F0DECF92F0DECF93F0905130
:104A98009111921193110FE020EE13F09851D9263D
:104AA8009951DA22DE50905DDE509159DE509259CC
:104AB800DE50935952E3010E906F916B926B936B9A
:104AC8004CD081C045F082C046F083C047F084C016
:104AD80048F085C049F086C04AF0DDEC2CF045C0AE
:104AE8009AF046C09BF047C09CF048C09DF000017A
:104AF8009D519C119B1109E1020E9A5D06E2010E7F
:104B0800816F826B836B846B000C9A290FE19B2960
:104B18000DE19C290BE19D2909E19AC081F09BC018
:104B280082F09CC083F09DC084F0120020EE13F048
:104B38009851D9269951DA22DE509A5DDE509B5958
:104B4800DE509C59DE509D59E8E383C090F084C044
:104B580091F085C092F086C093F020EE0FF0985146
:104B6800D9269951DA22DE50DE10DE10DE1005E17A
:104B7800816B826B836B846B1200946B956B966B65
:104B8800976B8351901909E18451911906E1855178
:104B980092197DE186519319D8A479D09029946F00
:104BA800000E9121956F000E9221966F000E9321B1
:104BB800976F20EE13F09851D9269951DA22DE50DA
:104BC800945DDE509559DE509659DE50975905E3AD
:104BD800020E946F956B966B976B81C045F082C0FF
:104BE80046F094C047F095C048F096C049F097C089
:104BF8004AF0DDEC2CF045C09AF046C09BF047C067
:104C08009CF048C09DF000019A059B119C119D11D4
:104C180084E09A2907E19B2905E19C2903E19D2964
:104C280001E17BD79A519B119C119D1130E020EE38
:104C38000BF09851D9269951DA22DECF9AF0DECFBF
:104C48009BF0DECF9CF0DECF9DF09D519C119B1117
:104C580003E1020E9A5D17E320EE13F09851D9266E
:104C68009951DA22DE509A5DDE509B59DE509C59EC
:104C7800DE509D5908E29AC090F09BC091F09CC00C
:104C880092F09DC093F0946B956B966B976B9451D3
:104C980095119611971162E190C094F091C095F02A
:104CA80092C096F093C097F0942B000E952396230C
:104CB800972320EE13F09851D9269951DA22DE5025
:104CC800945DDE509559DE509659DE5097590DE3A4
:104CD800020E946F956B966B976B9351921191118D
:104CE80004E1020E905D01E243D781C045F082C025
:104CF80046F094C047F095C048F096C049F097C078
:104D08004AF0DDEC2CF045C09AF046C09BF047C055
:104D18009CF048C09DF000019A519B119C119D1177
:104D28001DE09A059B119C119D1101E1F6D69A2967
:104D380007E19B2905E19C2903E19D2901E1EDD6C5
:104D480090519419B1E191519519AEE1925196198A
:104D5800ABE19351971901E10BD7A6D798C060F042
:104D680099C061F094C062F095C063F096C064F099
:104D780097C065F06669676968696969F0EC1EF053
:104D88008F6F8F511CE1835184118511861117E0B3
:104D980098C060F099C061F083C062F084C063F08D
:104DA80085C064F086C065F094C066F095C067F071
:104DB80096C068F097C069F0F0EC1EF08F6F8F51C5
:104DC80043E120EE0BF09851D9269951DA2294C08C
:104DD800DEFF95C0DEFF96C0DEFF97C0DEFF20EE47
:104DE8000FF09851D9269951DA2210EE13F0985104
:104DF800E1269951E222FE0EE6248B6FFF0EE62093
:104E08008C6FFF0EE6208D6FFF0EE6208E6FDE5052
:104E18008B5DDE508C59DE508D59DE508E590BE378
:104E280020EE0FF09851D9269951DA22DE06000EAD
:104E3800DE5ADE5ADE5A20EE04F09851D9269951EE
:104E4800DA22000EDB800DD08F0507E0010E946F8B
:104E5800000E956B966B976B04D09469956996696B
:104E6800976994C081F095C082F096C083F097C08E
:104E780084F0120052500C0D030EF324D96E020E6A
:104E8800F420DA6EDF2A52500C0D030EF324D96E8B
:104E9800020EF420DA6EDF500001C76FC86BC969D3
:104EA800CA6952500C0D0B0EF324D96E020EF42071
:104EB800DA6EDF50CB6FCC6BC951CB27CA51CC23EC
:104EC800C751CB5DCC51800ACD6FC851800ACD59EE
:104ED8004BE252500C0D030EF324D96E020EF4204F
:104EE800DA6EDF6A52500C0D020EF324D96E020EF0
:104EF800F420DA6EDF2A52500C0D020EF324D96E1C
:104F0800020EF420DA6EDF50C76FC86BC969CA6930
:104F180052500C0D0A0EF324D96E020EF420DA6EEC
:104F2800DF50CB6FCC6BC951CB27CA51CC23C751AB
:104F3800CB5DCC51800ACD6FC851800ACD5914E29F
:104F480052500C0D020EF324D96E020EF420DA6EC4
:104F5800DF6A52500C0D000EF324D96E020EF420B5
:104F6800DA6EDE2A000EDD2252500C0D030EF324F9
:104F7800D96E020EF420DA6EDF50C76FC7C0C8F0D2
:104F8800C96BCA6BCB6BCAC0CBF0C9C0CAF0C8C06A
:104F9800C9F0C86B52500C0D0B0EF324D96E020EDB
:104FA800F420DA6EDF50CC6FCCC0CDF0CE6BCF6B77
:104FB800D06B52500C0D020EF324D96E020EF42061
:104FC800DA6EDF50D16FD1C0D2F0D36BD46BD56B12
:104FD800D4C0D5F0D3C0D4F0D2C0D3F0D26BD25164
:104FE800CD03F3CFD6F0F4CFD7F0D86BD96BCE037F
:104FF800F350D727F450D823000ED923D351CD032B
:10500800F350D727F450D823000ED923D251CF0319
:10501800F350D827F450D923D351CE03F350D827CF
:10502800F450D923D451CD03F350D827F450D923C1
:10503800D051D203F350D927D351CF03F350D927F6
:10504800D451CE03F350D927D551CD03F350D927E6
:1050580052500C0D0A0EF324D96E020EF420DA6EAB
:10506800DF50DA6FDAC0DBF0DC6BDD6BDE6B5250E1
:105078000C0D0B0EF324D96E020EF420DA6EDF50FD
:10508800DF6FDFC0E0F0E16BE26BE36B52500C0DB9
:10509800000EF324D96E020EF420DA6EDECFE4F0AF
:1050A800DDCFE5F0E4C0E6F0E5C0E7F0000EE7BFCD
:1050B800FF0EE86FE96FE651E003F3CFEAF0F4CFB3
:1050C800EBF0EC6BED6BE103F350EB27F450EC23C2
:1050D800000EED23E751E003F350EB27F450EC23E7
:1050E800000EED23E651E203F350EC27F450ED23D4
:1050F800E751E103F350EC27F450ED23E851E003C6
:10510800F350EC27F450ED23E351E603F350ED2779
:10511800E751E203F350ED27E851E103F350ED279F
:10512800E951E003F350ED27ECC0EDF0EBC0ECF0F3
:10513800EAC0EBF0EA6BEA51DB03F3CFEEF0F4CF11
:10514800EFF0F06BF16BDC03F350EF27F450F02332
:10515800000EF123EB51DB03F350EF27F450F0235B
:10516800000EF123EA51DD03F350F027F450F12348
:10517800EB51DC03F350F027F450F123EC51DB033F
:10518800F350F027F450F123DE51EA03F350F127EE
:10519800EB51DD03F350F127EC51DC03F350F12719
:1051A800ED51DB03F350F127D651EE25F26FD751BD
:1051B800EF21F36FD851F021F46FD951F121F56F38
:1051C800C851F225F66FC951F321F76FCA51F4217E
:1051D800F86FCB51F521F96F52500C0D040EF324E2
:1051E800D96E020EF420DA6EF6C0DEFFF7C0DEFFDD
:1051F800F8C0DEFFF9C0DEFF5250220D380EF3244E
:105208009E6F020EF4209F6F52500C0D040EF32473
:10521800D96E020EF420DA6EDECFA0F0DECFA1F058
:10522800DECFA2F0DECFA3F05EEC12F04B6E4B5057
:1052380019E0520E9C6FFB0E9D6F52500C0D040E20
:10524800F324D96E020EF420DA6EDECF9EF0DECFA4
:105258009FF0DECFA0F0DECFA1F04BC0A2F0A36B91
:10526800B1EC61F001018B6B1200380E0001746F14
:10527800020E756F350E766F0B0E776F020E796F13
:10528800786BF30E7A6F7B6BF4EC17F00101966F75
:10529800790E00019C6FFD0E9D6FF3C09EF0F4C067
:1052A8009FF0B1EC61F0F56BF66BF16BF26BF76B9D
:1052B800F86BF751D30FD96EDA6ADF6AF751E20F4C
:1052C800D96EDA6A000EDF6EF74BF82BF8BFF1D70C
:1052D800F85103E10F0EF75DECE3F96BFA6B30D18F
:1052E800350EF925D96E0B0EFA21DA6E0D0EDE1881
:1052F80001E0EBD0950E0E6EFF0E0F6ED30E106E02
:10530800BFEC55F00E500F1007E1E20E156EB5EC2C
:105318004DF015500101FB6F8F0E0E6EFF0E0F6ED4
:10532800D30E106EBFEC55F00E500F1007E1E20ED1
:10533800156EB5EC4DF015500101976F6E0E0E6E9F
:10534800FF0E0F6ED30E106EBFEC55F00E500F10FF
:1053580007E1E20E156EB5EC4DF015500101926FA4
:10536800D30E0E6EFF0E0F6ED30E106EBFEC55F0FF
:105378000E500F1007E1E20E156EB5EC4DF015500A
:105388000101906FD70E0E6EFF0E0F6ED30E106ECA
:10539800BFEC55F00E500F1007E1E20E156EB5EC9C
:1053A8004DF015500101F96F0001FB6BFC6BC40E49
:1053B8007C6F7D6B750E7E6FFF0E7F6FFBC080F07C
:1053C800FCC081F006EC5FF0C40E0E6E0F6AD30EBF
:1053D800106EBFEC55F00E500F1018E10F0E0001C3
:1053E800FB03F3CFC2F0F4CFC3F0FC03F350C327A1
:1053F800350EC2250E6E0D0EC3210F6EE20E106E15
:10540800116A136A0F0E126E34EC5CF00001FB4B4C
:10541800FC2BFCBFCCD7FC5103E1100EFB5DC7E3AE
:10542800FC6B010EFB6FC40E7C6F7D6B7C0E7E6F78
:10543800FF0E7F6FFBC080F0FCC081F006EC5FF0D0
:10544800C40E0E6E0F6AD30E106EBFEC55F00E50E0
:105458000F1018E10F0E0001FB03F3CFC2F0F4CFD9
:10546800C3F0FC03F350C327250EC2250E6E0E0EA3
:10547800C3210F6EE20E106E116A136A0F0E126EC0
:1054880034EC5CF00001FB4BFC2BFCBFCCD7FC518F
:1054980003E1040EFB5DC7E3F76BF86BF751D30F1D
:1054A800D96EDA6ADF6AF751E20FD96EDA6A000E4E
:1054B800DF6EF74BF82BF8BFF1D7F85103E10F0E69
:1054C800F75DECE3F16BF26B15D0350EF925D96E6B
:1054D8000B0EFA21DA6E0A0EDE1830E0350EF925C9
:1054E800D96E0B0EFA21DA6E200EDE1806E1F26B89
:1054F800010EF16FF56BF66B21D0F151F21109E055
:10550800350EF925D96E0B0EFA21DA6EF551E20F38
:1055180008D0350EF925D96E0B0EFA21DA6EF55141
:10552800D30FE16EE26ADFCFE7FFF6BF05D0F65191
:1055380005E10F0EF55D02E2F54BF62BF94BFA2B60
:10554800F351F95DF451FA5901E2CAD6690E9C6F1C
:10555800FD0E9D6F92C19EF09F6BB1EC61F0E30E62
:105568009C6FFD0E9D6FFBC19EF09F6BB1EC61F0CF
:10557800C50E9C6FFD0E9D6F97C19EF09F6BB1ECA1
:1055880061F0D40E9C6FFD0E9D6FF9C19EF09F6B6C
:10559800B1EC61F0FB6BFC6BF70E9C6FFC0E9D6F22
:1055A800FBC09EF0FCC09FF00F0EFB03F3CFC2F0D0
:1055B800F4CFC3F0FC03F350C327350EC225A06F08
:1055C8000D0EC321A16FB1EC61F0FB4BFC2BFCBFAE
:1055D800E3D7FC5103E1100EFB5DDEE3FA6B010E2D
:1055E800F96F080E9C6FFD0E9D6FF9C09EF0FAC012
:1055F8009FF00F0EF903F3CFC2F0F4CFC3F0FA0314
:10560800F350C327250EC225A06F0E0EC321A16F2C
:10561800B1EC61F0F94BFA2BFABFE3D7FA5103E189
:10562800040EF95DDEE3980E9C6FF90E9D6FB1EFE5
:1056380061F0838E8380B0EC3CF0FC6FFC5118E085
:1056480052501C0D1B0EF324D96E010EF420DA6E95
:1056580052501C0D1B0EF324E16E010EF420E26E75
:10566800E7500409DF6E43EC60F00001FC511200C2
:10567800010190514EE0705171117211731149E09E
:10568800525047E152501C0D070EF324D96E010EFB
:10569800F420DA6E70C1A3F171C1A4F172C1A5F151
:1056A800A26B000EA225A66F010EA321A76F000E04
:1056B800A421A86F000EA521A96FAA6BAB6BAC6BD8
:1056C800AD6BDE50A61925E1DE50A71922E1DE50A8
:1056D800A8191FE1DE50A9191CE1DE50AA1919E129
:1056E800DE50AB1916E1DE50AC1913E1DE50AD19EE
:1056F80010E1350E2B6E0B0E2C6E905133EC4FF0E3
:105708000292000E9AEC5AF00292506A839050501E
:10571800120052501C0D170EF324D96E010EF420FE
:10572800DA6EDECF9AF1DECF9BF1DECF9CF1DECFD1
:105738009DF19BC19AF19CC19BF19DC19CF19D6B10
:105748009AC1F0F09BC1F1F09CC1F2F09DC1F3F059
:1057580052501C0D170EF324D96E010EF420DA6E88
:10576800DECF9AF1DDCF9BF19A510001F66FF76B0E
:105778000292F86BF96BFA6BFB6BF46BF56B94D0D8
:10578800F4C09AF1F5C09BF1000E9BBFFF0E9C6F11
:105798009D6FFF0E0001F02501019E6FFF0E0001B5
:1057A800F12101019F6FFF0E0001F2210101A06F9D
:1057B800FF0E0001F3210101A16F9A519E1910E11A
:1057C8009B519F190DE19C51A0190AE19D51A11906
:1057D80007E10001F651F71103E102500209026ED8
:1057E8005250220D380EF3240001746F020EF4207B
:1057F800756F350E766F0B0E776F010E796F786BBC
:10580800FD0E7A6F7B6BF4EC17F0FF6FFF5101E030
:1058180017D7FD51FE1101E113D7FD519AEC5AF04B
:105828000001FD51F827FE51F923000EFA23FB234E
:1058380052501C0D070EF324D96E010EF420DA6EB7
:10584800000EDE2401019A6F010EDE209B6F000E10
:10585800DE209C6F000EDE209D6F000EDE209E6F06
:10586800000EDE209F6F000EDE20A06F000EDE20EF
:10587800A16F52501C0D070EF324D96E010EF420AF
:10588800DA6E9AC1DEFF9BC1DEFF9CC1DEFF9DC1BF
:10589800DEFF9EC1DEFF9FC1DEFFA0C1DEFFA1C10A
:1058A800DEFF0001F44BF52BF4C09AF1F5C09BF133
:1058B800000E01019BBFFF0E9C6F9D6F0001F05110
:1058C80001019A5D0001F15101019B590001F2515A
:1058D80001019C590001F35101019D5901E250D782
:1058E8000001F651F71160E05250220D380EF324F2
:1058F800746F020EF420756F350E766F0B0E776F8E
:10590800F6C078F0F7C079F0FD0E7A6F7B6BF4EC97
:1059180017F0FF6FFF5101E093D602500209026EA3
:10592800F6519AEC5AF00001FD51F827FE51F9237F
:10593800000EFA23FB2352501C0D070EF324D96ED8
:10594800010EF420DA6E000EDE2401019A6F010EBA
:10595800DE209B6F000EDE209C6F000EDE209D6F08
:10596800000EDE209E6F000EDE209F6F000EDE20F0
:10597800A06F000EDE20A16F52501C0D070EF324FD
:10598800D96E010EF420DA6E9AC1DEFF9BC1DEFFEC
:105998009CC1DEFF9DC1DEFF9EC1DEFF9FC1DEFF11
:1059A800A0C1DEFFA1C1DEFF0292506A8390839EF0
:1059B800AED645C0D9FF46C0DAFFDECF72F0DDCFE4
:1059C80073F04A504910481003E1020E475C10E397
:1059D800000120EE13F07251D9267351DA22DE50FD
:1059E800475CDE504858DE504958DE504A5808E3B4
:1059F800010E00016C6F000E6D6B6E6B6F6B8FD1BB
:105A08006C696D696E696F6976D147C070F048C07E
:105A180071F0D8907131616F7031606F605170278B
:105A28006151712372C03AF073C03BF020EE1FF051
:105A38007251D9267351DA22DECF60F0DECF61F0E1
:105A4800DECF62F0DECF63F070C064F071C065F045
:105A5800090E666FD89065336433662FFBD764519F
:105A680060253C6E655161213D6E000E62213E6EDF
:105A7800000E63213F6E71EC55F0000901E04FD133
:105A880000016069010E616F70C062F071C063F05F
:105A9800605162176151631772C064F073C065F09A
:105AA80062516427635165232F0E6425D96E000E59
:105AB8006521DA6EDF506A6F6B6B704B712B72C0A9
:105AC8003AF073C03BF020EE1FF07251D9267351A3
:105AD800DA22DECF60F0DECF61F0DECF62F0DECF1B
:105AE80063F070C064F071C065F0090E666FD890FD
:105AF80065336433662FFBD7645160253C6E65516E
:105B080061213D6E000E62213E6E000E63213F6EE4
:105B180071EC55F0000901E002D100016069010E45
:105B2800616F70C062F071C063F0605162176151BB
:105B3800631772C064F073C065F0625164276351E3
:105B480065232F0E6425D96E000E6521DA6EDF50AD
:105B5800676F666B66516A1367516B1347B006D05F
:105B68006A51686F0F0E6B15696F0FD06AC060F0CD
:105B78006BC061F0040E626FD89061336033622F9E
:105B8800FBD760C068F061C069F068C06CF069C09C
:105B98006DF04ED072C03AF073C03BF020EE1FF0AB
:105BA8007251D9267351DA22DECF60F0DECF61F070
:105BB800DECF62F0DECF63F04850646F4950656F06
:105BC8004A50666F676B605164253C6E6151652170
:105BD8003D6E625166213E6E635167213F6E71ECE6
:105BE80055F0000901E09BD000016069010E616F6A
:105BF80047C062F048C063F0D8906237633760519D
:105C080062176151631772C064F073C065F0625126
:105C18006427635165232F0E64250E6E000E6521DF
:105C28000F6EC9EC5FF00EC06CF00FC06DF0000194
:105C38006E6B6F6B74D072C03AF073C03BF020EE9D
:105C48001FF07251D9267351DA22DECF60F0DECF11
:105C580061F0DECF62F0DECF63F047C064F048C089
:105C680065F049C066F04AC067F0080E05D0D890C4
:105C78006733663365336433E82EF9D7605164259A
:105C88003C6E615165213D6E625166213E6E6351E5
:105C980067213F6E71EC55F0000941E10001606930
:105CA800010E616F47C062F048C063F0D890623758
:105CB8006337D89062376337605162176151631751
:105CC80072C064F073C065F0625164276351652344
:105CD8002F0E64250E6E000E65210F6E7CEC54F0BD
:105CE8000E5000016C6F0F506D6F10506E6F0F0EDD
:105CF80011146F6F14D072C0D9FF73C0DAFFDF5070
:105D0800606F616B615101E073D66051010A01E176
:105D18007CD6030A01E13ED7010A8DE069D66CC042
:105D280045F06DC046F06EC047F06FC048F01200F5
:105D3800D70EF66EF80EF76E0900F5CFC5F00A001B
:105D4800F5CFC6F00001C76BCD6B0201ED6B030EFA
:105D58000101F96105D09650F919F00BF91905D030
:105D6800F9C193FF9650F00B0A09966ECD6ACE6A78
:105D78002ED1CC6B350E176E0B0E186EC50E196E24
:105D880054EC56F017C0CAF018C0CBF0CAC0D9FFFF
:105D9800CBC0DAFF3B0EDE1801E014D118D1CC518C
:105DA80022E1CAC012F0CBC013F0F3EC59F00001A5
:105DB800CD6F800ECD6503D0CD51800FC76F030E18
:105DC800C76501D0C76B9B0E9C6FF90E9D6FFCC118
:105DD8009EF09F6BCDC0A0F0A16BC7C0A2F0A36BD3
:105DE800B1EC61F0E4D0CC051BE10101FC510001EC
:105DF800CD1903E07F0ECD1913E1CAC012F0CBC054
:105E080013F0F3EC59F00101956F170E00019C6F28
:105E1800FF0E9D6F95C19EF09F6BB1EC61F0C7D0EE
:105E2800020ECC191BE10101FC510001CD1903E060
:105E38007F0ECD1913E1CAC012F0CBC013F0F3ECFA
:105E480059F00101946F200E00019C6FFF0E9D6FA9
:105E580094C19EF09F6BB1EC61F0A9D0020ECC65A5
:105E68002CD0080ECC6129D00101FC510001CD19BC
:105E78000CE07F0ECD1909E0810ECD1906E0820EE7
:105E8800CD1903E0830ECD1918E1C751050D800E19
:105E9800F324C86F030EF420C96FCAC012F0CBC038
:105EA80013F0F3EC59F00001C26FCC51C825C36F51
:105EB800000EC921C46FFD0E5AD0070ECC652CD038
:105EC8001B0ECC6129D00101FC510001CD190CE059
:105ED8007F0ECD1909E0810ECD1906E0820ECD198D
:105EE80003E0830ECD1918E1C751130D000EF324FA
:105EF800C86F030EF420C96FCAC012F0CBC013F0EC
:105F0800F3EC59F00001C26FCC51C825C36F000EE5
:105F1800C921C46FF80E2BD0280ECC6130D00101F6
:105F2800FC510001CD190CE07F0ECD1909E0810E5E
:105F3800CD1906E0820ECD1903E0830ECD191FE1BD
:105F4800C7510D0D4C0EF324C86F030EF420C96F12
:105F5800CAC012F0CBC013F0F3EC59F00001C26FC5
:105F6800CC51C825C36F000EC921C46FE50EC325E7
:105F7800D96EFF0EC421DA6EC2C0DFFF18D0280E1A
:105F8800CC1915E10101FC510001CD1903E07F0E88
:105F9800CD190DE1ED0E0E6E020E0F6ECAC010F097
:105FA800CBC011F0136A080E126E34EC5CF0CC2BE7
:105FB800176A186AC50E196E54EC56F017C0CAF065
:105FC80018C0CBF00001CA51CB1101E0E8D6350E5C
:105FD80000019F6F0B0EA06FA26B910EA16F380E80
:105FE800A36F020EA46F9EEC56F09F51A01101E022
:105FF800C0D6060E9C6FFB0E9D6FED0E9E6F020EB7
:106008009F6FB1EC61F0000EC86F030EC96FC8C076
:1060180021F0C9C022F0000E246E130E236E520E1A
:10602800256EFF0E266ECAEC3AF0130EC86F030EEB
:10603800C96FC8C021F0C9C022F0000E246E130E2B
:10604800236E590E256EFF0E266ECAEC3AF0260E08
:10605800C86F030EC96FC8C021F0C9C022F0000E76
:10606800246E130E236E600E256EFF0E266ECAEC8C
:106078003AF0390EC86F030EC96FC8C021F0C9C005
:1060880022F0000E246E130E236E670E256EFF0E8F
:10609800266ECAEF3AF0526A4F6A526A030E526489
:1060A80001D090D1525003E1216A226A03D0226ABA
:1060B800010E216E52501C0D1B0EF324D96E010ED9
:1060C800F420DA6EDF6A52501C0D000EF324D96EEC
:1060D800010EF420DA6EDF6A52501C0D070EF3240D
:1060E800D96E010EF420DA6E070EDE6AE806FDE2CC
:1060F8000D0E2102F3CF9AF1F4CF9BF12202F35057
:1061080001019B27570E9A25D96E030E9B21DA6E43
:10611800DF509C6F9CC19DF19E6B9F6BA06B9FC1D4
:10612800A0F19EC19FF19DC19EF19D6B9DC1A1F102
:106138009EC1A2F19FC1A3F1A0C1A4F1A56BA4BF08
:10614800A569A5C1A6F1A5C1A7F1A5C1A8F10D0E24
:106158002102F3CFA9F1F4CFAAF12202F350AA2722
:10616800560EA925D96E030EAA21DA6EDF50AB6F41
:10617800ABC1ACF1AD6BAE6BAF6BADC1AFF1ACC148
:10618800AEF1AD6BAC6BACC1B0F1ADC1B1F1AEC1AC
:10619800B2F1AFC1B3F1B46BB3BFB469B4C1B5F177
:1061A800B4C1B6F1B4C1B7F10D0E2102F3CFB8F105
:1061B800F4CFB9F12202F350B927550EB825D96E9C
:1061C800030EB921DA6EDF50BA6FBAC1BBF1BC6BEE
:1061D800BD6BBE6BBBC1BEF1BD6BBC6BBB6BBBC14A
:1061E800BFF1BCC1C0F1BDC1C1F1BEC1C2F1C36B39
:1061F800C2BFC369C3C1C4F1C3C1C5F1C3C1C6F13C
:106208000D0E2102F3CFC7F1F4CFC8F12202F350EB
:10621800C827540EC725D96E030EC821DA6EDF5081
:10622800C96FC9C1CAF1CB6BCC6BCD6BCE6BCF6BD1
:10623800D06BD16B200ED890CA37CB37CC37CD373F
:10624800CE37CF37D037D137E82EF5D7BF51CA254B
:10625800D26FC051CB21D36FC151CC21D46FC25161
:10626800CD21D56FC351CE21D66FC451CF21D76F61
:10627800C551D021D86FC651D121D96FB051D2257F
:10628800DA6FB151D321DB6FB251D421DC6FB35136
:10629800D521DD6FB451D621DE6FB551D721DF6F1F
:1062A800B651D821E06FB751D921E16FA151DA2554
:1062B800E26FA251DB21E36FA351DC21E46FA4510B
:1062C800DD21E56FA551DE21E66FA651DF21E76FDD
:1062D800A751E021E86FA851E121E96F52501C0D48
:1062E8000F0EF324D96E010EF420DA6EE2C1DEFF40
:1062F800E3C1DEFFE4C1DEFFE5C1DEFFE6C1DEFF8C
:10630800E7C1DEFFE8C1DEFFE9C1DEFF770E00016D
:106318009C6FFA0E9D6F52C09EF09F6B52501C0DE1
:106328000F0EF324D96E010EF420DA6EDECF9AF147
:10633800DECF9BF1DECF9CF1DECF9DF1DECF9EF16B
:10634800DECF9FF1DECFA0F1DECFA1F19AC1A0F0A0
:106358009BC1A1F09CC1A2F09DC1A3F09EC1A4F075
:106368009FC1A5F0A0C1A6F0A1C1A7F052501C0D75
:106378000F0EF324D96E010EF420DA6EDECFA2F1EF
:10638800DECFA3F1DECFA4F1DECFA5F1DECFA6F1FB
:10639800DECFA7F1DECFA8F1DECFA9F1A2C1A8F028
:1063A800A3C1A9F0A4C1AAF0A5C1ABF0A6C1ACF0E5
:1063B800A7C1ADF0A8C1AEF0A9C1AFF0B1EC61F0D2
:1063C800522A6CD601018F6B516A8E6B7E6B7F6B84
:1063D800020E506E8D6F8390020C9EC0D9FF9FC035
:1063E800DAFFDECFB2F0DDCFB3F020EE0EF09E5133
:1063F800D9269F51DA22DECFA2F0DECFA3F0DECF7E
:10640800A4F0DECFA5F0200EA225AE6F000EA321CA
:10641800AF6F000EA421B06F000EA521B16FB1516E
:1064280003E1200EB05D0AE320EE16F09E51D92656
:106438009F51DA22DE6ADE6ADE6ADD6A20EE16F035
:106448009E51D9269F51DA22DE50DE10DE10DE1072
:1064580001E1040CAE51A26F010EAF15A36FA46B3E
:10646800A56BA211A411A51101E029D120EE16F007
:106478009E51D9269F51DA22DE2A000EDE22DE2224
:10648800DE2220EE12F09E51D9269F51DA22DE50EC
:10649800DE10DE10DE102CE120EE07F0B251D92616
:1064A800B351DA22DECFA2F0DDCFA3F0A251A46F60
:1064B800A351A56FA66BA76BAEC0A8F0AFC0A9F09B
:1064C800B0C0AAF0B1C0ABF0060E05D0D890AB337F
:1064D800AA33A933A833E82EF9D7A451A85DA5514A
:1064E800A959A651AA59A751AB5901E2E8D06ED0D3
:1064F800A269A36920EE09F0B251D926B351DA2274
:10650800DECFA4F0DDCFA5F0A251A427A351A52387
:10651800AEC0A6F0AFC0A7F0B0C0A8F0B1C0A9F057
:106528000A0E05D0D890A933A833A733A633E82E8E
:10653800F9D7A451A615AA6FA551A715AB6FAC6BD7
:10654800AD6BAA11AC11AD1101E0B9D09EC045F0F8
:106558009FC046F020EE12F09E51D9269F51DA22B4
:10656800DECF47F0DECF48F0DECF49F0DECF4AF08D
:10657800DDEC2CF045C0B4F046C0B5F047C0B6F02D
:1065880048C0B7F00001B751B611B51104E1020EC9
:10659800B45D01E2020CB42907E1B52905E1B62989
:1065A80003E1B72901E1010C20EE13F0B251D9261D
:1065B800B351DA22DE50B45DDE50B559DE50B6591B
:1065C800DE50B75950E3A051A1110BE120EE16F0AF
:1065D8009E51D9269F51DA22DE6ADE6ADE6ADD6ABA
:1065E800040C9EC081F09FC082F020EE12F09E51F4
:1065F800D9269F51DA22DECF83F0DECF84F0DECFBA
:1066080085F0DECF86F030EC25F081C0B4F082C092
:10661800B5F083C0B6F084C0B7F0B451B511B61167
:10662800B71101E1070CB405B511B611B71101E1B5
:10663800020CB42907E1B52905E1B62903E1B72918
:1066480001E1010CB2C03AF0B3C03BF0B4C03CF079
:10665800B5C03DF0B6C03EF0B7C03FF033EC4DF0EA
:10666800000901E0010C000120EE12F09E51D9262C
:106678009F51DA22B4C0DEFFB5C0DEFFB6C0DEFF30
:10668800B7C0DEFFB2C00EF0B3C00FF0B4C010F058
:10669800B5C011F0B6C012F0B7C013F0A1EC4BF0C2
:1066A800000120EE16F09E51D9269F51DA220EC025
:1066B800DEFF0FC0DEFF10C0DEFF11C0DEFF20EEE0
:1066C8000EF09E51D9269F51DA22AEC0DEFFAFC030
:1066D800DEFFB0C0DEFFB1C0DEFFA269010EA36F0E
:1066E800AEC0A4F0AFC0A5F0A251A417A351A5173E
:1066F800B2C0A6F0B3C0A7F0A451A627A551A723FE
:106708002F0EA627000EA72320EE1AF09E51D92699
:106718009F51DA22A6C0DEFFA7C0DDFF000C000EE5
:106728000001E06F250EDF6F000EDE6F050EDD6FD6
:106738000101FB5105E1000E0001E06F280EDF6F3B
:10674800010192510DE1FC6B350E00017C6F0D0EBD
:106758007D6F880E7E6FFE0E7F6F06EC5FF00DD0AA
:10676800970E00019C6FFA0E9D6F92C19EF09F6B71
:10677800FCC1A0F0A16BB1EC61F0010E9C6FFE0EA4
:106788009D6F0101FC510F0D350EF32400019E6F22
:106798000D0EF4209F6FB1EC61F0050E0001DC6F67
:1067A8000F0EDB6FF10EE82EFED7DB2FFCD7DC2FA8
:1067B800FAD7E3D0E60E0F6EFC0E106E89EC5CF093
:1067C800030E0101F96105D09650F919F00BF9197A
:1067D80005D0F9C193FF9650F00B0A09966E380E52
:1067E8000001CE6F020ECF6F7B0ED06FFE0ED16F01
:1067F800010ED26F2CEC15F00101966F965105EC45
:106808005DF0010196510AE19CEC2EF0380E6D6F97
:10681800020E6E6FE9EC5EF00101966F965105EC81
:106828005DF0E06B280EDF6FA4D00101FC510F0D65
:10683800350EF324D96E0D0EF420DA6E200EDE1814
:1068480006E1FC2B0F0EFC6594D0FC6B92D0F70E82
:1068580000019C6FFB0E9D6F0101FC510F0D350E61
:10686800F32400019E6F0D0EF4209F6FB1EC61F0D0
:10687800380ECE6F020ECF6F0101FC510F0D350E91
:10688800F3240001D06F0D0EF420D16F030ED26FE8
:106898002CEC15F00101966F965105EC5DF00101A5
:1068A800965104E10001E06B3C0EDF6F040E01011C
:1068B800961904E10001E06B320EDF6F050E00014E
:1068C800DC6F0F0EDB6FF10EE82EFED7DB2FFCD747
:1068D800DC2FFAD74ED0B20E9C6FFC0E9D6F0101D3
:1068E800FC510F0D350EF32400019E6F0D0EF420A0
:1068F8009F6FB1EC61F0380ECE6F020ECF6F0101C1
:10690800FC510F0D350EF3240001D06F0D0EF4204D
:10691800D16F070ED26F2CEC15F00101966F9651CE
:10692800CDE10001E06B3C0EC8D78D0E9C6FFC0ECC
:106938009D6F0101FC510F0D350EF32400019E6F70
:106948000D0EF4209F6FB1EC61F013D0DFC0DBF0C7
:10695800E0C0DCF0DC510DE1DB51250A01E12AD76A
:106968000D0A01E162D7050A04E01F0AB4E00E0A25
:10697800DCE00001DD07D8A0DE070001DEBF08D09B
:10698800DE5102E1DD0504E33C0EDF19E011DEE132
:10699800030E010192193BE1839E000E0E6EC00E9C
:1069A80056EC5DF0C5EC60F0000E0E6EC00E56ECB5
:1069B8005DF03C0E0001DF19E01116E10201ED5116
:1069C8000CE0ED0E126E020E136ECCEC58F0AC0E0D
:1069D800126EFE0E136ECCEC58F09B0E126EFF0E6C
:1069E800136ECCEC58F0000C350E7C6F0D0E7D6FDD
:1069F800320E7E6FFF0E7F6F96C180F0816B06ECC2
:106A08005FF0350E126E0D0E136ECCEC58F0000CC4
:106A180074C0D9FF75C0DAFFDECF8CF0DDCF8DF002
:106A2800795109E1200E785DD8B0020C76C07AF071
:106A38001F0E7A1701E0020C20EE0EF07451D926D1
:106A48007551DA2276C0DEFF77C0DEFF78C0DEFF40
:106A580079C0DEFF20EE06F07451D9267551DA228E
:106A6800DECF88F0DECF89F0DECF8AF0DECF8BF084
:106A7800885189118A118B1115E18CC0D9FF8DC0FD
:106A8800DAFF020EDF640ED020EE23F08C51D926F7
:106A98008D51DA22DECF88F0DECF89F0DECF8AF0A2
:106AA800DECF8BF0885189118A118B1140E120EEDD
:106AB80007F08C51D9268D51DA22DECF7AF0DDCF5E
:106AC8007BF07A517C6F7B517D6F7E6B7F6B76C0DC
:106AD80080F077C081F078C082F079C083F0060E2C
:106AE80005D0D8908333823381338033E82EF9D7A9
:106AF8007C51805D7D5181597E5182597F518359E6
:106B080001E3020C20EE23F08C51D9268D51DA22B4
:106B180010EE16F07451E1267551E222DECFE6FF41
:106B2800DECFE6FFDECFE6FFDECFE6FF87D020EE42
:106B380009F08C51D9268D51DA22DECF7AF0DDCFDB
:106B48007BF07A517C6F7B517D6F7E6B7F6B090E7A
:106B5800D8907C377D377E377F37E82EF9D77CC0D1
:106B680084F07DC085F07EC086F07FC087F040D07D
:106B780074C045F075C046F088C047F089C048F039
:106B88008AC049F08BC04AF0DDEC2CF045C088F093
:106B980046C089F047C08AF048C08BF000018829B8
:106BA80007E1892905E18A2903E18B2901E1010C23
:106BB8008B518A11891104E1020E885DD8A0020C5C
:106BC80020EE13F08C51D9268D51DA22DE50885DE3
:106BD800DE508959DE508A59DE508B5901E3020C88
:106BE8008451765F8551775B8651785B8751795BF5
:106BF8008451765D855177598651785987517959ED
:106C0800B7E28CC00EF08DC00FF088C010F089C0BC
:106C180011F08AC012F08BC013F0A1EC4BF0000108
:106C280020EE16F07451D9267551DA220EC0DEFF17
:106C38000FC0DEFF10C0DEFF11C0DEFF20EE12F035
:106C48007451D9267551DA2288C0DEFF89C0DEFF6B
:106C58008AC0DEFF8BC0DEFF20EE16F07451D92605
:106C68007551DA22DE50DE10DE10DE1001E1020C72
:106C780076C07AF077C07BF078C07CF079C07DF080
:106C88000A0E05D0D8907D337C337B337A33E82ED7
:106C9800F9D720EE16F07451D9267551DA227A51B7
:106CA800DE267B51DE227C51DE227D51DE227A698E
:106CB800010E7B6F76C07CF077C07DF07A517C172F
:106CC8007B517D178CC07EF08DC07FF07C517E2774
:106CD8007D517F232F0E7E27000E7F2320EE1AF092
:106CE8007451D9267551DA227EC0DEFF7FC0DDFFE0
:106CF800000C350E0101A66F0B0EA76FE9C00EF050
:106D0800EAC00FF00AEC5EF00E5001019A6FC70E50
:106D180000019E6F9F6BA06BA16BA26BA36B5EECD7
:106D280012F00101A36FA3510DE0200E00019C6F2A
:106D3800FB0E9D6FB1EC61F00001C76BC86BC96BAE
:106D4800CA6B1200C70E0001746F756BA6C176F08E
:106D5800A7C177F0010E796F786BA10E7A6F010EDB
:106D68007B6FF4EC17F00101A36FA35108E0C90E83
:106D780000019C6FFB0E9D6FB1EC61F0DDD7A6C1E1
:106D8800D9FFA7C1DAFF800EDE1808E0D50E000192
:106D98009C6FFC0E9D6FB1EC61F0CED720EE0AF02F
:106DA800A651D926A751DA22DF500001EC6FEB6B10
:106DB800010120EE0BF0A651D926A751DA22DF50A7
:106DC8000001EB2501019F6F000E0001EC2101017C
:106DD800A06FB20E00019C6FFB0E9D6F9FC19EF0CD
:106DE800A0C19FF0B1EC61F0C70E9E6F9F6B0101CF
:106DF8009F510001EC6FEB6BEBC0A0F0ECC0A1F071
:106E0800A26BA36B5EEC12F00101A36FA35194E196
:106E1800C70E0001746F756BA6C176F0A7C177F035
:106E2800010E796F786BA10E7A6F010E7B6FF4EC0F
:106E380017F00101A36FA35101E07ED7A46BA56BE6
:106E4800E9C00EF0EAC00FF0A4C1EBF0A5C1ECF068
:106E5800050ED8900001EB37EC37E82EFAD7EB5146
:106E68000101A625106E0001EC510101A721116E48
:106E78009AC112F0136A30EC57F00E500F105DE112
:106E8800A4C1EBF0A5C1ECF0050ED8900001EB37DA
:106E9800EC37E82EFAD7A6C1EDF0A7C1EEF0EB511A
:106EA800ED27EC51EE230E0EED25D96E000EEE21E6
:106EB800DA6EDF50F06FEF6BA4C1F1F0A5C1F2F00C
:106EC800050ED890F137F237E82EFBD7A6C1F3F0BC
:106ED800A7C1F4F0F151F327F251F4230F0EF32573
:106EE800D96E000EF421DA6EDF50F56FF66BEF51B4
:106EF800F527F051F623F5C09BF1F6C09CF101018E
:106F0800000E9CBFFF0E9D6F9E6F890E00019C6F47
:106F1800FD0E9D6F9BC19EF09CC19FF09DC1A0F08E
:106F28009EC1A1F0B1EC61F09BC1C7F09CC1C8F053
:106F38009DC1C9F09EC1CAF01200A44BA52BA5BFE4
:106F48007FD7A55105E10F0EA45D01E3F5D678D7EB
:106F5800F3D61850D96EDA6ADECF22F0DDCF23F0EF
:106F68001C0E1624266E000E1720276E26C00EF063
:106F780027C00FF0116A200E106E136A0B0E126EE6
:106F880028EC61F0286A296A246A256A216A080EB1
:106F9800206E24502224196E255023201A6E19C001
:106FA800F6FF1AC0F7FF000EF86E0E0EF76403D056
:106FB8000800F55005D0F6CFE9FFF7CFEAFFEF500C
:106FC8002A6E244A252A210E2A6001D0BED02F0E0F
:106FD8002A1806E05C0E2A1803E036D0244A252A2F
:106FE80024502224196E255023201A6E19C0F6FF4A
:106FF8001AC0F7FF000EF86E0E0EF76403D00800F3
:10700800F55005D0F6CFE9FFF7CFEAFFEF502F0A8A
:10701800E5E024502224196E255023201A6E19C049
:10702800F6FF1AC0F7FF000EF86E0E0EF76403D0D5
:107038000800F55005D0F6CFE9FFF7CFEAFFEF508B
:107048005C0A01E082D0CAD72E0E2A1805E020502B
:10705800285C215029580FE30B0E20182110D8B4B2
:10706800060C2E0E2A1801E0060C296A080E286E56
:10707800216A0B0E8DD72A502EEC5DF00E500F10A2
:1070880044E024502224196E255023201A6E19C07A
:10709800F6FF1AC0F7FF000EF86E0E0EF76403D065
:1070A8000800F55005D0F6CFE9FFF7CFEAFFEF501B
:1070B8001F6E244A252A1F502BEC5AF00E500F1031
:1070C800D8B4060C19681A6820C01BF021C01CF03F
:1070D80019501B261A501C221B50285C1C5029587A
:1070E80001E3060C28502624D96E29502720DA6E91
:1070F8002AC0DFFF284A292A28502624D96E295079
:107108002720DA6E1FC0DFFF1DD0A70E0E6EFD0E02
:107118000F6E2AC010F0116A40EC5FF00E500F108D
:1071280001E0060C600E2A6405D07B0E2A6002D0AE
:10713800200E2A5E28502624D96E29502720DA6E80
:107148002AC0DFFF284A292A24D724502224196E6E
:10715800255023201A6E1850D96EDA6A19C0DEFF3E
:107168001AC0DDFF2850291001E1060C26C0D9FFFE
:1071780027C0DAFFE50EDE1806E126C0D9FF27C0D2
:10718800DAFF050EDF6E200E2A6403D01D6A1E6A20
:1071980003D01E6A040E1D6E20EE0BF02650D92671
:1071A8002750DA221DC0DFFF000C02500209026ED0
:1071B800350E0E6E0B0E0F6E116A106A010E136EED
:1071C800126AD2EC48F0000EE8CF35FBFF0EE8CF8C
:1071D80036FB52501C0D1B0EF324D96E010EF42001
:1071E800DA6E0101DFA403D0010EE8CF37FB52505D
:1071F8001C0D1B0EF324D96E010EF420DA6EDFA8E5
:1072080003D0020EE8CF37FB52501C0D1B0EF3249F
:10721800D96E010EF420DA6EDFA003D0020EE8CF9B
:1072280039FB52501C0D1B0EF324D96E010EF420AD
:10723800DA6EDFA203D0020EE8CF39FB52501C0DE4
:107248001B0EF324D96E010EF420DA6EDFA603D0EC
:10725800800EE8CF38FB8FA403D0080EE8CF3BFBA5
:10726800236A246A300E2324D96E020E2420DA6E93
:10727800DF1C226E370E2324D96E0B0E2420DA6E03
:10728800370E2324E16E0B0E2420E26EE750221401
:10729800DF6E234A242A24BEE5D7245003E1070ED3
:1072A800235CE0E3506A020E4F6448D052501C0D34
:1072B800010EF324D96E010EF420DA6EDF50216E30
:1072C80021C040FB52501C0D020EF324D96E010E52
:1072D800F420DA6EDF50216E21C041FB52501C0DA4
:1072E800030EF324D96E010EF420DA6EDF50216EFE
:1072F80021C042FB52501C0D040EF324D96E010E1E
:10730800F420DA6EDF50216E21C043FB52501C0D71
:10731800050EF324D96E010EF420DA6EDF50216ECB
:1073280021C044FB52501C0D060EF324D96E010EE9
:10733800F420DA6EDF50216E21C045FB140E9AEC62
:107348005AF0050E00019C6FFF0E9D6FB1EC61F0C5
:10735800236A246A1C0E9C6FFF0E9D6F350E232432
:10736800D96E0B0E2420DA6EDF509E6F9F6BB1EC46
:1073780061F0234A242A24BEEDD7245003E1130EDA
:10738800235CE8E352501C0D1B0EF324D96E010E4A
:10739800F420DA6EDF6A02928390000C276E0001F7
:1073A800C35102E04FEC30F0266A0001C25101E1FE
:1073B800D6D0040E271802E1515003E1140E271805
:1073C80009E101018E6B7E6B7F6B0001C36B070EB9
:1073D800C26F070C3F0E271807E1516A01018E6B37
:1073E8000001C26BC36B12005F0E271807E1010191
:1073F8008F6B8E6B0001C26BC36B12003F0E27644C
:1074080006D05F0E276003D0400E2718F0E1400E2B
:10741800271809E1010E01018F6F01018E6B000130
:10742800C26BC36B1200200E271803E1010E516EC8
:10743800F4D7650E271809E1515007E001017E6B6A
:107448007F6B010E8E6F8380EAD76E0E271803E1DB
:10745800020E01018E6F700E271807E101018F518E
:1074680004E07E6B7F6B030E8E6F700E271808E1A9
:10747800515006E0838001017E6B7F6B040E0DD0B6
:10748800720E27186CE151506AE083804F6A1C0E17
:1074980001017F6F2A0E7E6F050E8E6FC0D72750B1
:1074A8000DEC0CF0266E6DD08380275046EC58F01A
:1074B800266E01018E6B65D08380350E0E6E0B0E25
:1074C8000F6E116A106A010E136E126AD2EC48F040
:1074D80002500209026E2BEE35F050C0DFFF010E9C
:1074E8009AEC5AF00292080E266E01018E6B506AD1
:1074F80048D08390266A45D0080E271813E1839058
:10750800526A266A506A030E4F6412D00F0E4F1843
:107518000FE0010E506E1B5110091B6F09D07E6BD6
:107528007F6B2FD0090E271805E18390266A506AD1
:107538008E6BF5D71F0E276424D0300E276021D01C
:10754800E00E00019C6FFB0E9D6F27C09EF09F6BA5
:10755800B1EC61F027500F0B4F6E266AC8D70101B6
:107568008E51246E256A25500CE124500AE0010A48
:1075780096E0030A99E0010A9FE0070ABAE0010AC7
:10758800BBE026C0C2F00001C36B1200950E0001DB
:107598009C6FFE0E9D6F25C09EF026C09FF021C0F7
:1075A800A0F022C0A1F023C0A2F024C0A3F0B1EC47
:1075B80061F02D6A2E6AC1D0980E9C6FF90E9D6FEE
:1075C800B1EC61F02F6A306A28D02DC027F02EC0A8
:1075D80028F0273A283AF00E281627500F0B2812C1
:1075E800F00E271621C029F022C02AF0275029269C
:1075F80028502A222F502924D96E30502A20DA6E9A
:10760800DF502C6EA10E9C6FFF0E9D6F2CC09EF05C
:107618009F6BB1EC61F02F4A302A30BE05D0305054
:1076280019E1100E2F5C16E22DC027F02EC028F0AD
:10763800273A283AF00E281627500F0B2812F00E7A
:1076480027162F502726305028222750235C2850F1
:107658002458BBE2DF0E9C6FFF0E9D6FB1EC61F00A
:107668002F6A306A4BD02DC027F02EC028F0273A59
:10767800283AF00E281627500F0B2812F00E27165E
:1076880021C029F022C02AF02750292628502A2272
:107698002F502924D96E30502A20DA6E200EDF644C
:1076A80025D0FB0E9C6FFF0E9D6F2DC027F02EC0BE
:1076B80028F0273A283AF00E281627500F0B2812E0
:1076C800F00E271621C029F022C02AF027502926BB
:1076D80028502A222F502924D96E30502A20DA6EB9
:1076E800DF509E6F9F6BB1EC61F006D0E60E9C6F89
:1076F800FE0E9D6FB1EC61F02F4A302A30BE05D0E6
:10770800305019E1100E2F5C16E22DC027F02EC064
:1077180028F0273A283AF00E281627500F0B28127F
:10772800F00E27162F502726305028222750235C8A
:107738002850245898E22D4A2E2A2EBE05D02E50C5
:1077480016E1500E2D5C13E22DC027F02EC028F054
:10775800273A283AF00E281627500F0B2812F00E59
:1077680027162350275C2450285801E225D7980E65
:107778009C6FF90E9D6FB1EF61F0838E8380506A24
:10778800B0EC3CF00101B66FB65102E0B651120000
:10779800996BAE6BAF6BB06BB16BB46B010EB36F23
:1077A800B96BCFD0B76BB86B1CD0A3EC5DF0215090
:1077B800221015E0B90E0E6E010E0F6EBEEC57F0DA
:1077C8000101B26F000E9925D96EDA6A040EDA2229
:1077D800B2C1DFFF992BB74BB82BB9BB05D08EAC24
:1077E80003D00101B805E1E30101B751AE27B85153
:1077F800AF23000EB023B12352501C0D170EF324F3
:10780800D96E010EF420DA6EDE50AE5DDE50AF594F
:10781800DE50B059DE50B15902E3B36BB46BB9AB6B
:1078280002D0B36BB46B8EBC02D0B36BB46BB8052B
:1078380019E2000E99250E6E0F6A040E0F22FF0E34
:107848009925D96EDA6A030EDA22DF50106E116AB2
:1078580099510008126E000ED8A0E82A0108136E8C
:10786800D2EC48F00101905145E07051711172114C
:10787800731140E052503EE152501C0D070EF324A4
:10788800D96E010EF420DA6E70C1A3F171C1A4F1B2
:1078980072C1A5F1A26B000EA225A66F010EA3214D
:1078A800A76F000EA421A86F000EA521A96FAA6BCF
:1078B800AB6BAC6BAD6BDE50A6191CE1DE50A719A3
:1078C80019E1DE50A81916E1DE50A91913E1DE50BE
:1078D800AA1910E1DE50AB190DE1DE50AC190AE12E
:1078E800DE50AD1907E1000E256E040E266E90518C
:1078F80077EC57F06DEC53F00101B56FB55121E00D
:107908006A0E00019C6FFB0E9D6FB5C19EF09F6BC8
:10791800B1EC61F0010E506E52501C0D1B0EF32499
:10792800D96E010EF420DA6E52501C0D1B0EF32492
:10793800E16E010EF420E26EE7500409DF6E50504C
:107948001200B351B41101E02DD78FA402D0010E5B
:10795800506E8390839E000C52501C0D070EF3242A
:10796800D96E010EF420DA6EDECFEBF0DECFECF04C
:10797800DECFEDF0DECFEEF052501C0D070EF324F3
:10798800D96E010EF420DA6E52501C0D0F0EF3243E
:10799800E16E010EF420E26EDE50E65CDE50E65841
:1079A800DE50E658DE50E658DE50E658DE50E6581F
:1079B800DE50E658DE50E65815E2010E506E525081
:1079C8001C0D1B0EF324D96E010EF420DA6E5250F2
:1079D8001C0D1B0EF324E16E010EF420E26EE7503D
:1079E8000409DF6E52501C0D070EF324D96E010EE8
:1079F800F420DA6EDECFC7F0DECFC8F0DECFC9F0F4
:107A0800DECFCAF0DECFCBF0DECFCCF0DECFCDF0CC
:107A1800DECFCEF052501C0D170EF324D96E010E96
:107A2800F420DA6EDECFCFF0DECFD0F0DECFD1F0AB
:107A3800DECFD2F00001CF51D36FD051D46FD151E6
:107A4800D56FD251D66FD76BD86BD96BDA6BC7515C
:107A5800D325DB6FC851D421DC6FC951D521DD6F27
:107A6800CA51D621DE6FCB51D721DF6FCC51D82137
:107A7800E06FCD51D921E16FCE51DA21E26F52503A
:107A88001C0D0F0EF324D96E010EF420DA6EDB51B3
:107A9800DE5CDC51DE58DD51DE58DE51DE58DF5148
:107AA800DE58E051DE58E151DE58E251DE5815E269
:107AB800010E506E52501C0D1B0EF324D96E010E90
:107AC800F420DA6E52501C0D1B0EF324E16E010EE9
:107AD800F420E26EE7500409DF6E506A5250220D1E
:107AE800380EF3249E6F020EF4209F6FEBC0A0F0B7
:107AF800ECC0A1F0EDC0A2F0EEC0A3F05EEC12F075
:107B0800EF6FEF5115E0010E506E52501C0D1B0E19
:107B1800F324D96E010EF420DA6E52501C0D1B0EA0
:107B2800F324E16E010EF420E26EE7500409DF6EE3
:107B3800505012008EA604D0AB0E216EFE0E03D05C
:107B4800B60E216EFF0E226E8EAA04D0AB0E236EE7
:107B5800FE0E03D0B10E236EFF0E246E8EA804D045
:107B6800AB0E256EFE0E03D0D80E256EFE0E266EC9
:107B78008EAE04D0AB0E276EFE0E03D0BB0E276E62
:107B8800FF0E286E8EAC04D0AB0E296EFE0E03D00D
:107B9800AC0E296EFF0E2A6E8EA404D0AB0E2B6E8F
:107BA800FE0E03D0C50E2B6EFF0E2C6E8EA204D0D7
:107BB800AB0E2D6EFE0E03D0CA0E2D6EFF0E2E6E6E
:107BC8008EA004D0AB0E2F6EFE0E03D0C00E2F6E0B
:107BD800FF0E306E90AE04D0AB0E316EFE0E03D0A9
:107BE800F80E316EFF0E326E90AC04D0AB0E336ED1
:107BF800FE0E03D0F50E336EFF0E346E90AA04D03D
:107C0800AB0E356EFE0E03D0F20E356EFF0E366EDD
:107C180090A804D0AB0E376EFE0E03D0EF0E376E71
:107C2800FF0E386E90A604D0AB0E396EFE0E03D050
:107C3800EC0E396EFF0E3A6E90A404D0AB0E3B6E7C
:107C4800FE0E03D0E90E3B6EFF0E3C6E90A204D0F0
:107C5800AB0E3D6EFE0E03D0E60E3D6EFF0E3E6E81
:107C680090A004D0AB0E3F6EFE0E03D0E30E3F6E25
:107C7800FF0E406E1E0E00019C6FF90E9D6F901C4A
:107C88009E6F9F6B8ECFA0F0A16B3FC0A2F040C04B
:107C9800A3F03DC0A4F03EC0A5F03BC0A6F03CC098
:107CA800A7F039C0A8F03AC0A9F037C0AAF038C088
:107CB800ABF035C0ACF036C0ADF033C0AEF034C078
:107CC800AFF031C0B0F032C0B1F02FC0B2F030C068
:107CD800B3F02DC0B4F02EC0B5F02BC0B6F02CC058
:107CE800B7F029C0B8F02AC0B9F027C0BAF028C048
:107CF800BBF025C0BCF026C0BDF023C0BEF024C038
:107D0800BFF021C0C0F022C0C1F0B1EF61F0070E92
:107D18000E241D6E000E0F201E6E0EC0D9FF0FC060
:107D2800DAFFDF50126E12380F0B0A0DF3CF13F083
:107D3800F4CF14F00EC0D9FF0FC0DAFFDF500F0BDD
:107D48001326000E142213281B6E000E14201C6E1E
:107D5800206A010E1F6E216A226A236A246AB2D041
:107D68001F50201054E021C012F022C013F023C08D
:107D780014F024C015F00A0E1202F3CF16F0F4CF57
:107D880017F0186A196A1302F3501726F4501822CC
:107D9800000E19221202F3501726F4501822000E72
:107DA80019220A0E1402F3501826F4501922000E54
:107DB8001302F3501826F4501922000E1202F35041
:107DC8001826F45019220A0E1502F3501926000E2F
:107DD8001402F3501926000E1302F3501926000E50
:107DE8001202F35019261DC0D9FF1EC0DAFFDF505A
:107DF8001A6E1A380F0B1624216E000E1720226EE9
:107E0800000E1820236E000E1920246E54D021C0B5
:107E180012F022C013F023C014F024C015F00A0E8B
:107E28001202F3CF16F0F4CF17F0186A196A13028A
:107E3800F3501726F4501822000E19221202F3509C
:107E48001726F4501822000E19220A0E1402F350B5
:107E58001826F4501922000E1302F3501826F45075
:107E68001922000E1202F3501826F45019220A0E95
:107E78001502F3501926000E1402F3501926000EAD
:107E88001302F3501926000E1202F35019261DC0D2
:107E9800D9FF1EC0DAFFDF500F0B1624216E000E2B
:107EA8001720226E000E1820236E000E1920246E53
:107EB8001D06D8A01E061F502010010ED8A4000EC3
:107EC8001F6E206A1B06D8A01C061B2802E11C286E
:107ED800D8A446D721C00EF022C00FF023C010F05E
:107EE80024C011F012000001D16B010ED06F838EF7
:107EF8008380D26BD36BD46BD56BCED05250220D0E
:107F0800380EF324746F020EF420756F350E766FF9
:107F18000B0E776F010E796F786BD80E7A6F7B6BCB
:107F2800F4EC17F0DA6FDA5118E0180E0101896FD6
:107F3800010E8B6F0001D96BD86F550E9C6FFA0E2E
:107F48009D6F52C09EF09F6BDAC0A0F0A16BD8C0A5
:107F5800A2F0D9C0A3F0B1EC61F00101905135E075
:107F6800705171117211731130E052500C0D040EE2
:107F7800F324D96E020EF420DA6E70C1C7F071C115
:107F8800C8F072C1C9F00001C66B000EC625CA6FE1
:107F9800010EC721CB6F000EC821CC6F000EC9217E
:107FA800CD6FDE50CA1911E1DE50CB190EE1DE505B
:107FB800CC190BE1DE50CD1908E1350E2B6E0B0EF6
:107FC8002C6E0101905133EC4FF00292010189515E
:107FD80003E002500209026E0001D8519AEC5AF0EF
:107FE80004C0D6F005C0D7F00001D651D227D7512A
:107FF800D323000ED423D5238EAC53D0D851D61911
:1080080003E1D951D7190CE0D06BD16B470E9C6FA7
:10801800FE0E9D6FD6C09EF0D7C09FF0B1EC61F008
:108028005DEC61F0A3EC5DF02150221004E0010E3C
:1080380001018B6F36D00001CF6B050ECE6F1CD0BF
:10804800D00E0001C26FC90EE82EFED7C22FFCD792
:1080580000D0A3EC5DF0215022100EE00001D06B9F
:10806800D16B190E9C6FFD0E9D6FCEC09EF0CFC0D8
:108078009FF0B1EC61F008D00001CE07D8A0CF077F
:10808800CE29DEE1CF29DCE1A3EC5DF021502210FE
:1080980003E00001D06BD16B0001D051D11101E098
:1080A8002DD701018B6B839E8390120046C027F069
:1080B80047C028F068EC44F0486E485001E0D4D03E
:1080C80046C0D9FF47C0DAFF030EDE1801E0BCD076
:1080D80020EE04F04650D9264750DA22DE0401E0AB
:1080E800B3D02F0E46240E6E000E47200F6E116A75
:1080F800106A020E136E126A28EC61F02D0E4624E7
:108108000E6E020E47200F6EAA0E116E550E106EDF
:10811800EEEC60F02F0E46240E6E000E47200F6E18
:10812800520E106E116E610E126E410E136E06EC39
:108138005BF0130E46240E6E020E47200F6E720E71
:10814800106E116E410E126E610E136E06EC5BF02E
:10815800170E46240E6E020E47200F6E20EE0FF00B
:108168004650D9264750DA22DECF10F0DECF11F084
:10817800DECF12F0DECF13F006EC5BF01B0E4624C8
:108188000E6E020E47200F6E20EE0BF04650D926D9
:108198004750DA22DECF10F0DECF11F0DECF12F03A
:1081A800DECF13F006EC5BF020EE1BF04650D9262C
:1081B8004750DA22DECF60F0DECF61F0DECF62F02A
:1081C800DECF63F0010E00016025646F000E6121AF
:1081D800656F000E6221666F000E6321676F20EEE7
:1081E8002BF04650D9264750DA2264C0DEFF65C01E
:1081F800DEFF66C0DEFF67C0DEFF2F0E46241D6E61
:10820800000E47201E6E20EE2BF04650D926475010
:10821800DA22DECF1FF0DECF20F0DECF21F0DECF76
:1082280022F0246A010E236E20EE01F04650D92672
:108238004750DA22DF5094EC50F020EE04F046501C
:10824800D9264750DA22DF6A1D6A1E6A1F6A20EEA5
:1082580001F04650D9264750DA22DF500DEC21F0C4
:10826800000902E0010E486E485012009051D8B43F
:108278001200390E00019C6FFD0E9D6FB1EC61F08C
:1082880022EC55F021C0AAF122C0ABF123C0ACF119
:1082980024C0ADF10101AA51AB11AC11AD1117E128
:1082A800250E00019C6FFC0E9D6FAAC19EF0ABC10C
:1082B8009FF0ACC1A0F0ADC1A1F0B1EC61F00A0E25
:1082C800116E000E126A136A146AB3EC5CF00101B5
:1082D800AE6BAF6BDB0E00019C6FFF0E9D6FAA0E9D
:1082E8000101AE25D96E010EAF21DA6EDF50000113
:1082F8009E6F9F6BB1EC61F00101AE4BAF2BAFBF2E
:10830800E9D7AF5103E1040EAE5DE4E3980E000136
:108318009C6FF90E9D6FB1EC61F0EC0E9C6FFA0E3C
:108328009D6FB1EC61F022EE38F000EEC7F0210E3F
:10833800DBCFEBFFE806FCE2D30EE96FFF0EEA6F36
:108348007DEC36F0C7C070F1C8C071F1C9C072F1D8
:10835800CAC073F101017051711172117311D8B44F
:108368001200D20E00019C6FFA0E9D6F70C19EF034
:1083780071C19FF072C1A0F073C1A1F0B1EC61F0BE
:10838800380E9E6F020E9F6F70C1F8F071C1F9F040
:1083980072C1FAF0F76B000EF725A06F010EF821F5
:1083A800A16F000EF921A26F000EFA21A36F5EECF7
:1083B80012F00101966F380E0001746F020E756F8E
:1083C800350E766F0B0E776F796B080E786FA80EE7
:1083D8007A6F010E7B6FF4EC17F00101966FB06BAA
:1083E800B16B1C0E00019C6FFF0E9D6F350E0101D5
:1083F800B025D96E0B0EB121DA6EDF5000019E6FE9
:108408009F6BB1EC61F00101B04BB12BB1BFE9D763
:10841800B15105E1080EB05DD8B01200E2D71200E4
:10842800C0C0D9FFC1C0DAFFDECFCAF0DDCFCBF0C4
:1084380003D00001C24BC32BC2C0F6FFC3C0F7FF75
:10844800000EF86E0E0EF76403D00800F55005D044
:10845800F6CFE9FFF7CFEAFFEF502F0AEAE0C2C0F4
:10846800F6FFC3C0F7FF000EF86E0E0EF76403D0D8
:108478000800F55005D0F6CFE9FFF7CFEAFFEF5037
:108488005C0AD7E0000120EE06F0C051D926C151A0
:10849800DA22DE6ADE6ADE6ADD6AC2C0F6FFC3C0BF
:1084A800F7FF000EF86E0E0EF76403D00800F550C3
:1084B80005D0F6CFE9FFF7CFEAFFEF500001C46F10
:1084C800200EC46114D020EE27F0C051D926C15126
:1084D800DA22800EDF6EC0C074F0C1C075F0000EE5
:1084E800766F776F786F796F0CEC35F023D0C0C05A
:1084F80016F0C1C017F0C20E186EADEC37F00001CF
:10850800CD6FCD5158E1C0C0B8F0C1C0B9F068EC2A
:1085180049F0CD6F20EE27F0C051D926C151DA229B
:10852800DF50CC6FCD5108E0040ECD1944E1CCB535
:1085380042D0050ECD6F3FD0CCB53DD020EE04F033
:10854800C051D926C151DA22DFA8F3D7CAC015F025
:10855800CBC016F0C469010EC56F20EE0EF0C051F5
:10856800D926C151DA22DECFC6F0DDCFC7F0C4511B
:10857800C617C551C717CAC0C8F0CBC0C9F0C65185
:10858800C827C751C9232F0EC825176E000EC92149
:10859800186E80EC59F0000120EE06F0C051D92683
:1085A800C151DA2215C0DEFF16C0DEFF17C0DEFF9C
:1085B80018C0DEFF9CD7CD51120081C0D9FF82C000
:1085C800DAFFDECF98F0DDCF99F08651851184115E
:1085D80004E1020E835DD8A0020C20EE13F098513E
:1085E800D9269951DA22DE50835DDE508459DE5057
:1085F8008559DE50865901E3020C8751881189118B
:108608008A1117E098C060F099C061F087C062F0E5
:1086180088C063F089C064F08AC065F066696769DC
:1086280068696969F0EC1EF0976F975102E09751FD
:10863800120081C045F082C046F083C047F084C074
:1086480048F085C049F086C04AF0DDEC2CF045C002
:1086580093F046C094F047C095F048C096F00001EA
:10866800935194119511961170E0930594119511F9
:10867800961101E1020C932907E1942905E1952956
:1086880003E1962901E1010C98C060F099C061F0FE
:1086980083C062F084C063F085C064F086C065F072
:1086A800666B676B686B696BF0EC1EF0976F9751A0
:1086B800BEE120EE13F09851D9269951DA22FE0E28
:1086C800DE248B6FFF0EDE208C6FFF0EDE208D6F99
:1086D800FF0EDE208E6F20EE0FF09851D9269951AB
:1086E800DA228B51DE5C8C51DE588D51DE588E516A
:1086F800DE5813E220EE0FF09851D9269951DA226C
:10870800DE2A000EDE22DE22DE2220EE04F0985160
:10871800D9269951DA22000EDB8093C083F094C0E9
:1087280084F095C085F096C086F020EE13F098513D
:10873800D9269951DA22DE50835DDE508459DE5005
:108748008559DE50865901E274D7000C1E6E1E5002
:1087580001E0010C55A202D055501200000EDAECCF
:1087680060F00A0E296E03D0CDEC61F0290629507D
:10877800FBE1266A000E176A186A196A1A6A5CEC25
:108788005FF0E80601E097D0AA0E176E010E186E8A
:10879800196A1A6A080E5CEC5FF0E80651E1296A6A
:1087A80029501F0FD96EDA6ACDEC61F0DF6E292AE5
:1087B800030E2964F5D721047EE1AA0E22187BE175
:1087C800030E286EE80E276E15D0176A186A196A04
:1087D800400E1A6EA90E5CEC5FF000090EE0150E53
:1087E8001D6EC60EE82EFED71D2EFCD700D027061C
:1087F800D8A0280627502810E8E1275028105BE069
:10880800176A186A196A1A6A3A0E5CEC5FF000096E
:1088180052E1296A29501F0FD96EDA6ACDEC61F04E
:10882800DF6E292A030E2964F5D71FBC03D0246AFA
:10883800040E02D0246A0C0E236E23C026F03BD00F
:10884800176A186A196A1A6AA90E5CEC5FF01D6E3D
:10885800020E1D6003D0266EA90E02D0010E266EF0
:10886800256E030E286EE80E276E14D0176A186A54
:10887800196A1A6A25505CEC5FF000090EE0150EC3
:108888001D6EC60EE82EFED71D2EFCD700D027067B
:10889800D8A0280627502810E9E1275028100AE018
:1088A800176A020E186E196A1A6A100E5CEC5FF0ED
:1088B800000901E0266A26C053F0DEEC61F026507C
:1088C80001E14AD7559048D7396A20EE03F027507E
:1088D800D9262850DA22DF5001E1A7D02F0E27240D
:1088E8001D6E000E28201E6E20EE2BF02750D92674
:1088F8002850DA22DECF1FF0DECF20F0DECF21F0C5
:10890800DECF22F0246A010E236E20EE01F02750FC
:10891800D9262850DA22DF5094EC50F0000901E003
:1089280082D020EE03F02750D9262850DA22DF6AB9
:1089380020EE17F02750D9262850DA2210EE1FF023
:108948002750E1262850E222E6CF2DF0E6CF2EF080
:10895800E6CF2FF0E6CF30F010EE2BF02750E126CF
:108968002850E222E6CF31F0E6CF32F0E6CF33F0FE
:10897800E6CF34F02D50315C356E2E503258366EBD
:108988002F503358376E30503458386EDE50355CBF
:10899800DE503658DE503758DE50385846E220EE62
:1089A80002F02750D9262850DA22020EDE183DE1BF
:1089B8002F0E27241D6E000E28201E6E20EE17F0A5
:1089C8002750D9262850DA22DECF29F0DECF2AF028
:1089D800DECF2BF0DECF2CF020EE2BF02750D9265F
:1089E8002850DA22DECF2DF0DECF2EF0DECF2FF0AA
:1089F800DECF30F029502D241F6E2A502E20206EF5
:108A08002B502F20216E2C503020226E246A010E0C
:108A1800236E20EE01F02750D9262850DA22DF50A5
:108A280094EC50F002D0010E396E3950120049C052
:108A38000FF04AC010F0690E116E26EC54F00001D8
:108A4800686F685101E099D020EE0EF04950D926A0
:108A58004A50DA22DFAC91D069C03AF06AC03BF0E4
:108A680020EE1CF04950D9264A50DA22DECF3CF0DD
:108A7800DECF3DF0DECF3EF0DECF3FF071EC55F0BB
:108A88000001686F685179E120EE20F04950D9263D
:108A98004A50DA22DECF6BF0DDCF6CF020EE0BF01F
:108AA8006B51D9266C51DA22000EDB8A49C0D9FFF6
:108AB8004AC0DAFFDECF12F0DDCF13F06BC014F03E
:108AC8006CC015F020EE06F04950D9264A50DA223B
:108AD800DECF16F0DECF17F0DECF18F0DECF19F0BC
:108AE8008CEC5EF01C0E00016B250E6E000E6C21E6
:108AF8000F6E20EE0AF04950D9264A50DA22DECF0E
:108B080010F0DECF11F0DECF12F0DECF13F006EC5E
:108B18005BF0160E00016B250E6E000E6C210F6EB9
:108B2800106A116A210E126E500E136E06EC5BF07D
:108B3800120E00016B250E6E000E6C210F6E000EDA
:108B4800116A106AEEEC60F0000120EE03F0695142
:108B5800D9266A51DA22010EDF6E69C046F06AC072
:108B680047F05AEC40F00001686F20EE0EF04950D3
:108B7800D9264A50DA22BF0EDF16685112008968DA
:108B88008B688E280BE1390E00019C6FFB0E9D6FE0
:108B98008ECF9EF09F6BB1EC61F00AD00D0E0001F4
:108BA8009C6FFA0E9D6F8ECF9EF09F6BB1EC61F0BB
:108BB80090280AE10E0E9C6FFC0E9D6F8ECF9EF0E2
:108BC8009F6BB1EC61F009D0320E9C6FFA0E9D6F6D
:108BD8008ECF9EF09F6BB1EC61F0290E426E960E1F
:108BE800416E7F0EE82EFED7412EFCD7422EFAD7D3
:108BF80000F0610E00019C6FFE0E9D6FB1EC61F0FC
:108C080089988498090E426E1E0E416EE40EE82E75
:108C1800FED7412EFCD7422EFAD700D0540E0001C1
:108C28009C6FFE0E9D6FB1EC61F0899A849A090ED3
:108C3800426E1E0E416EE40EE82EFED7412EFCD782
:108C4800422EFAD700D0C60E00019C6FFE0E9D6F13
:108C5800B1EC61F088908D9090280AE00E0E9C6F20
:108C6800FC0E9D6F90CF9EF09F6BB1EC61F009D028
:108C7800C20E9C6FF90E9D6F90CF9EF09F6BB1EC6A
:108C880061F08D80A30E426E570E416E020EE82EE3
:108C9800FED7412EFCD7422EFAD700D089688B68C0
:108CA8008A6883928382290E426E960E416E7F0EE9
:108CB800E82EFED7412EFCD7422EFAD700F09EECC4
:108CC8003DF0EFD71F6A1DAE12D01D1E1C1E1B1EC5
:108CD8001A1E191E181E171E166C000E17221822AF
:108CE80019221A221B221C221D22010E1F6E15AEEC
:108CF80012D0151E141E131E121E111E101E0F1E3A
:108D08000E6C000E0F22102211221222132214229E
:108D18001522010E1F1A206A216A226A236A246A10
:108D2800256A266A276A16501710181019101A1083
:108D38001B101C101D1045E0010E1E6E0AD0D890A5
:108D480016361736183619361A361B361C361D369F
:108D58001E2A1DAEF4D7D890203621362236233667
:108D6800243625362636273616500E5C17500F58EF
:108D780018501058195011581A5012581B5013589F
:108D88001C5014581D50155811E316500E5E1750FC
:108D98000F5A1850105A1950115A1A50125A1B507B
:108DA800135A1C50145A1D50155A2080D8901D3241
:108DB8001C321B321A3219321832173216321E2E52
:108DC800CAD71F5010E0271E261E251E241E231E4C
:108DD800221E211E206C000E212222222322242260
:108DE80025222622272220C00EF021C00FF022C003
:108DF80010F023C011F024C012F025C013F026C0D3
:108E080014F027C015F01200176818680E50D96EB4
:108E1800DA6ADECF19F0DDCF1AF019C014F01AC0E3
:108E280015F019501A1003E10E680F68120014C0EB
:108E3800F6FF15C0F7FF000EF86E0E0EF76403D0AC
:108E48000800F55005D0F6CFE9FFF7CFEAFFEF505D
:108E5800166E144A152A200E166403D03A0E1618F8
:108E6800E6E13A0E161868E1000E136E010E126E56
:108E780019C0F6FF1AC0F7FF000EF86E0E0EF76461
:108E880003D00800F55005D0F6CFE9FFF7CFEAFF89
:108E9800EF50106E2F0E106439D019C0F6FF1AC0AB
:108EA800F7FF000EF86E0E0EF76403D00800F550B9
:108EB80005D0F6CFE9FFF7CFEAFFEF50106E3A0E74
:108EC800106024D0020E1924106E000E1A20116EA4
:108ED800145010181BE11550111818E119C0F6FFAD
:108EE8001AC0F7FF000EF86E0E0EF76403D00800E4
:108EF800F55005D0F6CFE9FFF7CFEAFFEF50106E37
:108F0800D00E1024126E136AFF0E132213BE04D063
:108F180013500DE112040BE212C017F013C018F041
:108F28000E50D96EDA6A14C0DEFF15C0DDFF17C017
:108F38000EF018C00FF012000E6A0F6A120060C01F
:108F480045F061C046F0476A486A496A4A6AB6EC21
:108F58004EF045C078F046C079F0020E000178194D
:108F680079110DE0795106E1030E785D03E2625153
:108F7800631105E178C060F079C061F012007A6B86
:108F88007B6B7AC064F07BC065F0643B653BF00E98
:108F9800651764510F0B6513F00E641760C066F017
:108FA80061C067F06451662765516723F50E662531
:108FB8000E6E010E67210F6E7CEC54F000017A51A1
:108FC800040DF350680FD96EDA6A0EC0DEFF0FC0C9
:108FD800DEFF10C0DEFF11C0DEFF7A4B7B2B7B511A
:108FE80003E1040E7A5DCDE36251631103E17A6B0C
:108FF8007B6B06D0FF0E62257A6FFF0E63217B6FB5
:109008007A51040DF350680FD96EDA6ADE50DE101B
:10901800DE10DE1004E1796B030E786F18D060C0A3
:1090280045F061C046F07A51040DF350680FD96ECF
:10903800DA6ADECF47F0DECF48F0DECF49F0DECF88
:109048004AF0B6EC4EF045C078F046C079F0000121
:10905800625163118FE1795103E1020E785D8AE371
:109068007A4B7B2B7B5186E1040E7A5D83E2C8D76D
:109078002F6C696664617461302E62696E20002FFE
:109088006C696664617461312E62696E20002F6CB0
:10909800696664617461322E62696E20002F6C69A2
:1090A8006664617461332E62696E20002F6C696694
:1090B80064617461342E62696E20002F6C69666485
:1090C800617461352E62696E20002F6C6966646177
:1090D8007461362E62696E20002F6C696664617453
:1090E80061372E62696E20002F6C69666461746155
:1090F800382E62696E20002F6C696664617461396C
:109108002E62696E20002F6C696664617461612E3D
:1091180062696E20002F6C696664617461622E62F8
:10912800696E20002F6C696664617461632E6269E0
:109138006E20002F6C696664617461642E62696ECA
:1091480020002F6C696664617461652E62696E2007
:10915800002F6C696664617461662E62696E200016
:1091680000000000000000000000000000000000F7
:1091780000000000000000000000000000000000E7
:1091880000000000000000000000000000000000D7
:109198000000000000000000000000000EC018F0F1
:1091A8000FC019F01250131001E1120018C0D9FFB6
:1091B80019C0DAFF10C0DFFF12501824146E1350C4
:1091C8001920156EFF0E1424D96EFF0E1520DA6EC5
:1091D80010C0DFFF135004E1030E125C01E212001D
:1091E80020EE01F01850D9261950DA2210C0DFFFFE
:1091F80020EE02F01850D9261950DA2210C0DFFFED
:1092080012501824146E13501920156EFE0E1424D3
:10921800D96EFF0E1520DA6E10C0DFFF1250182429
:10922800146E13501920156EFD0E1424D96EFF0EFE
:109238001520DA6E10C0DFFF135004E1070E125C30
:1092480001E2120020EE03F01850D9261950DA2254
:1092580010C0DFFF12501824146E13501920156E19
:10926800FC0E1424D96EFF0E1520DA6E10C0DFFF35
:10927800135004E1090E125C01E2120018C014F048
:1092880019C015F0141E151E144A152A030E1414BD
:10929800166E176A16501826175019221650125EA5
:1092A8001750135AFC0E12160BD018C0D9FF19C04C
:1092B800DAFF10C0DFFF1206D8A01306184A192AD1
:1092C80012501310F2E11200B8C0D9FFB9C0DAFF8A
:1092D800DECFBCF0DDCFBDF0B8C074F0B9C075F01A
:1092E800000E766F776F786F796F0CEC35F0BF6F83
:1092F800BF5103E00001BF511200BCC03AF0BDC02D
:109308003BF020EE16F0B851D926B951DA22DECF5B
:109318003CF0DECF3DF0DECF3EF0DECF3FF071EC2B
:1093280055F00001BF6FBF51E5E120EE1AF0B851CA
:10933800D926B951DA22DECFBAF0DDCFBBF0BAC0F8
:10934800D9FFBBC0DAFFDF50BE6FBE5103E1040E88
:10935800BF6FD0D720EE04F0B851D926B951DA2220
:1093680010EE1AF0B851E126B951E22200EE0BF0E6
:10937800E650E926E550EA22EF503F0BDF6E20EE7B
:109388001AF0B851D926B951DA2210EE0BF0DE5096
:10939800E126DD50E222E7B618D020EE1AF0B851E7
:1093A800D926B951DA22DECF0EF0DDCF0FF01C0E30
:1093B800B825106E000EB921116E136A0B0E126ECD
:1093C800D0EC5AF00E500F1095E0B8C09EF0B9C01E
:1093D8009FF00001A16BA06BF1EC31F00001BF6FB1
:1093E800BF5188E18AD71BC00EF01CC00FF0116A6C
:1093F800106A136A080E126ED2EC48F0266A020E42
:10940800256E25501B24D96E26501C20DA6E255057
:109418001B24216E26501C20226E2128E16E000E8E
:109428002220E26EE750236E233AF00E231623160D
:1094380025501B24E16E26501C20E26EE750246E56
:1094480024380F0B2310DF6E254A262A26BED9D7CB
:10945800265003E1070E255CD4E325501B24D96E62
:1094680026501C20DA6E1DC00EF01EC00FF01FC063
:1094780010F020C011F00A0E126E136A146A156AF1
:10948800A4EC5BF00E3AF00E0E1625501B24E16E8C
:1094980026501C20E26EE750216E21380F0B0E106B
:1094A800DF6E1BC0D9FF1CC0DAFFDF2A1DC00EF01B
:1094B8001EC00FF01FC010F020C011F00A0E126E6F
:1094C800136A146A156A45EC59F00EC01DF00FC0F6
:1094D8001EF010C01FF011C020F01D501E101F10EC
:1094E80020108CE11BC0D9FF1CC0DAFFDF06090E73
:1094F800DF64090C1BC0D9FF1CC0DAFF100EDF6E39
:10950800100C000E0101DC6F0A0EDB6F000EDA6F23
:10951800050ED96F7DD00101DC6B140EDB6F70D0A6
:10952800650E0F6EFC0E106E89EC5CF08FB204D0E5
:109538000101DC6B1E0EDB6F090E0001FE6F1E0EB3
:10954800FD6FE40EE82EFED7FD2FFCD7FE2FFAD7CD
:1095580000F056D0AE0E0F6EFE0E106E89EC5CF069
:10956800060E0001B16F090EB26F9A0EB36FF90EB5
:10957800B46FB56BE8EC56F00101966F965105ECA7
:109588005DF001019651D8E1DC6B230ED4D7F20EC1
:109598000F6EFD0E106E89EC5CF0380E0001CE6F78
:1095A800020ECF6FE20ED06F020ED16F010ED26F96
:1095B8002CEC15F00101966F965105EC5DF0010158
:1095C80096510AE139EC29F0380E6D6F020E6E6F74
:1095D800E9EC5EF00101966F965105EC5DF0010C27
:1095E800DBC1FDF0DCC1FEF00001FE5109E1FD51D7
:1095F8000A0A91E01E0A94E00A0AACE03D0AC7E0B4
:10960800140E0101DB19DC1103E0D907D8A0DA0731
:10961800DABF000CDA51E4E1D905E2E2000C1F6A76
:1096280015AE12D0151E141E131E121E111E101E6A
:109638000F1E0E6C000E0F2210221122122213226E
:1096480014221522010E1F6E1DAE10D01D1E1C1EE9
:109658001B1E1A1E191E181E171E166C000E172226
:10966800182219221A221B221C221D2216501710FA
:10967800181019101A101B101C101D103BE0010EB9
:109688001E6E0AD0D89016361736183619361A367E
:109698001B361C361D361E2A1DAEF4D716500E5C1E
:1096A80017500F5818501058195011581A5012586E
:1096B8001B5013581C5014581D50155810E31650C1
:1096C8000E5E17500F5A1850105A1950115A1A5046
:1096D800125A1B50135A1C50145A1D50155AD89020
:1096E8001D321C321B321A32193218321732163216
:1096F8001E2ED4D71F5010E0151E141E131E121E46
:10970800111E101E0F1E0E6C000E0F2210221122A9
:1097180012221322142215220EC00EF00FC00FF0D1
:1097280010C010F011C011F012C012F013C013F0E5
:1097380014C014F015C015F01200020E105E000ED1
:10974800115A125A135A20EE13F00E50D9260F5000
:10975800DA22FE0EDE24146EFF0EDE20156EFF0EDA
:10976800DE20166EFF0EDE20176E1450105C1550AA
:109778001158165012581750135805E30E6A0F6AFD
:10978800106A116A120020EE27F00E50D9260F50E9
:10979800DA22DECF14F0DECF15F0DECF16F0DECF02
:1097A80017F020EE09F00E50D9260F50DA22DECF3E
:1097B80018F0DDCF19F018501A6E19501B6E1C6A7C
:1097C8001D6A1A501002F3CF1EF0F4CF1FF0206A62
:1097D800216A1102F3501F26F4502022000E212284
:1097E8001B501002F3501F26F4502022000E212295
:1097F8001A501202F3502026F45021221B50110255
:10980800F3502026F45021221C501002F350202639
:10981800F450212213501A02F35021261B50120231
:10982800F35021261C501102F35021261D5010021E
:10983800F350212614501E240E6E15501F200F6E53
:1098480016502020106E17502120116E1200838EA2
:1098580083800001FB6BFC6B09EC59F025C0FDF01F
:1098680026C0FEF0040E0001FE5D07E3000EFD2594
:10987800FB6FFC0EFE21FC6F04D0FDC0FBF0FEC0A8
:10988800FCF00101905133E07051711172117311A4
:109898002EE052500C0D040EF324D96E020EF42063
:1098A800DA6E70C19FF171C1A0F172C1A1F19E6B16
:1098B800000E9E25A26F010E9F21A36F000EA0210E
:1098C800A46F000EA121A56FDE50A21910E1DE5091
:1098D800A3190DE1DE50A4190AE1DE50A51907E12C
:1098E800000E256E040E266E905177EC57F08FB45B
:1098F80015D05250220D380EF32400019E6F020E2F
:10990800F4209F6F000EA06F040EA16F010EA36FCD
:10991800A26BFB0EA46FCEEC08F0FA6F0001FA51AF
:1099280009E0290E9C6FFD0E9D6FFAC09EF09F6B9B
:10993800B1EC61F03EEC27F08B6B8390839EC40EF4
:1099480000019C6FFC0E9D6FCECF9EF09F6BCDCF1C
:10995800A0F0A16BB1EF61F0FCC123F071D03BEC3A
:1099680061F0236EFC1979E0290E226E960E216EA5
:109978007F0EE82EFED7212EFCD7222EFAD700F034
:109988006CD07EEC5DF0246E245067E024B0542A3D
:1099980024B254060F0E5416000E0E6EC00E56EC6E
:1099A8005DF0C5EC60F0000E0E6EC00E56EC5DF07A
:1099B80054500F0D350EF324126E0D0EF420136E55
:1099C800CCEC58F0110E226E3C0E216ECB0EE82E18
:1099D800FED7212EFCD7222EFAD700F024A43DD0A2
:1099E8000F6A0E6A54C010F023EC5FF0510E0001AC
:1099F8009C6FFC0E9D6F54C09EF09F6BB1EC61F0A4
:109A080054C023F0000E0E6E800E56EC5DF0C5ECCF
:109A180060F0000E0E6E800E56EC5DF054500F0D87
:109A2800350EF324126E0D0EF420136ECCEC58F0A4
:109A3800000E0E6EC00E56EC5DF0C5EC60F00DD059
:109A480001019251216E226A225007E12150010A38
:109A580086E0030A84E0010A94E0235012003AC029
:109A680027F03BC028F068EC44F0000901E0010C45
:109A78003AC00EF03BC00FF03CC010F03DC011F0F2
:109A88003EC012F03FC013F0A1EC4BF00EC044F002
:109A98000FC045F010C046F011C047F020EE2BF083
:109AA8003A50D9263B50DA2244C0DEFF45C0DEFFDB
:109AB80046C0DEFF47C0DEFF2F0E3A240E6E000EB2
:109AC8003B200F6E116A106A020E136E126A28ECA0
:109AD80061F02F0E3A24426E000E3B20436E496A15
:109AE800010E486E4A6A4B6A04D048504A264950CB
:109AF8004B2220EE09F03A50D9263B50DA22DE50AC
:109B08004A5CDE504B581FE242C01DF043C01EF0B5
:109B18004A5044241F6E4B504520206E000E4620AC
:109B2800216E000E4720226E48C023F049C024F061
:109B380020EE01F03A50D9263B50DA22DF5094EC5F
:109B480050F00009D2E020EE09F03A50D9263B50F7
:109B5800DA224A50DE1803E14B50DE18D8A4010C73
:109B6800000C226A236A1B6A1C6A01D0152A010E9E
:109B7800216E1550D96EDA6A200EDE1813E0F70E42
:109B8800176E18681550D96EDA6ADF50196E1A6A9E
:109B98001750192618501A221A5003E1050E195C9D
:109BA80001E3216A21C01DF01E6A1D501E1006E047
:109BB800DDD71C6A010E1B6E152A25D01550D96EEB
:109BC800DA6ADF50176E186A18501DE117502B0A11
:109BD800F3E0060AEEE017D00A0E2202F3CF17F0E0
:109BE800F4CF18F02302F35018261550D96EDA6A0C
:109BF800DF50175E000E185A300E1724226E000E22
:109C08001820236ED9D7D00E176E18681550D96E44
:109C1800DA6ADF50196E1A6A1750192618501A2274
:109C28001A5005E10A0E195C02E2010E01D0000E7D
:109C38001F6E206A1F502010CFE11B501C100DE131
:109C480022C017F023C018F0171E181E174A182A2A
:109C580017C015F018C016F0120022C015F023C066
:109C680016F01200818E819C780EF66E900EF76EBB
:109C7800000EF86E0DEE35F011EE2CF00900F5CF60
:109C8800EEFFE550E150FAE1E250F8E1140EF66E0D
:109C9800AC0EF76E000EF86E03EE00F010EE94F0C6
:109CA8000900F5CFEEFFE550E150FAE14C0EF66EF3
:109CB800C30EF76E000EF86E02EEE2F010EE15F02D
:109CC8000900F5CFEEFFE550E150FAE1D60EF66E49
:109CD800C30EF76E000EF86E01EEF7F010EE04F00A
:109CE8000900F5CFEEFFE550E150FAE1E40EF66E1B
:109CF800C30EF76E000EF86E0900F5CF55F005EEAD
:109D080000F018EE35F0EE6AE550E150FCE1E25063
:109D1800FAE104EE00F011EE00F0EE6AE550E150D1
:109D2800FCE1E250FAE103EE94F0200EEE6AE80658
:109D3800FDE102EE00F0E20EEE6AE806FDE101EE5A
:109D480000F09A0EEE6AE806FDE100EE4CF0090E0E
:109D5800EE6AE806FDE156905692000EF86E000194
:109D680038EF0FF020EE03F04550D9264650DA229E
:109D7800DF6A20EE2BF04550D9264650DA22DE68FD
:109D8800DE68DE68DD6845C03AF046C03BF047C093
:109D98003CF048C03DF049C03EF04AC03FF071EC8D
:109DA80055F0000904E0466A040E456E040C2D0EB9
:109DB80045240E6E020E46200F6EC9EC5FF0550E5C
:109DC8000E1803E1AA0E0F1804E0466A030E456E4A
:109DD800030C20EE2FF04550D9264650DA22E90E22
:109DE800DE1812E020EE2FF04550D9264650DA2230
:109DF800EB0EDE1809E020EE2FF04550D92646502C
:109E0800DA22E80EDE1827E1650E45240E6E000EF4
:109E180046200F6ECF0E106EFF0E116E136A030EE2
:109E2800126ED0EC5AF00E500F1003E1456A466AE4
:109E38001200810E45240E6E000E46200F6E890E0C
:109E4800106EFF0E116E136A050E126ED0EC5AF0EA
:109E58000E500F10EBE0466A020E456E020C2F6E94
:109E6800A00E00019C6FFC0E9D6F2FC09EF09F6B93
:109E78002BC0A0F02CC0A1F0B1EC61F05DD022ECB9
:109E880055F021C030F022C031F023C032F024C098
:109E980033F02BC0D9FF2CC0DAFFDF6A20EE01F0C7
:109EA8002B50D9262C50DA2233C0DFFF20EE02F0E7
:109EB8002B50D9262C50DA22DF6A20EE03F02B50E3
:109EC800D9262C50DA2232C0DFFF20EE04F02B50C6
:109ED800D9262C50DA22DF6A20EE05F02B50D9263D
:109EE8002C50DA2231C0DFFF20EE06F02B50D926A5
:109EF8002C50DA22DF6A20EE07F02B50D9262C509E
:109F0800DA2230C0DFFF120022EC55F021C030F019
:109F180022C031F023C032F024C033F02BC01BF034
:109F28002CC01CF030C01DF031C01EF032C01FF034
:109F380033C020F0F7EF49F02F502D6E2E6A2E50C7
:109F4800D8A412002D50010A9AE0030ADDE012009D
:109F58000001FC6B8380838E6AD009EC59F025C020
:109F6800FAF026C0FBF0040E0001FB5D03E3010ECE
:109F7800FC6F03D0FFC0FDF0FE6B8FB414D05250BD
:109F8800220D380EF3249E6F020EF4209F6F000EF0
:109F9800A06F040EA16F010EA36FA26BFD0EA46F3C
:109FA800CEEC08F0FF6FFF5109E0290E9C6FFD0E03
:109FB8009D6FFFC09EF09F6BB1EC61F00101905165
:109FC80033E070517111721173112EE052500C0D63
:109FD800040EF324D96E020EF420DA6E70C19FF1DC
:109FE80071C1A0F172C1A1F19E6B000E9E25A26FF6
:109FF800010E9F21A36F000EA021A46F000EA121C6
:10A00800A56FDE50A21910E1DE50A3190DE1DE5054
:10A01800A4190AE1DE50A51907E1000E256E040E09
:10A02800266E905177EC57F03EEC27F08B6B0001D1
:10A03800FC5193E0839E839012000F015969116BC4
:10A04800196B216B8C948C928C90889A110E136EDC
:10A058003C0E126ECB0EE82EFED7122EFCD7132E16
:10A06800FAD700F0110E136E3C0E126ECB0EE82ECE
:10A07800FED7122EFCD7132EFAD700F0020E136E5D
:10A08800A00E126E920EE82EFED7122EFCD7132EBB
:10A09800FAD700D0000E0E6E300E56EC5DF02A0E88
:10A0A800126E8E0EE82EFED7122EFCD7000E0E6E04
:10A0B800300E56EC5DF0000E0E6E300E56EC5DF074
:10A0C800000E0E6E390E56EC5DF0000E0E6E140E7C
:10A0D80056EC5DF0000E0E6E560E56EC5DF0000E5E
:10A0E8000E6E6D0E56EC5DF0000E0E6E700E56EC98
:10A0F8005DF0000E0E6E0C0E56EC5DF0000E0E6E4E
:10A10800060E56EC5DF0000E0E6E010E56EC5DF07C
:10A11800D00E126ECA0EE82EFED7122EFCD71200F1
:10A12800266E2650D8A4040C2350241001E1040CF8
:10A1380055B0030C55B4020C53B608D0090ED8908C
:10A148001F36203621362236E82EF9D7230424106C
:10A158001AE11FC017F020C018F021C019F022C062
:10A168001AF0180E5CEC5FF0000945E11DC010F014
:10A178001EC011F0FE0E126E5FEC5CF000093BE0B1
:10A18800236A246A38D053C025F0060E251609E044
:10A1980023C017F024C018F0196A1A6A970E5CECED
:10A1A8005FF01FC017F020C018F021C019F022C0BE
:10A1B8001AF0190E5CEC5FF000091DE11DC010F0EB
:10A1C8001EC011F0FC0E126E5FEC5CF0000908E096
:10A1D800020E1E262306D8A0240623502410EEE1E2
:10A1E800106A116AFD0E126E5FEC5CF0000903E163
:10A1F800246A010E236EDEEC61F023502410D8A4EB
:10A20800010C000CB8C0D9FFB9C0DAFFDECFBFF02F
:10A21800DDCFC0F0B8C074F0B9C075F0000E766F2D
:10A22800776F786F796F0CEC35F0C36FC35153E1DA
:10A23800C16BC26BBFC03AF0C0C03BF020EE16F055
:10A24800B851D926B951DA22DECF3CF0DECF3DF045
:10A25800DECF3EF0DECF3FF071EC55F00001C36F6A
:10A26800C35139E120EE1AF0B851D926B951DA2292
:10A27800DECFBCF0DDCFBDF0BCC0D9FFBDC0DAFF7A
:10A28800E50EDE1810E020EE1AF0B851D926B951C3
:10A29800DA22DECFBCF0DDCFBDF0BCC0D9FFBDC037
:10A2A800DAFFDF5009E1C14BC22BBA51C11906E1EF
:10A2B800BB51C21910E002D0C16BC26BB8C09EF08E
:10A2C800B9C09FF0A16B010EA06FF1EC31F0000155
:10A2D800C36FC351AFE0040EC31902E1070EC36F89
:10A2E800C3511200838E83800001D16BD26BD36B74
:10A2F800D46B5250220D380EF324746F020EF420E2
:10A30800756F350E766F0B0E776F010E796F786B60
:10A31800D50E7A6F7B6BF4EC17F0D06F010190517A
:10A3280035E0705171117211731130E052500C0DFB
:10A33800040EF324D96E020EF420DA6E70C1C7F051
:10A3480071C1C8F072C1C9F00001C66B000EC62504
:10A35800CA6F010EC721CB6F000EC821CC6F000E4B
:10A36800C921CD6FDE50CA1911E1DE50CB190EE1BB
:10A37800DE50CC190BE1DE50CD1908E1350E2B6EFD
:10A388000B0E2C6E0101905133EC4FF0029200013C
:10A39800D5519AEC5AF004C0CEF005C0CFF00001B8
:10A3A800CE51D127CF51D223000ED323D42301017C
:10A3B8008B6B839E83901200B50E00019C6FFA0E82
:10A3C8009D6FCECF9EF09F6BCDCFA0F0A16B52C0FA
:10A3D800A2F0A36BB1EC61F002500209026E040E08
:10A3E800526033D0350E0E6E0B0E0F6E5250050DA7
:10A3F800800EF324106E030EF420116E136A050EFE
:10A40800126EE9EC5DF03A0E0E6E0B0E0F6E5250A6
:10A41800130D000EF324106E030EF420116E136A50
:10A42800130E126EE9EC5DF04D0E0E6E0B0E0F6EF4
:10A4380052500D0D4C0EF324106E030EF420116EC5
:10A44800136A0D0E126EE9EC5DF0030E526409D02A
:10A45800010E506E01011B5110091B6F000EE8CF51
:10A4680036FB250E9AEC5AF0350E216E0B0E226E35
:10A47800000E246E250E236EFC0E256EFE0E266E33
:10A48800CAEC3AF002928390120001018C6B4E6A7A
:10A498007C6B7D6B020E8B6F83908A6B896B526A23
:10A4A800030E526401D049D052500C0D030EF32410
:10A4B800D96E020EF420DA6EDF6A52500C0D020ECD
:10A4C800F324D96E020EF420DA6EDF6A52500C0DB6
:10A4D800000EF324D96E020EF420DA6EDE6ADD6A0D
:10A4E80052500C0D040EF324D96E020EF420DA6ECD
:10A4F800DE6ADE6ADE6ADD6A52500C0D0B0EF3244A
:10A50800D96E020EF420DA6E100EDF6E52500C0D6A
:10A518000A0EF324D96E020EF420DA6E020EDF6EF4
:10A5280052500C0D080EF324D96E020EF420DA6E88
:10A53800240EDE6EDD6A522AB3D7100E02010B6FAD
:10A54800020E0A6F096B240E086F526A0101886BAC
:10A55800120052501C0D070EF324D96E010EF42080
:10A56800DA6E000EDE24C76F010EDE20C86F000E03
:10A57800DE20C96F000EDE20CA6F000EDE20CB6F12
:10A58800000EDE20CC6F000EDE20CD6F000EDE2028
:10A59800CE6F52501C0D070EF324D96E010EF42015
:10A5A800DA6EC7C0DEFFC8C0DEFFC9C0DEFFCAC0A2
:10A5B800DEFFCBC0DEFFCCC0DEFFCDC0DEFFCEC0ED
:10A5C800DEFF52501C0D070EF324D96E010EF42045
:10A5D800DA6EDECFCFF0DECFD0F0DECFD1F0DECF37
:10A5E800D2F05250220D380EF3249E6F020EF42042
:10A5F8009F6FCFC0A0F0D0C0A1F0D1C0A2F0D2C050
:10A60800A3F05EEC12F0D36FD35103E0010E506E4D
:10A61800010C506A1200C4C0D9FFC5C0DAFFDECFF2
:10A62800C6F0DDCFC7F0C4C0B8F0C5C0B9F0000EA1
:10A63800BB6F010EBA6F06EC51F0C86FC85147E105
:10A64800C6C03AF0C7C03BF020EE16F0C451D92678
:10A65800C551DA22DECF3CF0DECF3DF0DECF3EF052
:10A66800DECF3FF071EC55F00001C86FC8512FE103
:10A6780020EE1AF0C451D926C551DA22DECF0EF0E9
:10A68800DDCF0FF0116A106A136A200E126E28ECE3
:10A6980061F0000120EE1AF0C451D926C551DA2222
:10A6A800DECF0EF0DDCF0FF01C0EC425106E000EAD
:10A6B800C521116E136A0B0E126E2BEC5EF020EEA4
:10A6C80003F0C651D926C751DA22010EDF6EC851F0
:10A6D800120052501C0D070EF324D96E010EF420FF
:10A6E800DA6EDECFF0F0DECFF1F0DECFF2F0DECFC3
:10A6F800F3F0DECFF4F0DECFF5F0DECFF6F0DECF0C
:10A70800F7F0F1C0F0F0F2C0F1F0F3C0F2F0F4C0ED
:10A71800F3F0F5C0F4F0F6C0F5F0F7C0F6F000017C
:10A72800F76BF0C0F8F0F1C0F9F0F2C0FAF0F3C03E
:10A73800FBF0B0EC3CF0FE6FFE5102E0FE5112005F
:10A748008FB414D05250220D380EF3249E6F020E8F
:10A75800F4209F6F000EA06F040EA16F010EA36F6F
:10A76800A26BFC0EA46FCEEC08F0FF6FFF510BE05C
:10A77800290E9C6FFD0E9D6FFFC09EF09F6BB1EC84
:10A7880061F0FF511200ADEC52F0000C8380838E13
:10A79800000E0E6E040E0F6E116AF60E106E010E8C
:10A7A800136E126AD2EC48F0100E00019C6FFE0E78
:10A7B8009D6FB1EC61F0CB6BCC6BCBC04BF0010E55
:10A7C8004B164B324B3283504B187F0B4B18836E12
:10A7D8002E0E9BEC61F08FB415D05250220D380E1E
:10A7E800F32400019E6F020EF4209F6F000EA06FED
:10A7F800040EA16F010EA36FA26BC80EA46FCEEC5E
:10A8080008F0CA6F0001CA5109E04B0E9C6FFF0E99
:10A818009D6FCAC09EF09F6BB1EF61F0CB4BCC2B04
:10A82800CCBFCBD7CC5103E1640ECB5DC6E3F20EAF
:10A838009C6FFE0E9D6FB1EC61F0839E83908390B8
:10A84800506A1200090E186E0F5010103BE00FC02E
:10A85800D9FF10C0DAFFDE50DE1034E00FC0D9FF98
:10A8680010C0DAFFDECF12F0DDCF13F012C0D9FF2F
:10A8780013C0DAFFDF5026E00FC0D9FF10C0DAFF9F
:10A8880010EE05F0DE50E126DD50E22220EE02F067
:10A898000F50D9261050DA22E650DE1813E1E650A0
:10A8A800DE1810E10FC0D9FF10C0DAFF10EE01F07A
:10A8B800DE50E126DD50E222E750D4EC61F0126E62
:10A8C80012A0186A185003E0166A176A08D00FC059
:10A8D800D9FF10C0DAFFDECF16F0DDCF17F0115028
:10A8E800D96EDA6A16C0DEFF17C0DDFF18501200F5
:10A8F80020EE03F00E50D9260F50DA22DF50166EE4
:10A90800176A186A196A20EE02F00E50D9260F50FD
:10A91800DA22DF5016C013F017C014F018C015F073
:10A92800126A1210166E1350176E1450186E1550C6
:10A93800196E20EE01F00E50D9260F50DA22DF50A2
:10A9480016C013F017C014F018C015F0126A1210D0
:10A95800166E1350176E1450186E1550196E0EC0DF
:10A96800D9FF0FC0DAFFDF5016C013F017C014F07C
:10A9780018C015F0126A1210166E1350176E145084
:10A98800186E1550196E16C00EF017C00FF018C0CB
:10A9980010F019C011F01200256E2550D8A4040C2F
:10A9A8002350241001E1040C55B0030C53B608D011
:10A9B800090ED8901F36203621362236E82EF9D7D0
:10A9C800245006E1020E235C03E2276A110E02D02E
:10A9D800276A120E266E26C028F01FC017F020C066
:10A9E80018F021C019F022C01AF028505CEC5FF072
:10A9F80000091DE11DC00EF01EC00FF0020E116E01
:10AA0800106A05EC5CF0000908E0020E1E26230619
:10AA1800D8A0240623502410EDE1120E281807E1CF
:10AA2800176A186A196A1A6A0C0E5CEC5FF0DEEC99
:10AA380061F023502410D8A4010C000C78EC5FF0CE
:10AA4800CC0E6BEC61F0660E6BEC61F04EEC61F0D5
:10AA5800276E275005E1216A226A236A246A1200B8
:10AA6800256A266A2550270FD96EDA6A4EEC61F0FE
:10AA7800DF6E254A262A26BEF5D7265003E1040EA6
:10AA8800255CF0E33C0E00019C6FFC0E9D6F27C017
:10AA98009EF09F6B28C0A0F0A16B29C0A2F0A36B09
:10AAA8002AC0A4F0A56B27C0A6F028C0A7F029C02B
:10AAB800A8F02AC0A9F0B1EC61F02A50291028109A
:10AAC80003E1060E275CC7E327C021F028C022F067
:10AAD80029C023F02AC024F01200446A20EE2BF08B
:10AAE8003A50D9263B50DA223C50DE1809E13D5055
:10AAF800DE1806E13E50DE1803E13F50DE1839E06B
:10AB08003AC027F03BC028F068EC44F0446E44504B
:10AB180030E12F0E3A241D6E000E3B201E6E3CC005
:10AB28001FF03DC020F03EC021F03FC022F0246A53
:10AB3800010E236E20EE01F03A50D9263B50DA225E
:10AB4800DF50D0EC54F0000906E03C683D683E68F0
:10AB58003F68010E446E20EE2BF03A50D9263B5048
:10AB6800DA223CC0DEFF3DC0DEFF3EC0DEFF3FC054
:10AB7800DEFF4450120003D00E4A0F2A102A10504C
:10AB8800D96EDA6ADF50116E0EC0F6FF0FC0F7FFFC
:10AB9800000EF86E0E0EF76403D00800F55005D0CD
:10ABA800F6CFE9FFF7CFEAFFEF50111813E10EC017
:10ABB800F6FF0FC0F7FF000EF86E0E0EF76403D015
:10ABC8000800F55005D0F6CFE9FFF7CFEAFFEF50C0
:10ABD8000009D2E10EC0F6FF0FC0F7FF000EF86EB5
:10ABE8000E0EF76403D00800F55005D0F6CFE9FF44
:10ABF800F7CFEAFFEF50116E1050D96EDA6ADF50C6
:10AC0800115C0E6E0F6AD8A00F06120001091220FF
:10AC1800010001001700002D119420D00F00010140
:10AC2800091220010001001700002D119420D00FF7
:10AC3800000101091220010001001700002D1194E4
:10AC480020D00F00010109122001000100170000A7
:10AC58002D119420D00F000100004F01000F0000BB
:10AC6800000009FF0000004F01000F00000000096C
:10AC7800FF0000004F01000F0000000009FF000066
:10AC8800004F01000F0000000009FF00800102E8EA
:10AC980005800102E805800102E805800102E80557
:10ACA800175018100AE174C117F075C118F0175041
:10ACB800181003E1176A186A120017C012F018C0BA
:10ACC80013F019C014F04CEC5EF012501726135014
:10ACD800182217C0D9FF18C0DAFFDF5006E10101BA
:10ACE800746B756B176A186A120017C012F018C0D7
:10ACF80013F019C014F06CEC5EF012501724010127
:10AD0800746F13501820756F74C1D9FF75C1DAFFBD
:10AD1800DF5009E074C1D9FF75C1DAFF000EDF6AA0
:10AD2800744B752B02D0746B756B17C017F018C075
:10AD380018F01200A96BAA6B9FC0ABF0A0C0ACF0D2
:10AD4800A107D8A0A20727D0A3C074F0A4C075F0AB
:10AD5800A50E766F776B796B010E786FB10E7A6FEF
:10AD68007B6BF4EC17F0B105B2111EE1A551AD6F84
:10AD7800AE6BAF6BB06BABC0D9FFACC0DAFFADC088
:10AD8800DFFFAB4BAC2BA94BAA2B0A0EAD19AE11AA
:10AD9800AF11B01109E0A151A95DAA51800A4B6E0B
:10ADA800A251800A4B58D0E3ABC0D9FFACC0DAFF40
:10ADB800DF6AA951AA1103E19F6BA06B12009FC023
:10ADC8009FF0A0C0A0F01200B3C0B7F0B4C0B8F0B4
:10ADD800B70E0E6E08EC47F00EC0BBF00FC0BCF00B
:10ADE8000001BCBF0B0CD890BB35D96EBC35DA6EF0
:10ADF800820ED926010EDA22DECFB9F0DDCFBAF005
:10AE0800B951BA1105E0B9C0D9FFBAC0DAFFDF6A93
:10AE1800B151B21105E0B1C0D9FFB2C0DAFFDF6AA3
:10AE2800D890BB35D96EBC35DA6E820ED926010EA4
:10AE3800DA22B1C0DEFFB2C0DDFFB55101E1000C7E
:10AE4800B30E7C6FB10E7D6F7E6B7F6BAFEC00F045
:10AE58000001B66FB65112000EC015F00FC016F003
:10AE680010C017F011C018F01206D8A01306122847
:10AE78000CE113280AE10E6A0F6A1200154A162A15
:10AE8800174A182A1206D8A0130615C0F6FF16C0CE
:10AE9800F7FF0800F55015E017C0D9FF18C0DAFF12
:10AEA800DF500FE0125013100CE017C0D9FF18C084
:10AEB800DAFF15C0F6FF16C0F7FFDE500900F518D7
:10AEC800DDE015C0F6FF16C0F7FF0800F5CF14F057
:10AED80017C0D9FF18C0DAFFDF50145C0E6E0F6A76
:10AEE800D8A00F061200296E39D020EE01F02550A7
:10AEF800D9262650DA22DF502D6E20EE03F0255099
:10AF0800D9262650DA22DF502C6E20EE05F0255087
:10AF1800D9262650DA22DF502B6E20EE07F0255076
:10AF2800D9262650DA22DF502A6E2AC011F02BC00B
:10AF380012F02CC013F02DC014F0B3EF5CF025C054
:10AF48000EF026C00FF08BEC3EF00EC02AF00FC0BA
:10AF58002BF010C02CF011C02DF0E7D72950276E28
:10AF6800286A2850D8A412002750010ABEE0030A14
:10AF7800E6E0120025EE04F0DE50DE10FBE000C52E
:10AF880016F001C517F0060E1624D96E050E172007
:10AF9800DA6EDF50146E060E1624D96E070E1720CF
:10AFA800DA6EDF50156E164A172A1068010E116EF8
:10AFB80016C012F017C013F01050121611501316C5
:10AFC80012C000F513C001F5F29E25EE04F0DE066E
:10AFD800000EDD5AF28E0EC0D9FF0FC0DAFF15C081
:10AFE800DFFF25EE04F0010EDBBE05D0000EDE5CAF
:10AFF800010EDE5801E2898214501200115002E05D
:10B00800115003E10F5090EF61F01150D96EDA6AD8
:10B01800040ED926DE50DE1014E01150D96EDA6A1B
:10B02800040ED9261150E16EE26A020EE126DE50C6
:10B03800E65CE650800A166EDE50800A1658D8B0D4
:10B0480012001150D96EDA6A020ED926DECF12F03C
:10B05800DDCF13F01150D96EDA6ADECF14F0DDCFF0
:10B0680015F012501424D96E13501520DA6E0FC043
:10B07800DFFF1150D96EDA6A020ED926DE2A000ED9
:10B08800DD22000C980E00019C6FFD0E9D6F7EC1A5
:10B098009EF07FC19FF0B1EC61F011D0030E0BD090
:10B0A800050E236E01017E6B7F6B2DD00A0E03D037
:10B0B800010E01D0020E236E26D0236A24D07EC151
:10B0C80021F07FC122F0225009E0020A0DE00E0AA9
:10B0D8000FE0010A11E02A0A13E0EFD721500A0A0B
:10B0E800DDE01E0ADDE0E9D72150BC0AE3E0E5D740
:10B0F80021501C0ADBE0E1D72150AC0AD9E0DDD7AA
:10B1080021500F0ADAE1235012000E501202F3CF39
:10B1180016F0F4CF17F0186A196A0E501302F3509C
:10B128001726F4501822000E19220F501202F3505D
:10B138001726F4501822000E19220E501402F3504C
:10B148001826F45019220F501302F3501826F45001
:10B15800192210501202F3501826F45019221550D3
:10B168000E02F35019260F501402F35019261050EE
:10B178001302F350192611501202F350192616C063
:10B188000EF017C00FF018C010F019C011F012001F
:10B19800150E146EC60EE82EFED7142EFCD700D05E
:10B1A80020D0150E146EC60EE82EFED7142EFCD72E
:10B1B80000D0010E0E6E12C0F6FF13C0F7FF000E8E
:10B1C800F86E0E0EF76403D00800F55005D0F6CFE0
:10B1D800E9FFF7CFEAFFEF5056EC5DF0124A132A69
:10B1E800D7D712C0F6FF13C0F7FF000EF86E0E0E89
:10B1F800F76403D00800F55005D0F6CFE9FFF7CF84
:10B20800EAFFEF500009CDE11200286A296A01011E
:10B21800996B2A6A2FD0A3EC5DF0215022101FE011
:10B228002A0E0E6E0F6ABEEC57F0276E2AA80BD0B6
:10B23800D20E00019C6FFE0E9D6F27C09EF09F6B83
:10B24800B1EC61F00CD0000E01019925D96EDA6AD3
:10B25800040EDA2227C0DFFF992B284A292A2AAAB6
:10B2680007D0000E2824256E040E2920266E120011
:10B278008EAC02D02904CFE328C025F029C026F0DF
:10B288001200166A176A186A196A125013101410F5
:10B29800151029E0010E1A6E06D0D8901236133612
:10B2A800143615361A2A15AEF8D7D890163617362A
:10B2B8001836193612500E5C13500F581450105887
:10B2C8001550115809E312500E5E13500F5A1450BE
:10B2D800105A1550115A1680D8901532143213325C
:10B2E80012321A2EE2D716C00EF017C00FF018C08F
:10B2F80010F019C011F012001A0E17240E6E000E6D
:10B3080018200F6EC9EC5FF00EC01DF00FC01EF0C4
:10B318001F6A206A15C0D9FF16C0DAFF030EDE18AF
:10B328001CE1140E17240E6E000E18200F6EC9ECC7
:10B338005FF00E50196E0F501A6E1B6A1C6A1AC005
:10B348001CF019C01BF01A6A196A19501D121A50FC
:10B358001E121B501F121C5020121DC015F01EC0BB
:10B3680016F01FC017F020C018F01200166E0C0E51
:10B37800161807E0DEEC61F078EC61F0000901E1F5
:10B38800FF0C16504009C4EC61F01350C4EC61F096
:10B398001250C4EC61F01150C4EC61F01050C4ECD0
:10B3A80061F0010E156E165002E1950E156E080E2D
:10B3B800161802E1870E156E1550C4EC61F00C0EDC
:10B3C800161802E1CDEC61F00A0E156ECDEC61F0B5
:10B3D800146E14AE02D0152EF9D714501200125064
:10B3E8001310D8B4000C12C0D9FF13C0DAFFDF5015
:10B3F80001E1000C12C00EF013C00FF00AEC5EF071
:10B408000EC014F00FC015F0020E1418151001E04C
:10B41800000C160E0E6E12C0D9FF13C0DAFFDF50F3
:10B42800DCEC5CF00009D8B4000C170E0E6E20EEB0
:10B4380001F01250D9261350DA22DF50DCEC5CF010
:10B44800000901E1000C1638F00B17101200106EFD
:10B45800D10EF66EF80EF76E0900F550105C2CE36D
:10B46800D20EF66EF80EF76E10500900F55C04E384
:10B478000F6A010E0E6E010CD30EF66EF80EF76E03
:10B488000900F550105C08E3D40EF66EF80EF76E5E
:10B4980010500900F55CECE2D50EF66EF80EF76E6A
:10B4A8000900F550105C08E3D60EF66EF80EF76E3C
:10B4B80010500900F55CDCE20E6A0F6A1200866A19
:10B4C800846A8B6889680101996B83928394866B7F
:10B4D800876B09D0000E8625D96E040E8721DA6E97
:10B4E800DF6A864B872B87BFF5D78705F3E3866B23
:10B4F800876B09D0350E8625D96E0B0E8721DA6E3B
:10B50800DF6A864B872B87BFF5D78705F3E30F01E3
:10B518001769D6501F0B4009D66ED6980F0ED61253
:10B52800D588D5120E01C29BD58E0F0C016E000076
:10B538000BEE35F08490849A1390F29E83A4FED784
:10B5480089688EA8FED701041AE0EE50866E861E22
:10B558008B6A8EA2FED789908EB2FED78EA4FED7B4
:10B568008980898A8EB4FED7012EEDD78B68F90EB3
:10B57800896E129012981380F28E015012008EA2DA
:10B58800FED702B2899AEE50866E861E8B6AE3D782
:10B598000000032EFDD7000C0EC015F00FC016F0EA
:10B5A80010C017F011C018F015C0D9FF16C0DAFF87
:10B5B800DF50146E17C0F6FF18C0F7FF000EF86EC4
:10B5C8000E0EF76403D00800F55005D0F6CFE9FF5A
:10B5D800F7CFEAFFEF50145C196E1A6AD8A01A0662
:10B5E800174A182A154A162A1206D8A01306125006
:10B5F800131003E019501A10D7E019C00EF01AC042
:10B608000FF012000EC0D9FF0FC0DAFF10C0DFFF25
:10B618000E4A0F2A1150106E1250116E1350126EEE
:10B62800136A0EC0D9FF0FC0DAFF10C0DFFF0E4A41
:10B638000F2A1150106E1250116E1350126E136AA9
:10B648000EC0D9FF0FC0DAFF10C0DFFF0E4A0F2A65
:10B658001150106E1250116E1350126E136A0EC0F4
:10B66800D9FF0FC0DAFF10C0DFFF0E4A0F2A120001
:10B67800838002500209026E88050DE1000EE8CFB2
:10B6880035FB500EE8CF36FB000EE8CF37FBE8CF8E
:10B6980038FB886B1AD02BEE35F089C1DFFF000E1E
:10B6A800E8CF36FB0D0EE8CF37FB000EE8CF38FBAE
:10B6B8008FA403D0600EE8CF38FB8FA406D037CB19
:10B6C8000EF0200E0E120EC037FB040E9AEC5AF044
:10B6D80002920101896B83901200526A030E526430
:10B6E80001D02AD052500C0D030EF324D96E020E4D
:10B6F800F420DA6EDF6A52500C0D020EF324D96E74
:10B70800020EF420DA6EDF6A52500C0D000EF3249C
:10B71800D96E020EF420DA6EDE6ADD6A52500C0D24
:10B72800040EF324D96E020EF420DA6EDE6ADE6AA5
:10B73800DE6ADD6A522AD2D7526A83908B6B120076
:10B74800125013101410151023E0010E166E06D0B7
:10B75800D8901236133614361536162A15AEF8D781
:10B7680012500E5C13500F581450105815501158A1
:10B7780008E312500E5E13500F5A1450105A155009
:10B78800115AD8901532143213321232162EE8D7C5
:10B798000EC00EF00FC00FF010C010F011C011F065
:10B7A8001200526A0E6A0F6A52501C0D070EF324DB
:10B7B800D96E010EF420DA6E070EDE6AE806FDE2A5
:10B7C80052501C0D1B0EF324D96E010EF420DA6EB4
:10B7D800DF6A52501C0D170EF324D96E010EF420A7
:10B7E800DA6EDE6ADE6ADE6ADD6A0E4A0F2A0FBE8C
:10B7F800DBD70F5003E1040E0E5CD6E38390506A4A
:10B808001200070E136ED00E126E0FD0CDEC61F041
:10B81800146E14280DE1E40E00D000D0E82EFCD7F9
:10B8280000D000D01206D8A0130612501310EEE173
:10B83800FE0E141801E0000CCDEC61F00EC0D9FF2B
:10B848000FC0DAFFDF6E0E4A0F2A1006D8A01106C5
:10B8580010501110F1E1CDEC61F0CDEC61F0010C6C
:10B868000EC014F00FC015F013D01206D8A013069E
:10B8780010C0D9FF11C0DAFF104A112A14C0E1FF25
:10B8880015C0E2FF144A152ADFCFE7FFE7500BE0A7
:10B898001250131008E0E9D714C0D9FF15C0DAFF19
:10B8A800DF6A144A152A1206D8A013061228F4E1F2
:10B8B8001328F2E1120093EC5FF0000901E1000C9B
:10B8C8001250C4EC61F0FD0E12181EE0020E146E48
:10B8D800136A10C0D9FF11C0DAFFDF50C4EC61F061
:10B8E800104A112A1306D8A0140613501410F1E1B7
:10B8F800CDEC61F0CDEC61F0CDEC61F0156E15503A
:10B908001F0B050A01E0000C010C15D00FC0F6FF53
:10B9180010C0F7FF000EF86E0E0EF76403D0080093
:10B92800F55005D0F6CFE9FFF7CFEAFFEF509BECD3
:10B9380061F00F4A102A0FC0F6FF10C0F7FF000E83
:10B94800F86E0E0EF76403D00800F55005D0F6CF58
:10B95800E9FFF7CFEAFFEF500009D8E1120011C064
:10B9680015F012C016F013C017F014C018F078ECD8
:10B978005FF0CC0E6BEC61F0990E6BEC61F00C0E85
:10B988006BEC61F0196A1A6A1950150FD96EDA6AE8
:10B99800DF506BEC61F0194A1A2A1ABEF5D71A5013
:10B9A80002E078EF5FF0040E195CEEE378EF5FF0E9
:10B9B8000F6E0E5001E1000C2F0E0F6409D03A0EE5
:10B9C8000F6006D00E50D96EDA6A0F50D00F17D01C
:10B9D800400E0F6409D0470E0F6006D00E50D96E86
:10B9E800DA6A0F50C90F0BD0600E0F64000C670E97
:10B9F8000F60000C0E50D96EDA6A0F50A90FDF6E77
:10BA0800010C226ED90E236EF80E246E216A0AD01C
:10BA180023C0F6FF24C0F7FF234A242A0800F55064
:10BA2800F7E1212A2250211807E023C0F6FF24C09D
:10BA3800F7FF0800F550ECE11E0E00019C6FFE0EAA
:10BA48009D6F22C09EF09F6B23C0A0F024C0A1F080
:10BA5800B1EF61F0106ECD0EF66EF80EF76E0900BC
:10BA6800F550105C1CE3CE0EF66EF80EF76E105013
:10BA78000900F55C04E30F6A010E0E6E010CCF0E8F
:10BA8800F66EF80EF76E0900F550105C08E3D00E5C
:10BA9800F66EF80EF76E10500900F55CECE20E6ACF
:10BAA8000F6A12000F6E87920A0EE82EFED700D09A
:10BAB8000EB002D0879401D08784000E116E010E5B
:10BAC800106E0FAE02D0838A01D0839AD8900F36B9
:10BAD800879000F000F0878000F000F08790104A0F
:10BAE800112A11BEEED7115003E1090E105CE9E3EB
:10BAF80087821200010E0E6E0F6A888687828784FD
:10BB080000F000F0879400F000F0106A116A8DA62A
:10BB180002D00E500F12D8900E36879000F000F029
:10BB2800878000F000F08790104A112A11BEEFD7E5
:10BB3800115003E1030E105CEAE30F50120025EEEA
:10BB480004F0010EDBBE05D0000EDE5C010EDE58EF
:10BB580001E2898225EE04F0010EDBBE0FD0DE285B
:10BB6800010EDE580BE31C0E00019C6FFF0E9D6F4B
:10BB780004C59EF005C59FF0B1EC61F004C521F045
:10BB880005C522F012009F0E166E176814C018F033
:10BB980015C019F01650182617501922195005E12A
:10BBA8001A0E185C02E2010E01D0000E1A6E1B6A12
:10BBB8001A501B1005E05F0E1414146E156A12005B
:10BBC80014C014F015C015F0120010C016F011C002
:10BBD80017F00EC014F00FC015F010D016C0D9FF22
:10BBE80017C0DAFFDF50186E164A172A14C0D9FF9B
:10BBF80015C0DAFF18C0DFFF144A152A1206D8A0AC
:10BC080013061228EBE11328E9E112000EC010F028
:10BC18000FC011F002D00E4A0F2A0EC0F6FF0FC057
:10BC2800F7FF000EF86E0E0EF76403D00800F5500B
:10BC380005D0F6CFE9FFF7CFEAFFEF500009EBE1B7
:10BC480010500E5C0E6E11500F580F6E12000EC081
:10BC580014F00FC015F010C016F011C017F01250F4
:10BC68001310D8B4120016C0D9FF17C0DAFF14C0D9
:10BC7800E1FF15C0E2FFDFCFE7FF164A172A144A93
:10BC8800152A1206D8A0130612501310ECE1120060
:10BC9800156A166A04D0124A132A154A162A12C0BF
:10BCA800D9FF13C0DAFFDF500EE014C00EF012C047
:10BCB800D9FF13C0DAFFDF500F6E106A15EC61F080
:10BCC8000E500F10E8E115C012F016C013F0120064
:10BCD800156A166A04D0124A132A154A162A12C07F
:10BCE800D9FF13C0DAFFDF500EE014C00EF012C007
:10BCF800D9FF13C0DAFFDF500F6E106A15EC61F040
:10BD08000E500F10E8E015C012F016C013F0120024
:10BD18001A0E14240E6E000E15200F6E16C010F0A9
:10BD280017C011F0EEEC60F012C0D9FF13C0DAFFB3
:10BD3800030EDE18D8A41200140E14240E6E000E82
:10BD480015200F6E18C010F019C011F0EEEF60F05A
:10BD58008B6B8380838E000E0E6E040E0F6E116A3D
:10BD6800F60E106E010E136E126AD2EC48F0100E29
:10BD780000019C6FFE0E9D6FB1EC61F0F20E9C6F9E
:10BD8800FE0E9D6FB1EC61F0839E839012000E6EE3
:10BD98000E500EE0E5EC61F0200EE82EFED7E8EC40
:10BDA80061F0CC0E00D0E82EFDD700D000D01200F4
:10BDB800E5EC61F0C00E00D0E82EFDD7E8EC61F0AC
:10BDC800350EE82EFED700F012006DC049F06EC0A7
:10BDD8004AF01BEC45F0716F715112E16DC00FF024
:10BDE8006EC010F06F0E116E26EC54F00001716FEA
:10BDF800715106E16DC0D9FF6EC0DAFFDE6ADD6AF7
:10BE080071511200800E826F7CC083F07DC084F077
:10BE1800856B866B876B886B830E766F7EC077F039
:10BE28007FC078F0820E796F23EC05F00001855110
:10BE38007C25D96E86517D21DA6EDF6A000C000EF2
:10BE4800F2BE010E116E0F50030B7F6E0EC07EFF07
:10BE580010C080FF3F0E81168184F29E550E826EBF
:10BE6800AA0E826E818281B2FED7819411B002D06F
:10BE7800F29E01D0F28E120002D00E4A0F2A0EC096
:10BE8800F6FF0FC0F7FF0800F55009E00EC0F6FFF7
:10BE98000FC0F7FF0800F55010181110EEE10EC0A2
:10BEA800F6FF0FC0F7FF0800F5500E6E0F6A12007C
:10BEB8001B6E1BAE0ED01B9E106A116A126A136AA3
:10BEC800370EBAEC59F01C6E010E1C6402D01C50DF
:10BED800120017C010F018C011F019C012F01AC0E3
:10BEE80013F01B50BAEF59F0E5EC61F00A0E0F6E33
:10BEF800F80EE82EFED70F2EFCD700D0E8EC61F044
:10BF0800E00E00D0E82EFDD7BBEC61F0090E0F6EF5
:10BF1800840EE82EFED70F2EFCD7E8EF61F0130E43
:10BF28000F6E880E0E6E0ED0CDEC61F0FF0A0DE09C
:10BF3800E40E00D000D0E82EFCD700D000D00E06CA
:10BF4800D8A00F060E500F10EFE10E500F10D8A416
:10BF5800010C000C010E146E200E0E180F1011E0CB
:10BF6800F70E106E11680EC012F00FC013F01050CB
:10BF7800122611501322135003E1050E125C01E33F
:10BF8800146A14C00EF00F6A120020EE01F00E5071
:10BF9800D9260F50DA22DF50136E146A0EC0D9FF6B
:10BFA8000FC0DAFFDF50106E1350116E1050136E71
:10BFB80011C014F013C00EF014C00FF012006090FE
:10BFC8000F0E0F01596F070E396F356F4F0E936EB5
:10BFD8008A6A8A888A828A82010E8F6E130E0E01FF
:10BFE800B76F0F0EFA6F100EFC6F140EB86F140CAB
:10BFF8009F0E106E1168200E0E10126E000E0F109C
:10C00800136E1050122611501322135005E11A0E08
:10C01800125C02E2010E01D0000E0E6E0F6A1200D1
:10C0280021BE04D021500FE120040DE220C022F0EF
:10C0380021C023F0221E231E224A232A22C020F0D8
:10C0480023C021F0120020C020F021C021F01200EE
:10C058001B6A1C6A09D01AC00FF0106A19C011F0C7
:10C0680002EC58F01B4A1C2A1B501724D96E1C508E
:10C078001820DA6EDF501A6E1A50EDE11200350EF4
:10C088000E6E0B0E0F6E116A106A010E136E126A95
:10C09800D2EC48F0010EE8CF35FB02500209026EDF
:10C0A800010E9AEC5AF0029212009F0E106E11685F
:10C0B8000EC012F00FC013F01050122611501322A8
:10C0C800135005E11A0E125C02E2010E01D0000EB7
:10C0D8000E6E0F6A1200BF0E106E11680EC012F0BD
:10C0E8000FC013F01050122611501322135005E1FF
:10C0F8001A0E125C02E2010E01D0000E0E6E0F6ADB
:10C108001200D00E106E11680EC012F00FC013F09E
:10C118001050122611501322135005E10A0E125C1A
:10C1280002E2010E01D0000E0E6E0F6A12009F8609
:10C138009E84090E0E01FD6F9F98890E9B6E9C6A66
:10C148009E989D8E9D889D9AC599F28AF28E9E90A2
:10C158009D9C9E9A9E8A1200350E0E6E0B0E0F6ED7
:10C16800116A106A010E136E126AD2EC48F02BEEB7
:10C1780035F08BC1DFFF010E9AEC5AF001018B6B91
:10C188001200136A110E126E09D00A0EE82EFED79D
:10C1980000D0010E0E6E200E56EC5DF01206D8A0EF
:10C1A80013061228F2E11328F0E112000E6E0E5069
:10C1B80009E0966A4F0E936E220E966E400E956EAB
:10C1C800968A400C966A100E966E2A0E966E900EFF
:10C1D800936EF4D70EC0D9FF0FC0DAFF10C0DFFF8F
:10C1E8000E4A0F2A11C010F0116A0EC0D9FF0FC0F5
:10C1F800DAFF10C0DFFF0E4A0F2A1200E5EC61F0EB
:10C20800200EE82EFED7E8EC61F0300EE82EFED7BF
:10C21800BBEC61F00F6EB00E00D0E82EFDD70F50CA
:10C2280012000E50D96EDA6A0F50DE1804E10EC003
:10C238000EF00F6A12000E2A0E04D96EDA6ADF5069
:10C24800F0E10E6A0F6A12000EC014F00FC015F06C
:10C2580014C0D9FF15C0DAFF10C0DFFF144A152A31
:10C268001206D8A0130612501310F2E11200070E9E
:10C278008C6E9150070B0E6E888A8DAA02D0080E1C
:10C288000E26020E0101921903E10E1C0F0B0E6E11
:10C298000E501200106A116AD890103202EC61F048
:10C2A800000901E0108E112A070E1164F5D710500D
:10C2B8001200000EE8CF00F5E8CF01F5E8CF02F54F
:10C2C800E8CF03F5E8CF04F5E8CF05F5000C0F6ECD
:10C2D800106A0F50010BCBEC5EF0D8900F32102A89
:10C2E800070E1064F6D7070CEFEC61F0CDEC61F0A7
:10C2F80093EC5FF0000901E0010CDEEC61F0000C4A
:10C308000F50030B7F6E0EC07EFF3F0E811681809B
:10C3180000F000F0805012000E6E03D0F1EC61F0D6
:10C3280004000E01CDA9FAD70EC09AFF12000E6EB6
:10C3380003D0F1EC61F004000E01CDA9FAD70EC0CC
:10C348009AFF120068706469736B2E636667004811
:09C358005039313231440000007B
:10C362009E0E206E9CC01BF09DC01CF0200E1D6E08
:10C3720020EF23F088888DA803D0010E0E6E01D025
:10C382000E6A0E5012000E6E0EC092FF0E01CDA16B
:10C39200FDD7CD919250120092680E01CDA1FDD72A
:10C3A200CD91925012000E6E0E5001E0010C5550CC
:10C3B20012008380506A83901200EDEC61F0CDEFA1
:10C3C20061F083908B6B1200839888981200839897
:10C3D20088881200350B1FE78580120085901200B5
:03C3E20012000145
:10F8CC0000819FE0FC407E80FC000020004F4B003C
:10F8DC004449534B5F455252004E4F545F52454181
:10F8EC004459004E4F5F46494C45004E4F545F4FB4
:10F8FC0050454E4544004E4F545F454E41424C4599
:10F90C0044004E4F5F46494C455F53595354454D47
:10F91C0000000D0A2025325820253258202532733C
:10F92C002025327320253273202532732025327323
:10F93C002025327320253273202532732025347311
:10F94C0020253473202534732025347320253473FB
:10F95C0020253473202534732025347320000D0AA0
:10F96C0048504469736B204D6B204949202831382D
:10F97C004634364B343029202573202573202573CB
:10F98C00205374617274696E672E2E2E0D0A000D51
:10F99C000A4469736B6E6F3A2025642C20726F7762
:10F9AC00206469736B6E6F3A202564202C20696487
:10F9BC00783A202564000D0A4461746120706F72DE
:10F9CC0074206973202558202D2053686F756C6442
:10F9DC00206265203C3E2030784646000D0A536577
:10F9EC00656B20657272202564203E2025642C20D6
:10F9FC002564203E2025642C202564203E2025648F
:10FA0C00000D0A53746174757320706F72742069E1
:10FA1C0073202558202D2053686F756C6420626507
:10FA2C002030784646000D0A4461746120706F7274
:10FA3C0074206973202558202D2053686F756C64D1
:10FA4C002062652030784646000D0A5264207520ED
:10FA5C0025642072746E2025642C20256420627924
:10FA6C0074657320726561640D0A000D0A4D61782E
:10FA7C0020566563746F72206469736B2025642053
:10FA8C00256C642028256C582920000D0A44736BC2
:10FA9C0073656C2069732025642C206E756D62650E
:10FAAC007220697320256420000D0A2530325825F8
:10FABC003032582053533830783A4465736372208F
:10FACC00752025642000466F756E6420616E20528F
:10FADC0054432066696C652061742025580D0A001A
:10FAEC004C6F6F6B696E6720666F7220616E20526F
:10FAFC0054432066696C650D0A000D0A5573696ED6
:10FB0C0067206469736B2067656F6D65747279200B
:10FB1C002573200046696E6446696C6520666169D0
:10FB2C006C6564207365617263680D0A000D0A537D
:10FB3C00746174757320706F72742069732025580A
:10FB4C00202D204F4B000D0A5365656B20746F20E0
:10FB5C00256C64206661696C6564202564000D0A5F
:10FB6C0057726974655F736563746F727320666135
:10FB7C00696C202564000D0A454550524F4D206498
:10FB8C0069736B206E756D626572202564000D0AB9
:10FB9C004469736B2073656C656374206E756D625C
:10FBAC006572202564005365656B696E6720746F00
:10FBBC0020736563746F722025580D0A0046696EB8
:10FBCC006446696C65206661696C65642072656168
:10FBDC00640D0A000D0A5472616E73706172656E69
:10FBEC007420756E697420255820000D0A4F7065BD
:10FBFC006E696E67206578697374696E672025730A
:10FC0C0020000D0A4461746120706F727420697356
:10FC1C00202558202D204F4B000D0A476F742025AE
:10FC2C006C7520202D20726573657474696E670085
:10FC3C0020255820255820255820255820256C751E
:10FC4C002020200A000D0A57726F746520646973B6
:10FC5C006B6E6F3A20256420000D0A576169746938
:10FC6C006E6720666F72206361726420003C696469
:10FC7C00656E743E20255820255820256420256467
:10FC8C00000D0A46696C65202573206973206F701E
:10FC9C00656E20000D0A7274635F726561642825BD
:10FCAC00642C255829000D0A4F70656E696E67200B
:10FCBC006E657720257320000D0A253032582530CB
:10FCCC003258204578697420004E6F742061204CA6
:10FCDC004946206469736B0D0A000D0A5265616414
:10FCEC0020646573637269626520000D0A46696C55
:10FCFC006520255820697320257320000D0A44695E
:10FD0C00736B20255820697320257320000D0A4839
:10FD1C00737420627974657332202564000D0A5760
:10FD2C0072697465206661696C202564000D0A5245
:10FD3C00656164696E67205254430D0A000D0A41D7
:10FD4C006D69676F2039313231440D0A000D0A5349
:10FD5C00532F38302039313232440D0A000D0A4409
:10FD6C00736B73656C20697320256420000D0A5237
:10FD7C00656164202564206279746573005665633F
:10FD8C00746F722069732025580D0A000D0A5353A5
:10FD9C003830657865632025642000222A2B2C3AA4
:10FDAC003B3C3D3E3F5B5D7C7F000D0A4F70656EBA
:10FDBC00696E672025732020000D0A446562756703
:10FDCC0020697320256420000D0A436C6F636B203F
:10FDDC00697320256420000D0A50726F746F2069BE
:10FDEC007320256420000D0A5265616420636F6ED8
:10FDFC0066696720000D0A46696C656E616D652049
:10FE0C00257320000D0A466F726D617474696E67FC
:10FE1C00200072633D25752046525F25730D0A0044
:10FE2C002A2A204E4F204449534B202A2A002A2AA2
:10FE3C0020566572696679202A2A000D0A73627948
:10FE4C0074657331202564000D0A417373657274F7
:10FE5C0020454F49000D0A4173736572742041545B
:10FE6C004E000D0A4E6F206361726420256400649D
:10FE7C00657363726962652E636667002F6C6966D1
:10FE8C00646174612E62696E000D0A257320255819
:10FE9C002025580D0A00EB769045584641542020F9
:10FEAC0020000D0A4D6F756E74696E6720004A75DF
:10FEBC006C2020382032303231000D0A41737365CA
:10FECC0072742050500020255820772041544E2029
:10FEDC00004C6F6164696E672E2E2E002A2A205208
:10FEEC005141202A2A00466D7420657869742000DF
:10FEFC004465736372696265000D0A5374617475AD
:10FF0C00730032313A35383A3332000D0A494431F4
:10FF1C00202558000D0A494432202558005B253213
:10FF2C00582025645D004572726F7220256400486C
:10FF3C00504469736B20004E6F20636172640072D1
:10FF4C00633D25642000556E6974203000556E6940
:10FF5C0074203100556E6974203200556E6974201E
:10FF6C00330044534B53454C004E414D45255800EE
:10FF7C004449534B2558000D0A44534A00464154FA
:10FF8C0033320044454255470050524F544F0052B3
:10FF9C006561647900202530325800302E323000F3
:10FFAC004946432000454F49200052454E200053FE
:10FFBC005251200044415620004E444143004E52C1
:10FFCC004644004641540052544300434C4B0025D8
:10FFDC00325800207C200044300044310044320070
:10FFEC004433004434004435004436004437002583
:03FFFC006300009F
:020000040020DA
:10000000FF0FFF0FFF0FFF0FFF0FFF0FFF0FFF0F80
:020000040030CA
:0C0000008CFFFFFC8EFFFFFFFFFFFFFFE7
:00000001FF
